:020000041000EA
:1000000000B5324B212058609868022188439860DF
:10001000D860186158612E4B002199600221596106
:100020000121F02299502B49196001219960352056
:1000300000F044F80222904214D00621196600F024
:1000400034F8196E01211966002018661A6600F04E
:100050002CF8196E196E196E052000F02FF8012189
:100060000842F9D1002199601B49196000215960AB
:100070001A491B48016001219960EB211966A021F2
:10008000196600F012F800219960164914480160C1
:100090000121996001BC002800D000471248134993
:1000A000086003C880F30888084703B5996A0420EC
:1000B0000142FBD001200142F8D103BD02B5186610
:1000C0001866FFF7F2FF186E186E02BD00000240BE
:1000D000000000180000070000035F00212200005C
:1000E000F4000018222000A00001001008ED00E03C
:1000F00000000000000000000000000074B24E7A12
:1001000000200420F7010010C3010010C5010010F9
:10011000C1010010C1010010C1010010C101001097
:10012000C1010010C1010010C1010010C701001081
:10013000C1010010C1010010C9010010CB01001065
:10014000CD010010CD010010CD010010CD01001037
:10015000CD010010CD010010CD010010CD01001027
:10016000CD010010CD010010CD010010CD01001017
:10017000CD010010CD010010CD010010CD01001007
:10018000CD010010CD010010CD010010CD010010F7
:10019000CD010010CD010010CD010010CD010010E7
:1001A000CD010010CD010010CD010010CD010010D7
:1001B000CD010010CD010010CD010010CD010010C7
:1001C00000BE00BE00BE00BE00BE00BE00F04BF888
:1001D000103800BEF2EB88715CF9001084F9001051
:1001E0003402001090A31AE700202149086006C8D5
:1001F00081F3088810471F48006800282FD10DA4FC
:100200000ECC002902D000F012F8F9E71A491B4A77
:10021000002000E001C19142FCD1194988471949E9
:1002200088471949884700BEFDE701C901C29A42C3
:10023000FBD3704784F90010C0000020081E002086
:10024000CC1601100000042000000420CC16011080
:1002500000100420001004200000000070470B482C
:1002600007F0AEFC0047EFF30580C0B27047000016
:1002700008ED00E0000000D0081E00201040002023
:10028000394C0010F91A0010654D00105756000047
:1002900006005250ABB36053D4F300100600525026
:1002A000861C0302E4F30010060052505422A29D63
:1002B000ECF3001005005250DE65F468CC16011016
:1002C000F8B5C0460448054B10B5834203D0044B33
:1002D000002B00D0984710BD081E0020081E0020EB
:1002E0000000000006480749091A8910CB0F591869
:1002F00010B5491003D0044B002B00D0984710BD17
:10030000081E0020081E00200000000010B5074C49
:100310002378002B09D1FFF7D5FF054B002B02D026
:10032000044800E000BF0123237010BD101F00200F
:1003300000000000F8E80010054B10B5002B03D0BA
:100340000449054800E000BFFFF7CCFF10BDC046E0
:1003500000000000141F0020F8E800105A2370B5B8
:1003600004001B4D037029000A22013008F0FCFA3A
:10037000290020000C310A220B3008F0F5FA290080
:10038000200018310A22153008F0EEFA290020006A
:1003900024310A221F3008F0E7FA2900200030310A
:1003A0000A22293008F0E0FA290020003C3114220A
:1003B000333008F0D9FA074B0122A364064B200022
:1003C000E3645023E252054B6365054BA36570BDA2
:1003D00090E900100C0008000500110048E8010039
:1003E00098E1DA190FB400B50A4BC3B09B7F002B1C
:1003F0000BD1802145AB4900449A02A8019307F034
:10040000A1FB02A9044808F0ADFC43B008BC04B04D
:100410001847C046842F0020ACF0001010B52748C4
:10042000FFF7E0FF264C27482100FFF7DBFF802184
:1004300025484900FFF7D6FF2448FFF7D3FF2100E6
:1004400023483239FFF7CEFF210022482839FFF731
:10045000C9FF210020481E39FFF7C4FF21001F48B3
:100460001439FFF7BFFF21001D480A39333CFFF75D
:10047000B9FF1C48FFF7B6FFA16D1B48FFF7B2FF9D
:1004800048231A48E15AFFF7ADFF4A231848E15ABA
:10049000FFF7A8FF4C231748E15AFFF7A3FF4E23AD
:1004A0001548E15AFFF79EFF50231448E15AFFF721
:1004B00099FF616D1248FFF795FF10BD0CEB00101E
:1004C000132A002040EB001058EB001074EB0010D2
:1004D00084EB00109CEB0010B4EB0010CCEB001090
:1004E000E4EB001000EC001010EC001028EC001001
:1004F00040EC001058EC001070EC001088EC00107C
:10050000A0EC0010F0B5C64600B508F037FCFF229D
:100510000021514808F022FAFF2200214F4808F03C
:100520001DFA062003F09AF9052003F097F904203C
:1005300003F094F9022003F091F9032003F08EF9FF
:100540000820D024402120221023002604278046A2
:10055000434D240661626262636267626062A16108
:10056000F2302E70A2616E706361AE70676103F04D
:10057000E7FD4346A7613B48A361EE7003F0E0FD51
:10058000394D2B681B785A2B62D03848FFF72AFF69
:10059000374CA3220021200008F0E0F9EFF3108788
:1005A00072B63448FFF71EFF802180204901000306
:1005B0000EF072F9304E3000FFF714FF2F48FFF7AE
:1005C00011FF2100802280205C39520000030EF0D0
:1005D0004BF93000FFF706FF87F310888022284C84
:1005E00029685200200008F0BFF9FFF717FF2548DF
:1005F000FFF7F8FE244DA16D28000BF013FC002836
:1006000003D12248FFF7EEFEFEE74A232800E15A15
:100610000CF0B6FD2800616D0CF010FC5023E25A7E
:10062000023BE15A28000CF0F5F948232800E15A72
:100630000CF0AEFA4C232800E15A0CF04FFD2800D4
:100640000CF0E6FD1248FFF7CDFE04BC9046F0BD6D
:100650001048FFF7C7FEC1E7103B0020303C0020E8
:10066000842F002088130000C0140020F8EF001031
:100670003C2A0020B8EF0010D0EF0010D8EF001097
:10068000E02900207CF00010582F002090F000108E
:10069000A0F0001034F0001010B51148FFF7A2FED2
:1006A0001048FFF79FFE1048FFF79CFE0F48FFF72A
:1006B00099FE0F48FFF796FE0E48FFF793FE0E488F
:1006C000FFF790FE0D48FFF78DFE0D48FFF78AFEFD
:1006D0000C48FFF787FE0C48FFF784FE10BDC046AC
:1006E000FCE9001010EA001018EA001030EA0010CF
:1006F00038EA001054EA001068EA001090EA00108E
:10070000BCEA0010D0EA0010F8EA001070B51848F2
:10071000FFF768FE174D184CA96D20000BF082FB07
:10072000002803D11548FFF75DFEFEE74A232000AD
:10073000E95A0CF025FD696D20000CF07FFB502379
:10074000EA5A023BE95A20000CF064F948232000E1
:10075000E95A0CF01DFA4C232000E95A0CF0BEFCBB
:1007600020000CF055FD0648FFF73CFE70BDC0466A
:100770007CF00010E0290020582F002090F000109D
:10078000A0F00010F0B50021B3B006E06C464B1CA1
:10079000DBB26254202A4CD01900425C002AF5D109
:1007A000002219AD0023C5496846AB540DF080FE08
:1007B00000280FD1C24928000DF07AFE002800D190
:1007C0006AE0C04928000DF073FE002800D1BDE0AA
:1007D00033B0F0BDBC4968460DF06AFE00283BD03E
:1007E000BA4968460DF064FE002800D1B1E0B8496E
:1007F00068460DF05DFE041E00D085E028000DF077
:100800009BFE0928E4D82A78002A00D120E10023A1
:10081000B04901330C19DBB26270EA5C1C00002A9B
:10082000F7D100230C19AC4801316370FFF7DAFDF2
:10083000CEE71A0000216A44013A1170C15C002918
:10084000AED0002219AD0133DBB2A954C15C541CF7
:10085000E2B20029F7D1A5E7EFF3108572B69F4801
:10086000FFF7C0FD80218020490100030EF014F83D
:100870009B4C2000FFF7B6FD9A48FFF7B3FD80229E
:1008800080205200934900030DF0EEFF2000FFF797
:10089000A9FD85F310889BE7934D2B681B785A2B95
:1008A00000D191E09148FFF79DFD914CA3220021DA
:1008B000200008F053F8EFF3108772B68748FFF76F
:1008C00091FD80218020490100030DF0E5FF844E59
:1008D0003000FFF787FD8348FFF784FD2100802269
:1008E00080205C39520000030DF0BEFF3000FFF79E
:1008F00079FD87F31088802229685200754808F036
:1009000033F8FFF78BFD63E77A4968460DF0D0FDB9
:10091000041E2CD128000DF00FFE092800D957E73E
:100920002A78002A00D1C6E000236A4901330C1955
:10093000DBB2E272EA5C1C00002AF7D100230C193A
:100940006D480B31E372FFF74DFD41E7FFF766FDA0
:100950003EE76A48FFF746FD6948FFF743FD00217F
:10096000684808F061FA0122674B9A7730E76749D7
:1009700068460DF09DFD041E2AD0654968460DF0BD
:1009800097FD041E42D12E78302E00D123E128009D
:100990000DF0D2FD092800D91AE7002E00D123E17D
:1009A00000234C490C1901332934DBB22670EE5C6C
:1009B0001C00002EF6D100230C192934293155488A
:1009C0002370FFF70FFD03E75348FFF70BFD92E796
:1009D0002E78302E69D028000DF0AEFD092800D900
:1009E000F6E6002E00D1FDE000233A4901330C1950
:1009F000DBB2E677EE5C1C00002EF7D100230C1969
:100A000046481F31E377FFF7EDFCE1E644496846CD
:100A10000DF04EFD041E1DD128000DF08DFD09289E
:100A200000D9D5E62A782B49002A09D00023294984
:100A300001330C19DBB26275EA5C1C00002AF7D1A5
:100A400000230C19374815316375FFF7CBFCBFE65F
:100A50002049E6E6344968460DF02AFD00286DD1AC
:100A600028780300303B092B00D9B0E00021002298
:100A700004E00300303B092B00D9A8E08B005B1891
:100A80005B001B181900013292B2A85C30390028B3
:100A9000EFD1264A9A18264B9A4200D997E00D4B7F
:100AA00024489965FFF79EFC92E60A4BD8772248C6
:100AB000FFF798FC8CE6074940E7C04658ED001068
:100AC00060ED001068ED00106CED001074ED00108A
:100AD000D0ED0010E0290020D8ED0010B8EF001094
:100AE000D0EF0010D8EF0010C0140020F8EF001075
:100AF0003C2A0020ECED0010F8ED00107CED001019
:100B000094ED001060150020842F002010EE0010DE
:100B10003CEE001054EE001034F0001028EE0010EF
:100B200068EE001070EE001088EE0010D04EF7E670
:100B300080C3C901B4EE001018EE00108149684668
:100B40000DF0B6FC002820D128780300303B092B9B
:100B50003DD80021002203E00300303B092B36D8AA
:100B60008B005B185B001B181900013292B2A85C65
:100B700030390028F0D1363B062B28D84823724A5A
:100B80007248D152FFF72EFC22E6714968460DF0FB
:100B90008FFC00282AD06F4968460DF089FC002898
:100BA00045D12C782300303B092B10D801000200DE
:100BB0008B005B185B001B191900013292B2AC5C10
:100BC0003039002C29D02300303B092BF0D9624862
:100BD000FFF708FCFCE529235B4AD0545F48FFF788
:100BE00001FCF5E5584909E75749E4E62878030090
:100BF000303B092BEBD8002100228B005B185B00F7
:100C00001B181900013292B2A85C303900284CD070
:100C10000300303B092BF0D9D9E7353B032BD6D85D
:100C20004C23494A4E48D152FFF7DCFBD0E54D49F1
:100C300068460DF03DFC002820D04B4968460DF079
:100C400037FC002846D1010003000A3008E01400F8
:100C5000303C092CBBD841430133303951189BB289
:100C6000EA5C002AF3D1414B414ACB189342AED8FB
:100C7000354B40485965FFF7B5FBA9E52C782300B3
:100C8000303B092BA3D8010002008B005B185B00EE
:100C90001B191900013292B2AC5C3039002C0FD014
:100CA0002300303B092BF0D991E7334A363B93427E
:100CB0008DD84A23244A3148D152FFF793FB87E568
:100CC000323B0F2B83D84E231F4A2D48D152FFF7BA
:100CD00089FB7DE52B4968460DF0EAFB00281AD117
:100CE000010003000A3009E01400303C092C00D94F
:100CF0006DE741430133303951189BB2EA5C002A59
:100D0000F2D1012900D962E750230F4A1E48D1527F
:100D1000FFF768FB5CE51D4968460DF0C9FB00283C
:100D200000D055E51A4928000DF0C2FB002805D176
:100D30001848FFF757FBFFF7E9FC49E5FFF7ACFC64
:100D400046E5C046D0EE0010E0290020D8EE0010A5
:100D5000FCEE00101CEF001090EE001044EE0010AE
:100D600024EF001044EF001068EF001088E1FFFF4F
:100D7000C82C4C0070EF0010F9FF000000EF0010CD
:100D80004CEF00108CEF001090EF0010A4EF00105B
:100D9000ACEF0010B4EF0010F0B5C646CB4D00B577
:100DA0008046FD222800002107F0D8FDC423023D23
:100DB0005B422B80C64EC533AB707378002B00D1DD
:100DC000B0E1EB70B378002B00D1BAE12B71F3786E
:100DD000002B00D1B9E16B713379002B00D1B6E162
:100DE000AB717379002B00D18DE1EB71B379002BDE
:100DF00000D1AEE12B72F379002B00D1ABE16B7225
:100E0000337A002B00D1A8E1AB72737A002B00D1AA
:100E1000A5E10C27EB727B1CBA1C1D0010003E24C0
:100E2000AC49CC55777D002F3FD0CF54B57D5A1CAF
:100E300092B2002D00D160E18D54F57D981C80B2F6
:100E4000002D00D15BE10D54357EDA1C92B2002DED
:100E500000D152E18D54757E181D80B2002D00D155
:100E60004DE10D54B57E5A1D92B2002D00D144E1E2
:100E70008D54F57E981D80B2002D00D13FE10D54B8
:100E8000357FDA1D92B2002D00D136E118008D5465
:100E9000727F083080B2002A00D130E109339BB262
:100EA0000A545A1C92B21D001000F77F002F52D036
:100EB0002C2320204B558F54531C375C901C9BB225
:100EC00080B21D008446002F00D120E1CF542123A1
:100ED000F75CD31C9BB21D00002F00D128E10F54FA
:100EE0002220375C101D80B28446002F00D10EE115
:100EF000CF542323F75C531D9BB21D00002F00D15C
:100F000016E10F542420375C901D80B28446002FD8
:100F100000D1FCE0CF542523F75CD31D9BB21D000C
:100F2000002F00D104E10F542620375C1000083058
:100F300080B28446002F00D1E9E0CF542723F75C2C
:100F4000130009339BB21D00002F00D1F0E00A32DC
:100F500092B20F5410002927F75D002F4DD02C239B
:100F60002A204B558F54531C375C901C9BB280B287
:100F70001D008446002F40D0CF542B23F75CD31C98
:100F80009BB21D00002F00D1D7E00F542C20375CFE
:100F9000101D80B28446002F2FD0CF542D23F75C34
:100FA000531D9BB21D00002F00D1C6E00F542E2010
:100FB000375C901D80B28446002F1ED0CF542F2363
:100FC000F75CD31D9BB21D00002F00D1B5E00F547C
:100FD0003020375C1000083080B28446002F0CD0DF
:100FE000CF543123F75C130009339BB21D00002F4F
:100FF00000D1A2E00A320F5490B23A224A550A5464
:10100000F57A9F1CBFB2002D00D182E03C3AD31A82
:1010100000E017007A1C92B2D01880B2CD55351876
:10102000ED7A002DF5D108283BD820258D54421C9F
:10103000BB1C92B29BB2092A00D184E00230033774
:1010400080B2BAB2CD5409282BD02023461C551C9F
:10105000B6B2ADB28B54092E53D04B55851C961C9D
:10106000ADB2B6B2092D50D08B55C61CD51CB6B248
:10107000ADB2092E45D04B55051D161DADB2B6B209
:10108000092D42D08B55461D551DB6B2ADB2092E65
:1010900037D0961DB6B24B55032836D0073292B2E0
:1010A0008B553A238B5443461878561CB6B2002809
:1010B0001AD0FE2E18D84D1CAD198B19FD264446AA
:1010C000B21A92B20134AA180AE0C046323C00209B
:1010D000E0290020303C002001330134934203D04A
:1010E000187020780028F7D101221E4B1E481A7074
:1010F000FFF778F904BC9046F0BD1300D1E6030079
:10110000CFE62A00CDE7072785E63200C9E70200CF
:1011100021E720201A1D03339BB2C85592B2C85450
:101120001E3892E70520052204250423032776E6CE
:101130001A000500180063460DE705001800634615
:101140005BE7042767E61A00ABE7052763E6062797
:1011500061E608275FE609275DE60A275BE60B27BD
:1011600059E6C046413D0020E0EB0010F0B5DE46F8
:1011700057464E464546E0B5A54C85B00A220021AB
:10118000200007F0EBFB2000FF2200210A3007F0CF
:10119000E5FB20000A30FF220021FF3007F0DEFBD4
:1011A00082239B00E018FF22002107F0D7FB994B18
:1011B0006422E018002107F0D1FB974BFF22E018D2
:1011C000002107F0CBFB0023944AA354944AA35078
:1011D0000432A354934B1A78002A41D022703E2A3D
:1011E00000D10CE15A78002A3AD062703E2A00D130
:1011F00008E19A78002A33D0A2703E2A3CD0DA78EF
:10120000002A2DD0E2703E2A00D1F2E01A79002A9D
:1012100026D022713E2A00D1EEE05A79002A1FD052
:1012200062713E2A00D1F0E09A79002A18D0A271AA
:101230003E2A00D19EE1DA79002A11D0E2713E2ADD
:1012400000D19AE11A7A002A0AD022723E2A00D1ED
:1012500096E15A7A002A03D062723E2A00D198E1C0
:101260007148FFF7BFF86E4BE05A05B03CBC9046A2
:101270009946A246AB46F0BD0322022100206054ED
:101280008E21C9006054995C0029E9D0A1723A29E5
:1012900000D1A9E1012500E005000132995C002997
:1012A000DED0681C261871723A29F5D10021651923
:1012B000A9728E210120C900605499184878002134
:1012C000002809D001310D000935FF35605550184F
:1012D000181840780028F5D1002361180A31FF3131
:1012E0000B70A27A002A00D17BE1210000230B3190
:1012F0000026002000279C4604E001314B1E1A788E
:10130000002A1CD083001B185B00E3187D1CDB192E
:10131000404FB84643441A702F002C2AEDD1092DB6
:10132000EBDC6246013080B21A70092800D933E143
:1013300001314B1E1A7801260027002AE2D1002E27
:1013400000D06DE1334993008C4600219B185B006F
:10135000E318DB1963441970344D2178E87A81422F
:101360000BD1002910D0002301E000290CD001335B
:10137000E818E15CC07A8142F7D0002900D145E14C
:10138000002806D0884204D10A23FF33E35C3A2BBD
:1013900058D0274B274901325D181900FF39FF3912
:1013A000039119001E3102911900143101911900A5
:1013B0000A31009120482900FFF714F81F4B9B7F4A
:1013C000012B00D1DFE082239B00154DE35C605BC5
:1013D000002B00D149E782239B00E1180200184846
:1013E000FFF700F80D4BE35C002B00D0B8E0605B2A
:1013F0003BE70422032141E7052204213EE70122C5
:1014000000213BE70222012138E70622052135E7CA
:101410006C250020070300006B0300006A04000035
:101420006C040000103B00203CED0010E02900207F
:1014300073280020F9FCFFFFBCEC0010842F002073
:10144000F8EC00101423FF33E35C3A2BA1D16B7846
:10145000002B4AD085214900615C994299D1AB7833
:10146000002B42D00C21FF31615C994291D1EB7885
:10147000002B3AD086214900615C994289D12B79B1
:10148000002B32D00E21FF31615C994200D080E701
:101490006B79002B29D087214900615C994200D0EB
:1014A00077E7AB79002B20D01021FF31615C9942A6
:1014B00000D06EE7EB79002B17D088214900615CE2
:1014C000994200D065E72B7A002B0ED01221FF3114
:1014D000615C994200D05CE76B7A002B05D08921D2
:1014E0004900615C994200D053E78A235B00E15CCC
:1014F000002900D18EE00A3BFF3B00E0030018000A
:10150000FE30FF30215419000B31FF31615C581C53
:101510000029F3D10A3B822189008C460021E3187F
:10152000634419706346E11800239B4661339C466F
:1015300002339946083300260025002098460F788C
:10154000002F53D07B2F33D0002D5DD1B300F31883
:101550005B00303BDB199EB2012301319B46EEE775
:10156000314BE6183000FFF717FC31002F48FEF72B
:1015700039FF3CE70722062180E6082207217DE6A5
:10158000092208217AE62A4A29002A480BF0A4FEFB
:1015900019E7343A092171E6274BE0520233E2544D
:1015A0008300181840002018451945442A7057E652
:1015B0001D4B2718FD1863462B70DB239B00FD187D
:1015C0004B462B701D4BC51CF81843460370164B39
:1015D0004F789A46681C651955442F7001310125D2
:1015E000ADE7174BE254B7E600255FE6002D13D1B7
:1015F0005B46002B01D0134BE6520B4B20189C4648
:10160000002360440370C4E60500E0E7002800D032
:10161000BFE6B9E600237EE701250B496554E7E7FD
:10162000054B0200E0528DE66B03000020ED001038
:10163000681F0020E02A00206E0400006D030000F7
:10164000070300006C0400006A040000F8B5DE46E1
:1016500057464E4645469E48E0B5FEF7C3FE9D4CB4
:10166000FD222000002107F079F9C423023C5B42EF
:10167000994F2380C533A3703B78002B00D107E13D
:10168000E3707B78002B00D109E12371BB78002B3C
:1016900000D10BE16371FB78002B00D109E1A3714C
:1016A0003B79002B00D1E8E0E3717B79002B00D17E
:1016B00002E12372BB79002B00D100E16372FB7958
:1016C000002B00D1FEE0A3723B7A002B00D1FCE09E
:1016D000E3720C230D243E2280490026CA54804B1D
:1016E000FB5A9846002399462C339C464B469B0058
:1016F0009B464D465D446D007A4B7D19EB181B7877
:1017000020009A465246631C9BB2002A00D1A0E0FA
:10171000FE2C00D99DE00A55734AA8180278002AC9
:1017200000D19AE0FF2B00D18EE0CA5483239B00A6
:10173000EB181B78A01C80B29A46002B00D190E0D9
:10174000FF2800D180E052460A54684AE31CA818DA
:1017500002789BB2002A00D187E0FF2B00D173E012
:10176000CA54634B201D9A4655442D7880B2002DF3
:1017700000D17EE0FF2867D05A464A440D545200FB
:101780005C48BA1810180578631D9BB2002D00D173
:1017900076E0FF2B58D0CD5484239B00D3181D78BE
:1017A000A01D80B2002D6FD0FF284DD00D5452489F
:1017B000E31D101805789BB2002D6CD0FF2B43D091
:1017C000CD544E4B200099464A441278083080B2DE
:1017D000002A67D0FF2837D0230009339BB20A5470
:1017E00018000A34A4B262460136F6B20A54B14671
:1017F000464500DC7AE73A220A54B87A002813D02A
:10180000FE2B11D8FE263C004D1CED18CA18F31A09
:101810009BB20B34EB1803E0013201349A4203D03F
:10182000107020780028F7D10122354B35481A7006
:101830008E230022DB00FA54FEF7D4FD3CBC904618
:101840009946A246AB46F8BD8024FF206400FF23E2
:10185000C9E71A0023001400C5E702341800A4B237
:10186000C1E70334A4B20300BDE704341800A4B2F6
:10187000B9E70534A4B20300B5E7072308242AE733
:1018800006341800A4B2AEE70734A4B20300AAE7F6
:10189000042403231FE708341800A4B2A3E7042399
:1018A000052418E70934A4B203009CE705230624A5
:1018B00011E7062307240EE7082309240BE7092371
:1018C0000A2408E70A230B2405E70B230C2402E76C
:1018D0005CF00010323C0020E42A0020303C002064
:1018E0006E0200000A0200000B0200000D02000060
:1018F0000E0200000F0200001102000012020000A0
:10190000413D0020E0EB0010F0B5C64600B5484F61
:101910000020BB7F002B2DD107F034FA0400431CBC
:1019200025D0444B444F454D454E984607E042452F
:1019300052D0002007F026FA0400431C17D02100E3
:101940003800FEF74FFD2B685A1C2A60F4540D2C0A
:10195000EDD100223B48F2542A60FEF743FD3000EF
:101960000CF0EAFD02283AD93000FEF70BFF04BC68
:101970009046F0BD07F006FA431CF8D000232F4D27
:101980002F4E2C4C984604E0002007F0FBF9431C36
:10199000EDD02A68531C2B60B054A34202D14346B9
:1019A0002B600023C028EFD13278C02A04D0C02396
:1019B0003370BF3B2B60DAE7012BF8DD224A3100A0
:1019C00022480BF0FDFE02282BD0002801D1FFF7A2
:1019D0003DFE00232B60CAE7FF235B00B9E71C48EC
:1019E000FEF700FD1B48FEF7FDFC1B48FEF7FAFC66
:1019F0001A48FEF7F7FC1A48FEF7F4FC1948FEF700
:101A0000F1FC1948FEF7EEFC1848FEF7EBFC18480D
:101A1000FEF7E8FC1748FEF7E5FC1748FEF7E2FC86
:101A2000A5E70121154807F0FFF90023BB77D0E7B0
:101A3000842F0020FF010000B8EC0010A42F00202C
:101A4000A82F002070EB0010E42A0020E02A0020DC
:101A5000FCE9001010EA001018EA001030EA00104B
:101A600038EA001054EA001068EA001090EA00100A
:101A7000BCEA0010D0EA0010F8EA0010601500205F
:101A800010B51348FEF76AFC1249134C0B002000F6
:101A90000A6D503362609B885831238114220A30CA
:101AA00006F062FF8020002300220C4980000B52C8
:101AB0000B48A3770B520B490B480C4C0A540C48AB
:101AC0000B5004300A540B490B530A5410BDC04646
:101AD000E029002090E90010842F0020681F0020DA
:101AE000020600006C2500206A0400006E0200005F
:101AF0006C040000E42A0020F0B5DE4657464E464E
:101B00004546E0B597B0FEF7FDFC002301933F4B3F
:101B10003F4F98463F4B99463F4B9E1E3F4B9A4640
:101B2000D0231B069B4611E053461B78002B0BD09D
:101B3000019B002B03D13A4B9B6A9B059B0D5A1EC0
:101B400092B20192012B25D0FFF7DEFE0021404624
:101B50000AF0DAFC051EE7D040460AF065FE0100F7
:101B60003048FEF73FFC002400E01C00404609F02E
:101B7000D9FF4A46631C10559D42F6D100235355A8
:101B800013783C2B02D15378FF2B20D02648FEF748
:101B900029FCC9E7002140460AF002FB3178002900
:101BA00008D0002401344046A4B209F041FF315D61
:101BB0000029F7D1002140460AF0FEFB00214046F3
:101BC0000AF070FE0023524601931370BCE793782D
:101BD000012BDBD1032D05DD4B46A21ED91C484647
:101BE0000CF082FE00234C44023C49460F4823700F
:101BF000FEF7F8FBFFF7BAFA0500041E94D025287B
:101C000092D80B4A8300D3589F46C046582F0020D5
:101C1000E0290020103B0020323C0020413D002004
:101C200000400540B0F00010D0F00010E0EB0010D4
:101C3000F8E80010FD220021F54806F08FFEC422CE
:101C4000F34B5242023B1A80C5329A707A78002ACE
:101C500001D100F073FEDA70BA78002A01D100F0E9
:101C600007FF1A71FA78002A01D100F0A7FF5A7114
:101C70003A79002A01D101F0BAF89A717A79002AEA
:101C800001D101F059F9DA71BA79002A01D101F0D4
:101C9000BAF91A72FA79002A01D101F070FA5A726F
:101CA0003A7A002A01D101F032FB9A727A7A002A3C
:101CB00001D101F04CFCDA7218230E220C21102401
:101CC0000D930C93013B0B93013B09930133149348
:101CD000023B089301330A93023B079301331393AA
:101CE000023B069301331193023B05930133129398
:101CF000023B049301330F93023B039301330E9392
:101D0000023B9C46013B0293109208000133013ACA
:101D100001313E2535547D7D002D3FD0B554BA7D2F
:101D2000002A01D100F006FF02997254FA7D002AC0
:101D300001D100F0DDFF6346F2543B7E002B01D160
:101D400001F01DF8039AB3547B7E002B01D101F002
:101D500084F8049AB354BB7E002B01D101F01BF927
:101D6000059AB354FB7E002B01D101F066FA069A66
:101D7000B3543B7F002B01D101F090FB079AB35481
:101D80007B7F002B01D101F09AFB089A0A99B3548A
:101D90000D9B099A9C460B9B02930C9BFC7F002C8D
:101DA0005ED02C25B554029AB4542022BA5C002A85
:101DB00001D101F0AAF9604632542122CB1CBC5C4F
:101DC0009BB21A00002C01D101F07FFAF4542223B7
:101DD000081DFC5C80B20200002C01D101F016FB52
:101DE000232234544B1DBC5C9BB21A00002C01D141
:101DF00001F01BFCF4542423881DFC5C80B202001B
:101E0000002C01D101F057FC25223454CB1DB85CC5
:101E10009BB21A00002801D101F061FCF0540C00C3
:101E200026230834FB5CA4B22200002B01D101F070
:101E30008CFC3355080027230930FB5C80B202007C
:101E4000002B01D101F0DDFC0A0033540B000A32F3
:101E50000C330B3189B292B29BB202919C461100B5
:101E600029243C5D002C5DD02C25B554029AB45435
:101E70002A22BA5C002A01D101F066F96046325488
:101E80002B22CB1CBC5C9BB21A00002C01D101F0B0
:101E900035FAF454081D7C5D80B20200002C01D19B
:101EA00001F0ABFA2D2234544B1DBC5C9BB21A00DE
:101EB000002C01D101F0D2FBF4542E23881DFC5CD0
:101EC00080B20200002C01D101F0FFFB2F2234541C
:101ED000CB1DB85C9BB21A00002801D101F009FCAF
:101EE000F0540C0030230834FB5CA4B22200002B19
:101EF00001D101F034FC3355080031230930FB5C7B
:101F000080B20200002B01D101F085FC0A0033549D
:101F10000B000A320C330B3189B29BB292B20291A0
:101F20009C4611003A24B454029AB454F87A00281A
:101F300001D100F088FD002401E00B001400621CB8
:101F400092B2F054B818C07A591C89B20028F4D162
:101F50000800082A4AD820209D1CADB2844670543F
:101F60002800072C01D100F0B5FC6046DC1CA4B2AF
:101F700070552000072A01D100F0ACFC60461D1D01
:101F8000ADB230552800062A01D100F0A3FC60460E
:101F90005C1DA4B270552000052A01D100F09AFC06
:101FA00060460633305598B2042A01D100F092FC05
:101FB00020258B1D9BB235541800032A01D100F057
:101FC00089FCCC1DA4B2F5542000022A01D100F0F6
:101FD00081FC0B0008339BB235551800002A01D054
:101FE00000F078FC093189B20800F5543A233354E3
:101FF000084B4C1C9A7AA4B2002A16D0FE2C14D896
:10200000FD23591A89B201310023341907E0C04673
:10201000323C0020842F00200133994205D0E25445
:10202000C84AD218D27A002AF6D15346012231008A
:10203000C5481A70FEF7D6F940235A46936100232B
:10204000C04A137070E5FD220021C04806F086FCEE
:10205000C422BE4B5242023B1A80C5329A707A7833
:10206000002A01D100F0C0FCDA70BA78002A01D150
:1020700000F069FD1A71FA78002A01D100F0FAFD2A
:102080005A713A79002A01D100F03BFE9A717A79AF
:10209000002A01D100F0EAFEDA71BA79002A01D1F2
:1020A00000F0E0FF1A72FA79002A01D101F096F8E7
:1020B0005A723A7A002A01D101F0C1F99A727A7AF9
:1020C000002A01D101F00CFADA7218230E220C2139
:1020D0000E200D930C93013B0B93013B09930133AD
:1020E0001593023B089301330A93023B0793013394
:1020F0001493023B069301331393023B0593013380
:102100001293023B049301331093023B0393013378
:102110000F93023B029301330E9311928C46013BC5
:10212000013A01313E25644635557D7D002D3DD077
:10213000B554BA7D002A01D100F034FD3254FA7D45
:10214000002A01D100F0C5FD029BF2543B7E002B1A
:1021500001D100F00CFE039AB3547B7E002B01D119
:1021600000F073FE049AB354BB7E002B01D100F043
:10217000A8FF059AB354FB7E002B01D100F0EFFFBE
:10218000069AB3543B7F002B01D101F01EF9079A48
:10219000B3547B7F002B01D101F0D1F9089A0B9841
:1021A000B3540D9B099A02930A990C9BFD7F002D55
:1021B0005CD02C24B45420223554BA5C002A01D1BE
:1021C00000F0AEFF0298CB1C32542122BC5C9BB2C3
:1021D0001A00002C01D101F081F8F4542223081DCB
:1021E000FC5C80B20200002C01D101F0FEF8232239
:1021F00034544B1DBC5C9BB21A00002C01D101F081
:1022000025FAF4542423881DFC5C80B20200002CC3
:1022100001D101F02CFA25223454CB1DBC5C9BB2B9
:102220001A00002C01D101F06EFAF45408002623A4
:102230000830FB5C80B20200002B01D101F0ABFA48
:1022400033540C0027230934FB5CA4B22200002B7A
:1022500001D101F0B2FA0A0033550B000A320B31FA
:1022600092B288B211000C339BB2029329257D5D96
:10227000002D5DD02C24B4542A223554BA5CA446D7
:10228000002A01D100F02DFF0298CB1C32542B22E2
:10229000BC5C9BB21A00002C01D101F006F8F4548A
:1022A0006346081DFC5C80B20200002C01D101F0E5
:1022B00094F82D2234544B1DBC5C9BB21A00002CA8
:1022C00001D101F0AAF9F4542E23881DFC5C80B2E0
:1022D0000200002C01D101F0DCF92F223454CB1D77
:1022E000BC5C9BB21A00002C01D101F01DFAF45421
:1022F000080030230830FB5C80B20200002B01D1C3
:1023000001F052FA33540C0031230934FB5CA4B2BF
:102310002200002B01D101F059FA0A0033550B00BD
:102320000A320B3192B288B211000C339BB2029385
:102330003A25B5543554F87A002800D12CE300240E
:1023400008E0C046842F0020E0EB0010323C002063
:102350000B001400621C92B2F054B818C07A591CD9
:1023600089B20028F4D10800082A42D820209D1CF8
:10237000ADB2844670542800072C00D1ADE260460F
:10238000DC1CA4B270552000072A00D1A5E26046EB
:102390001D1DADB230552800062A00D19DE26046D1
:1023A0005C1DA4B270552000052A00D195E260465C
:1023B0000633305598B2042A00D18EE220258B1DB9
:1023C0009BB235541800032A00D186E2CC1DA4B27A
:1023D000F5542000022A00D17FE20B0008339BB2A3
:1023E00035551800002A00D077E2093189B208007B
:1023F000F5543A233354073BFA5C4C1CA4B2002A30
:1024000011D0FE2C0FD8FD23591A89B201310023B7
:10241000341902E001338B4205D0E2541A00343201
:10242000BA5C002AF6D1534601223100CB481A701B
:10243000FDF7D8FFFFF778FBC94B00211B78C9488F
:102440005A1E9341C64A3033137253785A1E934131
:10245000C34A3033D37193785A1E9341C04A303304
:102460009371D3785A1E9341BD4A30335371FD2284
:1024700006F074FAC422BB4B5242023B1A80C532AA
:102480009A707A78002A00D12BE2DA70BA78002AA2
:1024900000D11BE31A71FA78002A00D1BCE35A710B
:1024A0003A79002A01D100F073FC9A717A79002AF6
:1024B00001D100F012FDDA71BA79002A01D100F0E1
:1024C00073FD1A72FA79002A01D100F0BFFE5A7228
:1024D0003A7A002A01D100F049FF9A727A7A002AEA
:1024E00001D101F063F8DA7218230E250F240D22B2
:1024F0000C930D93013B0A93013B09930133159310
:10250000023B089301330B93023B0793013314936F
:10251000023B069301331193023B0593013312935F
:10252000023B049301331093023B039301330E9358
:10253000023B029301330F93023B1393023B9C46F1
:1025400001333E2061467054787D00283AD0B05463
:10255000BB7D002B00D1E6E27355FB7D002B00D143
:10256000BFE3029AB3543B7E002B00D1F8E3039AF9
:10257000B3547B7E002B01D100F0A7FC049AB35426
:10258000BB7E002B01D100F0A4FD059AB354FB7E65
:10259000002B01D100F0EBFD069AB3543B7F002BDA
:1025A00001D100F044FF079AB3547B7F002B01D187
:1025B00000F08EFF089A0A9DB3540C9B0D9C029369
:1025C000099A0B9BF87F00285CD02C21B154202263
:1025D0007055BA5C002A01D100F0ACFD0299D81CFC
:1025E00072542122BC5C80B20200002C01D100F0A8
:1025F0007DFE22223454191DBC5C89B20A00002CD5
:1026000001D100F00CFF23227454581DBC5C80B231
:102610000200002C01D101F011F824223454991D3C
:10262000BC5C89B20A00002C01D101F03BF82522E4
:102630007454D81DB95C80B202001C00002901D17D
:1026400001F07BF8262231540834B95CA4B2220090
:10265000002901D101F096F82722180031550930E0
:10266000B95C80B20200002901D101F0C1F81A0062
:102670001C000A320B3392B29DB213000C34A4B288
:10268000315402942920385C00285DD02C21B154AB
:102690002A227055BA5C8C46002A01D100F02BFD2D
:1026A0000299D81C72542B22BC5C80B20200002C10
:1026B00001D100F002FE62463454191DBC5C89B29F
:1026C0000A00002C01D100F0F2FE2D227454581D96
:1026D000BC5C80B20200002C01D100F096FF2E22DB
:1026E0003454991DBC5C89B20A00002C01D100F061
:1026F000C7FF2F227454D81DB95C80B202001C00A1
:10270000002901D101F008F8302231540834B95CB5
:10271000A4B22200002901D101F02BF831221800C7
:1027200031550930B95C80B20200002901D101F0B5
:1027300056F81A001C000A320B3392B29DB21300F5
:102740000C34A4B2315402943A20B0547055F87A43
:10275000002800D134E1002108E0C046E0EB001081
:10276000842F0020323C0020140019004B1C9BB227
:102770003055F818C07A621C92B20028F4D11000CB
:10278000082B3FD82020A51CADB28446B0542800A9
:10279000072900D1A3E06046E11C89B2705508000A
:1027A000072B00D19BE06046251DADB27054280078
:1027B000062B00D193E06046611D89B27055080078
:1027C000052B00D18BE0604606347054A0B2042B78
:1027D00000D184E02025911D89B235540800032BD7
:1027E0007DD0D41DA4B275542000022B77D01100E7
:1027F000083189B235550800002B70D1093292B2E8
:10280000100075543A233354EA4B541C1979A4B27E
:10281000002900D107E6FE2C00D904E6FD239A1A10
:1028200092B201320023341903E001339A4200D1FD
:10283000F9E5E154DF49C91849790029F5D1534632
:1028400001223100DC481A70FDF7CCFDFFF76CF96E
:102850005B460824FA205C6101F072FC5B460122B1
:102860009C61D44BDA70FFF75FF910235A4653612D
:102870000023D04A9370FFF757F920235A4653613B
:102880000122CC4B5A70FFF74FF920235A4693612F
:102890000023C84A5370FFF747F940235A46536153
:1028A0000122C44B1A70FFF73FF95B460424FA205B
:1028B0005C6101F045FC5B469C610023BD4AD3701E
:1028C000FFF732F910235A4693610122B94B9A70EF
:1028D000FFF72AF90100FFF789FB010089E50200F3
:1028E00090E70F230C930D93013B0A93013B09934F
:1028F00001331593023B089301330B93023B07937B
:1029000001331493023B069301331193023B059369
:1029100001331293023B049301331093023B039360
:1029200001330E93023B029301330F93023B139347
:10293000023B9C4605250422013302E60F230522B3
:1029400003210D930C93013B0B93013B099301333E
:102950001493023B089301330A93023B079301331C
:102960001393023B069301331193023B059301330A
:102970001293023B049301330F93023B0393013301
:102980000E93023B9C46013B0293109208000133D8
:10299000013A0131FFF7BDF920220298033189B2D3
:1029A00032547254991C89B27254D91C89B272542F
:1029B000191D89B2581D725480B219000022FDE41D
:1029C0002022029903339BB27254F254A31C9BB28F
:1029D000F254E31C9BB2F254231D9BB2601DF254CF
:1029E00080B222000023F5E60F23052203210D9378
:1029F0000C93013B0B93013B099301331593023B6D
:102A0000089301330A93023B079301331493023B6B
:102A1000069301331393023B059301331293023B58
:102A2000049301331093023B039301330F93023B52
:102A3000029301330E9311928C460520013B013A1B
:102A40000131FFF76FFB20226046033189B2325417
:102A50007254991C89B27254D91C89B27254191DCE
:102A600089B2581D725480B219000022FFF7A0FAF3
:102A7000102204210D920C92013A0B92013A099214
:102A800001321492023A089201320A92023A0792F3
:102A900001321392023A069201321192023A0592E1
:102AA00001321292023A049201320F92023A0392D8
:102AB00001320E92023A9446013A029210920800B4
:102AC0002B000824013A0131FFF723F910230C935E
:102AD0000D93013B0A93013B099301331593023B8C
:102AE000089301330B93023B079301331493023B8A
:102AF000069301331193023B059301331293023B7A
:102B0000049301331093023B039301330E93023B72
:102B1000029301330F93043B13959C46062507242B
:102B2000052201330DE5039B2A000F9C029D0293B1
:102B3000139B47E56146029A0291039923008C4654
:102B40001099FFF72BF91023062204210D930C9303
:102B5000013B0B93013B099301331593023B08930F
:102B600001330A93023B079301331493023B06930C
:102B700001331393023B059301331293023B0493F9
:102B800001331093023B039301330F93023B0293F3
:102B900001330E9311928C460620013B013A01311C
:102BA000FFF7C0FA039902000E9B02980291119957
:102BB000FFF7FCFA842F0020E0EB00101123052121
:102BC0000D930C93013B0B93013B09930133149339
:102BD000023B089301330A93023B0793013313939B
:102BE000023B069301331193023B05930133129389
:102BF000023B049301330F93023B039301330E9383
:102C0000023B9C46013B02930800109509240133C6
:102C100006220131FFF77DF8112205210C920D9259
:102C2000013A0A92013A099201321592023A089247
:102C300001320B92023A079201321492023A069242
:102C400001321192023A059201321292023A049232
:102C500001321092023A039201320E92023A02922B
:102C600001320F92023A2B00139207250824013AF1
:102C70008C4666E41123072205210D930C93013B3A
:102C80000B93013B099301331593023B08930133E6
:102C90000A93023B079301331493023B06930133DB
:102CA0001393023B059301331293023B04930133C8
:102CB0001093023B039301330F93023B02930133C2
:102CC0000E9311928C460720013B013A0131FFF728
:102CD00029FA0499029A0398029119000F9BFFF7B1
:102CE00065FA049B029A039D029323000E9C69E4FB
:102CF000039A0499029262468C4619000E9BFFF7D4
:102D00004DF81223082206210D930C93013B0B93DF
:102D1000013B099301331593023B089301330A9356
:102D2000023B079301331493023B06930133139341
:102D3000023B059301331293023B0493013310933A
:102D4000023B039301330F93023B029301330E9333
:102D500011928C460820013B013A0131FFF7E2F95C
:102D6000059B049D0293109C039A0F9B2AE4059BEC
:102D700004980293039A109B0E99FFF717FA059B8C
:102D8000039A9C46049B210002930F9BFFF706F8D1
:102D900012230C930D93013B0A93013B09930133DA
:102DA0001593023B089301330B93023B07930133C6
:102DB0001493023B069301331193023B05930133B5
:102DC0001293023B049301331093023B03930133AC
:102DD0000E93023B029301330F93023B1393023B8A
:102DE0009C460825092407220133FFF7AAFB12237A
:102DF00008220D930C93013B0B93013B0993013384
:102E00001493023B089301330A93023B0793013367
:102E10001393023B069301331193023B0593013355
:102E20001293023B049301330F93023B039301334C
:102E30000E93023B9C46013B0293109229000A2408
:102E40000133013A0620FEF764FF069B05980293C2
:102E5000049A129B0F99FFF7A9F9069B049A9C46C6
:102E6000059B0E990293129BFEF798FF13230922EC
:102E700007210D930C93013B0B93013B0993013305
:102E80001593023B089301330A93023B07930133E6
:102E90001493023B069301331393023B05930133D2
:102EA0001293023B049301331093023B03930133CB
:102EB0000F93023B029301330E9311928C4609202B
:102EC000013B013A0131FFF72DF9069B059D029365
:102ED000129C049A0E9BFFF775FB13230C930D9322
:102EE000013B0A93013B099301331593023B08937D
:102EF00001330B93023B079301331493023B069378
:102F000001331193023B059301331293023B049367
:102F100001331093023B039301330E93023B029360
:102F200001330F93023B1393023B9C4609250A246D
:102F300008220133FFF705FB1323092207210D9314
:102F40000C93013B0B93013B099301331493023B18
:102F5000089301330A93023B079301331393023B17
:102F6000069301331193023B059301331293023B05
:102F7000049301330F93023B039301330E93023BFF
:102F80009C46013B0293109208000B240133013A46
:102F90000131FEF7BEFE079B059A9C46069B0F99E2
:102FA0000293119BFEF7FAFE14230C930D93013B41
:102FB0000A93013B099301331593023B08930133B4
:102FC0000B93023B079301331493023B06930133A7
:102FD0001193023B059301331293023B0493013397
:102FE0001093023B039301330E93023B0293013390
:102FF0000F93023B1393023B9C460A250B240922A4
:103000000133FFF79EFA14230A2208210D930C9333
:10301000013B0B93013B099301331493023B08934B
:1030200001330A93023B079301331393023B069348
:1030300001331193023B059301331293023B049336
:1030400001330F93023B039301330E93023B9C46E3
:10305000013B0293109208000C240133013A013124
:10306000FEF757FE14230A2208210D930C93013B0F
:103070000B93013B099301331593023B08930133F2
:103080000A93023B079301331493023B06930133E7
:103090001393023B059301331293023B04930133D4
:1030A0001093023B039301330F93023B02930133CE
:1030B0000E9311928C460A20013B013A0131FFF731
:1030C00031F8079B06980293059A139B1099FFF716
:1030D0006DF8079B069D0293119C059A109BFFF7C4
:1030E00071FA9D1C581CACB2029A190080B202946D
:1030F0002300FFF71DF9A01C651C81B2029A230072
:10310000ADB202910C00FFF71FFB9C1C581C82B251
:10311000A1B2029262468C4619006346FEF7A0FEF9
:103120009D1C581CACB2029A190080B20294230074
:10313000FFF79CF8A01C651C81B2029A2300ADB277
:1031400002910C00FFF79EFA9C1C581C82B2A1B29F
:10315000029262468C4619006346FEF7E3FE089B26
:1031600007980293069A149B1299FFF71FF8089B81
:10317000079D0293149C069A129BFFF723FA1523CE
:103180000B2209210D930C93013B0B93013B0993F7
:1031900001331493023B089301330A93023B0793D4
:1031A00001331393023B069301331193023B0593C2
:1031B00001331293023B049301330F93023B0393B9
:1031C00001330E93023B9C46013B02931092080090
:1031D0000D240133013A0131FEF79BFD15230B222B
:1031E00009210D930C93013B0B93013B0993013390
:1031F0001593023B089301330A93023B0793013373
:103200001493023B069301331393023B059301335E
:103210001293023B049301331093023B0393013357
:103220000F93023B029301330E9311928C460B20B5
:10323000013B013A0131FEF775FF089B069A9C4657
:10324000079B12990293139BFEF7A8FD15230C937D
:103250000D93013B0A93013B099301331593023B04
:10326000089301330B93023B079301331493023B02
:10327000069301331193023B059301331293023BF2
:10328000049301331093023B039301330E93023BEB
:10329000029301330F93023B1393023B9C460B2591
:1032A0000C240A220133FFF74CF94B1D9BB2043169
:1032B00088B202931100FFF73BF85C1DA4B20433FF
:1032C0009DB202940300FFF73FFA4B1D043189B20F
:1032D0009BB202919C461100FEF7C2FD4B1D9BB2B2
:1032E000043188B202931100FEF7C0FF5C1DA4B246
:1032F00004339DB202940300FFF7C4F94B1D04315F
:1033000089B29BB202919C461100FEF70BFE162378
:103310000C220A210D930C93013B0B93013B099363
:1033200001331493023B089301330A93023B079342
:1033300001331393023B069301331193023B059330
:1033400001331293023B049301330F93023B039327
:1033500001330E93023B9C46013B029310920800FE
:103360000E240133013A0131FEF7D3FC16230C93EE
:103370000D93013B0A93013B099301331593023BE3
:10338000089301330B93023B079301331493023BE1
:10339000069301331193023B059301331293023BD1
:1033A000049301331093023B039301330E93023BCA
:1033B000029301330F93023B1393023B9C460C256F
:1033C0000D240B220133FFF7BCF8099B08980293E8
:1033D000079A0A9B1399FEF7E9FE8B1D9BB20531F4
:1033E00088B202931100FEF7A3FF8B1D9BB205313B
:1033F00088B202931100FEF739FF8B1D053189B2A7
:103400009BB202919C460100FEF78CFD8B1D05319D
:1034100089B29BB202919C460100FEF721FD9C1DE2
:10342000A4B205339DB202940B00FFF72BF9099B60
:10343000089D02930B9C079A119BFFF7C3F8162374
:103440000C220A210D930C93013B0B93013B099332
:1034500001331593023B089301330A93023B079310
:1034600001331493023B069301331393023B0593FC
:1034700001331293023B049301331093023B0393F5
:1034800001330F93023B029301330E9311928C464A
:103490000C20013B013A0131FEF744FE099B079ADB
:1034A0009C46089B119902930A9BFEF777FC9C1D92
:1034B000A4B205339DB202940B00FFF745F90B9BB4
:1034C000089A9C46099B13990293149BFEF766FC8D
:1034D0000A9B099D0293159C089A149BFFF772F8AA
:1034E00017230D220B210D930C93013B0B93013BF2
:1034F000099301331593023B089301330A93023B6E
:10350000079301331493023B069301331393023B59
:10351000059301331293023B049301331093023B52
:10352000039301330F93023B029301330E931192E5
:103530008C460D20013B013A0131FEF7F3FD0B9B58
:1035400009980293089A159B1499FEF72FFE1723EA
:103550000D220B210D930C93013B0B93013B09931F
:1035600001331493023B089301330A93023B079300
:1035700001331393023B069301331193023B0593EE
:1035800001331293023B049301330F93023B0393E5
:1035900001330E93023B9C46013B029310920800BC
:1035A0000F240133013A0131FEF7B3FB17230C93CB
:1035B0000D93013B0A93013B099301331593023BA1
:1035C000089301330B93023B079301331493023B9F
:1035D000069301331193023B059301331293023B8F
:1035E000049301331093023B039301330E93023B88
:1035F000029301330F93023B1393023B9C460D252C
:103600000E240C220133FEF79CFFDC1DA4B206330E
:103610009DB202940300FFF797F8CB1D9BB20631D1
:1036200088B202931100FEF783FECB1D063189B2EA
:103630009BB202919C461100FEF712FCDC1DA4B265
:1036400006339DB202940300FFF71CF8CB1D9BB21A
:10365000063188B202931100FEF708FECB1D063139
:1036600089B29BB202919C461100FEF75BFC0B00F5
:10367000083307319BB288B202931100FEF7F6FDC2
:103680001C0008340733A4B29DB202940B00FFF76C
:103690005BF80B00083307319BB288B2029311002C
:1036A000FEF746FE1C0008340733A4B29DB2029414
:1036B0000B00FEF7E7FF0B000731083389B29BB21E
:1036C00002919C460100FEF7CBFB0B00073108334B
:1036D00089B29BB202919C460100FEF723FC0B00CD
:1036E0000831093389B29BB202919C461100FEF762
:1036F000B7FB0B000831093389B29BB202919C469B
:103700001100FEF70FFC0B00093308319BB288B2A1
:1037100002931100FEF7AAFD09340833A4B29DB24A
:1037200002940300FFF710F80B00093308319BB235
:1037300088B202931100FEF7FBFD09340833A4B2EE
:103740009DB202940300FEF79DFF0B0009310A337E
:1037500089B29BB202919C462100FEF781FB0B00CF
:1037600009310A3389B29BB202919C462100FEF7CF
:10377000D9FB1C000A340933A4B29DB20294130091
:10378000FEF7E2FF1C000A340933A4B29DB2029492
:103790001300FEF777FF0B000A3309319BB288B2A2
:1037A00002931100FEF762FD0B000A3309319BB250
:1037B00088B202931100FEF7BBFD0B000B330A31F8
:1037C0009BB288B202932100FEF750FD0B000B3331
:1037D0000A319BB288B202932100FEF7A9FD1C00BA
:1037E0000B340A33A4B29DB202940300FEF7ACFF7F
:1037F0001C000B340A33A4B29DB202940300FEF7FE
:1038000041FF0B000A310B3389B29BB202919C46F7
:103810000100FEF725FB0B000A310B3389B29BB286
:1038200002919C460100FEF77DFBC046094A8300D9
:1038300094464022634410B51C68C0006240C02416
:1038400014408022520113431C60034B9C46604489
:10385000416010BD04C00140004001400123D0225E
:103860008340120693629361094A83009446402282
:1038700063441968C0004A40C021114080225201AF
:1038800013431960034B9C46052360444360704713
:1038900004C0014000400140F8B5EFF3108772B654
:1038A0000D4E3368002BFCD0BFF35F8F0725CB088C
:1038B000C01801230D40AB401D000478254007D1FE
:1038C00023430370BFF35F8F356087F31088F8BD23
:1038D000100001F049FAC0462C0100D0F8B5CE46E0
:1038E00047468C4680B5EFF3108972B6214D2C689F
:1038F000002CFCD0BFF35F8F9A422CD80721012502
:1039000011408D40D4080419267835421FD0072174
:103910008846063909E045460F001540AF40D408F7
:10392000041926783D00374211D001329342F2D279
:1039300001204042BFF35F8F00220E4B1A6089F3D3
:10394000108800280FDB0CBC90469946F8BD354323
:1039500025701000EEE7BFF35F8F00232B6089F323
:103960001088012040426346002BECD0089801F0FB
:10397000FBF9C0462C0100D0024B18688007C00F2D
:103980007047C04600C006400021044B044ABFF304
:103990005F8F02C39342FAD17047C046000100D046
:1039A000800100D0044A1078431CDBB2172B00D9E9
:1039B000102313707047C046C414002000B5054B97
:1039C00083B00100009318221F230348FFF786FFEE
:1039D00003B000BDF4F000104C36002083680B48A3
:1039E00010B5844661446244090112019A185918BD
:1039F00054684B6801209C4201D802D00020C0B21C
:103A000010BD12680B689A42F9D8F7E7FFFFFF0F65
:103A10000A4B1968EFF3108072B60A68002AFCD0CE
:103A2000BFF35F8F1B68BFF35F8F00221A6080F3C4
:103A3000108840BF002000217047C046143C002081
:103A4000F8B557464E464546DE46E0B51F000CAB7E
:103A50001D780DAB1B7881469A4603681600984680
:103A6000002D3BD1987B002832D042464546440089
:103A700012682418033C121951780300A973002915
:103A800000D1E9730021050091705170117029E097
:103A9000D31814199D702278002A00D05A705B4602
:103AA000237043465D734B463200187D3B0000F0A7
:103AB00033FD041E07D05346002B04D14B4629008A
:103AC000186800F019FF0E9B002B44D028001C70D2
:103AD0003CBC90469946A246AB46F8BD2B006C0014
:103AE0006419033C1D4A94464A46926863449446CE
:103AF0001B010A9A63449A600B9A1E605F60DA6049
:103B0000434600221B681B199A705A701A7043466C
:103B10005B7B9B46002BC4D043462A0098685946DD
:103B20005B6898475B4642465B005B44033B126818
:103B30000028ADD0D31814195A46A2701A78002A5A
:103B400007D11D705A46434628005A73AB45BFD172
:103B5000A9E76270F5E72800BAE7C046FFFFFF0F4C
:103B6000F0B5DE46454657464E46724B8200E0B5FC
:103B7000D55800238DB00B909B4627E0069A079BF3
:103B80001100194303D02B69002B00D093E02B6860
:103B9000DA7B002A07D051008A1819688C464946FA
:103BA0006244033A51704A46DA73EA684B469446D7
:103BB000013B63441A7801321A705B462B616B68D3
:103BC000BFF35F8F5A461A6084F3108800F012FC2E
:103BD0006A68EFF3108472B61368002BFCD0BFF351
:103BE0005F8F2B689C465B7B9946002B5BD0AA6855
:103BF000514B90464B441B01984443461A685B68FE
:103C000016001F00361A8F41002F6EDD0B9800F052
:103C100083FC0022002300270026089209936B688A
:103C2000BFF35F8F5A461A6084F31088002E76D057
:103C3000534618024B4639001843B0476A6806904D
:103C40000791EFF3108472B61368002BFCD0BFF31A
:103C50005F8F079B002B91DA2B69002B97D006987A
:103C60000799089A099B121A8B410898099906929C
:103C70000793079A914203D807D1069A904204D934
:103C800001225242D317069207935B460121049307
:103C90004B460391029301970096069A079B2800D2
:103CA000FFF7CEFE89E70022002300270892099340
:103CB00000260020B3E700F09DFB069A079B121830
:103CC0004B41994202D804D1904202D9012252427A
:103CD000D317594604910121039149460197029156
:103CE00000962800FFF7ACFE67E7002F01D1002EF9
:103CF0008CD10021604600F053FD43461A685B6892
:103D00000892099343469E68DF68EB684B44013B89
:103D10001B789A461B021843286100207FE7002881
:103D200000D053E70DB03CBC90469946A246AB4646
:103D3000F0BDC046F83A0020FFFFFF0F10B5124C4F
:103D40006368002B04D00A21104800F071FC10BDFC
:103D500023000F4A1021206800F004FD032000F02A
:103D60003DFB032000F044FC0A49032000F08EFBD9
:103D7000FFF718FE084B9C46032360442375074B4E
:103D800080006060DC60DEE7C8140020143C002086
:103D9000DD390010613B001040000034F83A00208B
:103DA00000487047C8140020F0B54546DE46574627
:103DB0004E46E0B585B00092019310AB1B7805002C
:103DC0009B4600239A4698466A68EFF3108972B6BC
:103DD0001368002BFCD0BFF35F8F2E68B47B002CE0
:103DE00050D067003F193368033FDB195A78B2732C
:103DF000002A00D1F27342469A705A701A70AA686B
:103E0000534B94460099019AE3181B0163441960CF
:103E10005A600E9A9A600F9ADA6042463368DB194C
:103E20009A705A701A70737B0393002B40D019005C
:103E3000736822009C46B068E047039932688C465C
:103E40004B006344033B00282BD0D719D318B9701B
:103E50001A78002A00D073E01C70039B73739C4295
:103E600027D0EB681B19013B18786B68BFF35F8F95
:103E700042461A6089F310885346002B26D100026F
:103E8000204307E06B68BFF35F8F1C6089F31088E5
:103E90000120404205B03CBC90469946A246AB4644
:103EA000F0BDD318D7199C703A78002A44D13970E4
:103EB0007473287D009A019B00F02EFB8246002837
:103EC000CFD02100286800F017FDCAE75B46002B21
:103ED00030D00E9B0F990020984703000B4329D048
:103EE00006000F1E15DA0098019902000B00921BC4
:103EF000BB41994202D808D1904206D901235B42C6
:103F0000DC1700930194DA465EE700920193DA46EB
:103F10005AE700F06FFA36184F4100960197B94200
:103F2000ECD8F0D1B042EED901235B42DC1700930C
:103F30000194E8E70020ADE75A70039B3B70B7E7B8
:103F40007A701C70039B73739C4200D089E7B0E7C2
:103F5000FFFFFF0FF0B557464E464546DE460400CC
:103F6000E0B50D0006267642F71736196F4185B089
:103F70008F4200D987E000D182E000F03BFA3200A6
:103F80003B00121A8B41002B00DC87E0674B9946FF
:103F90005A68EFF3108B72B61368002BFCD0BFF396
:103FA0005F8F4B461B6898469B7B9A46002B7BD0C5
:103FB0005B0053444246033B9C46414612680093D3
:103FC000624453788B73002B00D1CB730023494696
:103FD0009370537013708968554A8C465244554902
:103FE00012016244166057609160D36000994246A6
:103FF0008C461268624493705370137043465B7B27
:104000000393002B00D16FE019004046434652460F
:104010005B6880689847039B9C465A006244033A59
:10402000002854D0009940468C46036803999A189A
:10403000634499701178002900D059705346137069
:104040004246039B53739A4551D04B465B68BFF37E
:104050005F8F00221A608BF31088BC46B046009434
:10406000019500266546344F344A7B6A9D424CD800
:10407000B96A414501D29D4247D0009C019D1BE099
:10408000864200D879E70026002700F0B3F9320015
:104090003B00121A8B41002B00DD77E7002B0BD180
:1040A000002A00D072E707E04B465B68BFF35F8FE2
:1040B00052461A608BF310882000290000F0D6F9D0
:1040C00005B03CBC90469946A246AB46F0BD43467F
:1040D0001968009B8A18CB185146917019780029ED
:1040E00000D05170039A1A70434652465A734B4699
:1040F0003200187D3B0000F00FFA0028A5D04B4697
:104100005146186800F0F8FB9FE71168EFF3108044
:1041100072B60B68002BFCD0BFF35F8F1368BFF340
:104120005F8F1E6080F3108820BF9EE7C8140020B8
:10413000FFFFFF0F113A001000400540143C002023
:1041400070B5060000F056F9FA2204000D00920046
:1041500000233000002104F095FB001969418D42D5
:1041600005D901204042C117FFF7F4FE70BD8D4212
:10417000FAD18442F5D8F7E7F8B557464E46DE4601
:104180004546664CE0B581460F006268EFF3108843
:1041900072B61368002BFCD0BFF35F8F2668B57B27
:1041A000002D00D19FE06B005B19033B9A463368FA
:1041B00053441A005B78B373002B00D1F3730023D0
:1041C000937053701370A168554A8C464946AA18DB
:1041D0001201624411605349D360576091603268A4
:1041E0005244937053701370737B9B46002B6DD0B9
:1041F0002A001900B068736898475B465A005A4411
:10420000033A002857D0594633689A185344997096
:104210001178002900D059705B46157073735D45A5
:1042200055D00026E36862685B19013B1B78BFF339
:104230005F8F0021116088F31088002E59D11B0276
:104240001D4320BF6268EFF3108872B61368002B1D
:10425000FCD0BFF35F8FFF232068E9B2427B2B4085
:104260008A4250D05A00924602689A449446524676
:104270006244033A9278002A45D123699D4200D1D5
:1042800022616368BFF35F8F00221A6088F3108891
:10429000254A536A9F4207D8926A01264A4503D2AB
:1042A000FF1A7B1E9F41FEB230003CBC90469946EF
:1042B000A246AB46F8BD534631688A18CB189570B4
:1042C0001978002900D051705A461A707573207DF4
:1042D0004A463B0000F020F9061EA2D029002068C3
:1042E00000F00AFB9EE76368BFF35F8F1D6088F3F1
:1042F00010880D4A0026536A9F42D5D8926A01362B
:104300004A45CDD3D0E7E2682D0A94466344013B89
:104310001B78AB42B5D100F0EFFAB2E7C814002029
:10432000FFFFFF0F113A001000400540F0B5C646F0
:1043300000B5EFF305833F22134018001038EFF368
:10434000108772B61F4D2A68002AFCD0BFF35F8F1A
:10435000012211008140884644461B494C631B4C96
:104360002678A4463400C440224007D1BFF35F8FB3
:104370002A6087F3108804BC9046F0BD4C6A14494B
:10438000820051588C420FD3124BD25843469E4361
:1043900063461E70BFF35F8F00232B6087F3108886
:1043A000002AE8D09047E6E70B4A9B009446634416
:1043B0001A681A60BFF35F8F00232B6087F31088A1
:1043C000D9E7C046280100D000400540483D002004
:1043D000203C00203C350020D03F054010B50100B6
:1043E000024A0348FFF758FA10BDC04610F100100A
:1043F000453D0020044A516A00E01900906A536A62
:104400009942FAD17047C04600400540164A70B53F
:10441000546A00E01C00956A536AA342FAD12A004C
:1044200023008018594105000E008C4216D813D085
:1044300032000D4C636A9342FCD39A420BD10A4B73
:104440002800996AA94203D305E0996A814202D201
:10445000596A9142F9D070BD8242E9D90122012501
:104460006D42EE175242E4E700400540064A536AA7
:104470009942FCD807D1044B02E05A6A914202D11A
:104480009A6A8242F9D370470040054070B5040033
:104490000D00EFF3108672B61A4A1368002BFCD099
:1044A000BFF35F8F002D1BD0200000F0FFFD1649E9
:1044B00088420AD0200000F001FE0121200000F017
:1044C000DBFD0123A340114A1360114BA400E5500A
:1044D000BFF35F8F00220B4B1A6086F3108870BD0C
:1044E0000B4BA200D5500122A2400A4920000B78B4
:1044F00093430B70044900F00BFE0021200000F0F4
:10450000BBFDE5E7280100D02D43001038600540D1
:104510003C350020483D0020F0B5D6464F46464683
:104520002E4CC0B5656A00E00D00A66A616AA9421A
:10453000FAD1AB4248D9EFF3108972B6284C216802
:104540000029FCD0BFF35F8F264901268C460978ED
:1045500086400F00884661463743FFB20F70041D46
:104560001E49A400204D4E636250840063510D6AC1
:10457000002435421BD04D6A00E025008C6AA2461B
:104580004C6AAC42F9D1AB4224D801D1524521D872
:10459000474521D0114B154A1E625E631F23184008
:1045A0001E3B834013606346424601241A70BFF3EA
:1045B0005F8F00220A4B1A6089F3108820001CBC10
:1045C00090469946A246F0BDAB4201D1B242B2D864
:1045D0000124F3E70024EAE70124E8E7004005406E
:1045E000280100D0483D0020203C002080E200E06F
:1045F00010B5EFF3108472B60A490B68002BFCD09B
:10460000BFF35F8F01238340074A08481362027893
:104610009A430270BFF35F8F00230B6084F310880E
:1046200010BDC046280100D000400540483D002094
:10463000024B9C4661448900016070474000003491
:1046400010B50400FFF7AEF901002000FFF7F0FFFE
:10465000FF232371BFF35F8F10BDC04610B5040068
:10466000FFF7A0F901002000FFF7E2FFFF23A3807E
:10467000BFF35F8F10BDC04610B504000120FFF7E7
:104680009DF9044B9C46604480002060BFF35F8F1F
:1046900010BDC04640000034F8B54746CE4680B550
:1046A0004C0003686418033C1A19567807000D0083
:1046B000002E04D128000CBC90469946F8BD71002C
:1046C000891903398846434459788946002159702D
:1046D0005170002D11D07B68320029008068984706
:1046E0003B68002832D01A1943449D701178002984
:1046F00000D059701670A04600E035004B46002BE4
:10470000D8D049463800FFF7C7FF041ED2D00200B8
:104710007B682900B868984763001B19033B3A6817
:10472000002809D1D318424494701978002900D088
:1047300051701D702500BDE74146D31851189D707A
:104740000A78002A00D05A700C70B3E742461C1950
:104750009A18A6701378002B00D06370157035007E
:10476000CCE7C04610B583600023CCB2437301335D
:10477000047342608373C4730068012C06D9421C21
:104780000133DBB2137003329C42F9D8FF23194086
:104790004B005918002340180338437010BDC04621
:1047A000F0B54E4657464546DE46E0B5467B0368C3
:1047B0007400A419033C1A19177883B005008946C0
:1047C000002F1ED1002911D0C07B00282AD0410023
:1047D0000918591803394E70EE73002F06D079006E
:1047E000C9190339884600214344997000233000D9
:1047F00053706F7303B03CBC90469946A246AB46DB
:10480000F0BD7900C919033988465918487882469D
:10481000002809D149460029E5D0E87B0028D6D1F7
:10482000EE73DCE7EE73E1E742005244033A93464D
:104830005B445A78019200225A704A706B680200F9
:104840003900A86898472B68002830D14146504667
:104850005A4659189A1888701078002800D0487065
:104860001770D8465746019A002A2DD0110028000B
:10487000FFF712FF8246002825D0020039006B683E
:10488000A868984753465900514403392B680028BB
:104890001CD04246591898188F70027894461A19FD
:1048A0006446002C00D04C7051460170B2E7594666
:1048B000424659189A188F701078002800D0487016
:1048C00051461170CFE72B681A19A3E75A1898447C
:1048D00093465046424690705A4612789446604637
:1048E0001A19002802D0404664464470584688464B
:1048F000077057468EE7C046F0B54546DE46574638
:104900004E46E0B50C0083B005000023002927D0F7
:104910006600477B01683619033E8819A74233D0E9
:104920008278002A1CD053009B18033BCB181A78BE
:10493000A2421FD142781A7000230278837043701C
:104940009146002A33D1EA7B002A66D053009B1897
:10495000C91803394C70EC730023437001236F7343
:10496000180003B03CBC90469946A246AB46F0BD49
:10497000002AE1D053009B18033BCB185A78A2427F
:10498000F6D142785A70D7E702780192002A46D1D0
:10499000EA7B002A3FD053009B18C91803394F7097
:1049A000EF7300234370019B6B730123D8E7520020
:1049B0004A44033A90468A185778002F42D1EB7B3D
:1049C000002B00D029E14F466E7BEC7300239370DF
:1049D0004370002EC2D03A006B683100A868984737
:1049E00073009B19033B2A68002808D0D31842445F
:1049F0009670197800290CD11F703700AEE7414638
:104A0000D31851189F700A78002A00D05A700E707F
:104A1000A4E75170F0E7EF73C3E7EC739CE7140071
:104A2000A44652006244033A90468A185478A1463C
:104A3000002C58D1EB7B002B00D0F7E0EF73002364
:104A40009370AEE77800C019033882465144487825
:104A50004B7053706B6883463A004946A868984784
:104A60002B68002800D1A2E04246981852469918B7
:104A70004A468A70019002000078002801D0019A0D
:104A8000487017704F465A46002A28D059462800C9
:104A9000FFF702FE8146002820D002006B68390033
:104AA000A86898474B465B004B44033B9C46002854
:104AB0006DD042462B689818624699188F70019005
:104AC0000078002800D083E04A4601980270E97B14
:104AD00098196E7B002951D1019A76E72B684246DE
:104AE0009A180192F3E76000484403388246514423
:104AF00048784B7053706146220083466B68A86803
:104B0000644698472968002878D0524643468A1858
:104B1000CB1894701878002800D050704A46C246CE
:104B20001A705B46002B50D059462800FFF7B4FDA1
:104B30008046002848D0019C020021006B68A868CC
:104B4000984743465A004244D31E2968002844D05F
:104B50005246CB188A189C701078002800D05870E4
:104B600043461370EB7B8819002B00D166E75E008B
:104B7000F318C91803394F70EF7360E74A00944681
:104B800061445B18033B5C70019AEC731EE7296873
:104B90004846CA184346CB18987010788046881942
:104BA0004646002E00D05E701770E04607E741468B
:104BB000524659189A188F701078002800D0487003
:104BC0004946D04611705EE729685346CA18C9E7BE
:104BD0004A46487001990A7079E7CA185346404618
:104BE000CB1898701078844664468819002C00D041
:104BF0005C70019B1370434601931BE75346CA1830
:104C000043464846CB1898701078002800D058705A
:104C1000019B13704B46019383E703267343C91826
:104C200003394C706E7BEC734F46CFE6032673431B
:104C3000C91803394F7001E72D4B2E4A70B51A6021
:104C40002D4A2E4B2E491A6010008B689843FBD1D9
:104C50002C4C2D4DAC4209D20322231D0335ED1AF5
:104C60009543ED1808CC9847AC42FBD100F09AF878
:104C7000264A224B1A60224A9368DB018033FBD11B
:104C80004022234B2348244D9A675A671A67DA66F5
:104C9000A84205D30EE0FFF7E1FC2000AC4209D2A8
:104CA000040003680834002BF5D1FFF7C9FC20008D
:104CB000AC42F5D3194D1A4CC022A168280003F06C
:104CC00053FEA560FEF760FE00F05CFBFFF736F8D0
:104CD000144C154DAC4209D20322231D0335ED1AA5
:104CE0009543ED1808CC9847A542FBD170BDC0464E
:104CF00000E00040BFCDFBFEFE7F3C0000F0004026
:104D000000C00040E81D0020F81D0020FFFFFF014B
:104D100000F00140E01D0020E81D00200000002000
:104D200000ED00E0F81D0020081E002000BEFDE799
:104D3000094A1368002B06D008491818884208D879
:104D4000106018007047064B044918181360884219
:104D5000F6D901235B42F4E7E83600200000042086
:104D60001040002000BEFDE70FB400B5084883B036
:104D700003F01CFF049B002B07D005A9180001912C
:104D800002F0FEFE034803F011FF00BEFDE7C0463F
:104D900040F1001070EB001010B50148FFF7E4FF80
:104DA00034F1001030B50C2083B000F04FFBFEF75B
:104DB000E3FD00280ED0964B964A1A605A609A601E
:104DC000DA601A615A619A61DA611A62924A5A6229
:104DD00003B030BD914CA06700F08CFB0122904BDA
:104DE0001A60636C012BFCD103228E4B1A608B4A34
:104DF000936B012BFCD1022405338B4A01218B4894
:104E0000009400F0D1FA0523894A009401218948D1
:104E100000F0CAFA884B5A68FF2A02D88022520052
:104E20005A6080227A4C7F4B21691201824D1A60B0
:104E3000002900D0E5E0E0217F4B02201A681140F4
:104E4000802252012A431160196848400321014021
:104E5000116004219A681142FCD0802280219201C5
:104E60002A4309011160802252005A60734B23616A
:104E7000734B5968FF2900D8C1E00322684B704882
:104E80001A60012103009A681142FCD0E0251A68DB
:104E9000154080225201024315601B684B400321DC
:104EA000194011600221664A93681942FCD08023A0
:104EB00080219B010343090119608021614B490056
:104EC00051606361604B5A68FF2A00D859608022A4
:104ED0005E4BE16912015C4D1A60002905D06069E2
:104EE00002F0C4FE01300138FDD1E02256490B68C2
:104EF0001A4080235B012B431A60802380229B0190
:104F00002B4312011A608022424B52004A60E36137
:104F10004F4B5968FF2900D85A6080224D4B216AB7
:104F200012014B4D1A60002905D0606902F09EFE07
:104F300001300138FDD1E02245490B681A40802339
:104F40005B012B431A60802380229B012B431201BB
:104F50001A6080235B004B602E4B3F4A23623F4B1D
:104F60005968914201D801325A6080223C4B616AF3
:104F700012013A4D1A60002905D0606902F076FEF0
:104F800001300138FDD1E02234490B681A408023FA
:104F90005B012B431A60802380229B012B4312016B
:104FA0001A608023DB024B601B4B63622D4B5A68F7
:104FB000FF2A02D8802252005A6080222A4BA1691F
:104FC0001201284D1A60002905D0606902F04EFEDA
:104FD00001300138FDD1E02222490B681A408023BC
:104FE0005B012B431A60802380229B012B4312011B
:104FF0001A6080235B004B60124BA361E8E65A60A5
:105000003BE7606902F032FE01300138FDD112E762
:1050100050360020006CDC021BB70000008000400E
:105020003CB0004030B00040002F68590080024082
:1050300000389C1C00C0024030800040001BB700BC
:105040003C800040405973075480004054B00040F9
:105050006080004060B00040FFFF03006C800040B3
:105060006CB000404880004048B00040014B8000D8
:10507000C05870475036002001238340002902D1D8
:10508000034A13607047034A1360034A1360F9E749
:1050900080E100E080E200E000E100E001238340E5
:1050A000014A13607047C04600E200E0024B103036
:1050B0009B688000C058704700ED00E070B50D009F
:1050C000EFF3108672B60F4A1368002BFCD0BFF3C3
:1050D0005F8F0D4B10309B6884001B590B4A934225
:1050E00003D09D4201D0FFF757FE074B9B681D512F
:1050F000BFF35F8FBFF35F8F0022024B1A6086F30E
:10510000108870BD240100D000ED00E0CD0100103A
:10511000F0B54546DE4657464E46E0B50D0083B035
:10512000EFF3108A72B65D4A1368002BFCD0BFF310
:105130005F8F1022914681444A46594B96009B68E6
:105140009C59584B98469C4205D0AC4251D0564F82
:10515000E31B2F2B12D9524B9B689C51BFF35F8FDF
:10516000BFF35F8F00224D4B1A608AF3108803B0A3
:105170003CBC90469946A246AB46F0BD0123834015
:105180009B465A46494B1B681A4000925A46484B68
:105190001A60BFF35F8FFBF766F80190002803D019
:1051A000814501D0FFF7F8FD012322009A43414BCE
:1051B00006209C4613006146DB1B5B415943090DE9
:1051C00093688C4610569D420AD151E043001B184B
:1051D00006209B00FB1899681856A94211D01A00A6
:1051E0000028F3DA009B002B05D15A46304B1A6099
:1051F000B1E71C00AFE75A462F4B1A602B4B1A60E1
:10520000A9E7002825DB4200111889007D1888468F
:10521000A9689960E979D971062169569971A979C6
:105220007F2913D8AD88F91A6D052D154544491904
:10523000E0250905490D2D022943998012181F4BBD
:105240009200BF181A781870BA71CBE7BD21090215
:10525000F3E70199002913D1002A0FD0FF209071A4
:1052600017489080154A1078987163461370B9E713
:1052700013000028C7DA019A002A01D14446F1E759
:10528000104A1149D21A083A5002400D0143998040
:105290000E4952080A43DA80A4E7C046240100D030
:1052A00000ED00E0CD010010F014002000E100E06E
:1052B00080E100E0AAAA000080E200E0463D002074
:1052C00000BDFFFF2A15002000F0FFFF00F8FFFFE0
:1052D000F8B5012504000543FAF7C5FFEFF3108682
:1052E00072B6214A1368002BFCD0BFF35F8F1F4BAF
:1052F0001F4A2100C91A49414A43120D1D49800025
:105300008F6852B23F58AF421CD006215956914285
:1053100026D012215956914224D01E21595691422D
:1053200014D02A2159560320914210D0124B1978DB
:105330001A70A171BFF35F8F00220B4B1A6086F3C6
:105340001088F8BD8B680D491950EFE70220410025
:10535000091889005B18FF21997109499980E5E7CF
:105360000020F4E70120F2E7240100D0F01400202F
:10537000AAAA000000ED00E0463D0020CD0100108B
:1053800000BDFFFF054B064A1360064A13605360D9
:105390009360D36013615361936170478080808014
:1053A00000E400E004E400E0F8B504000C201E0076
:1053B00017000D0002F05AFC4201121A9101891ADD
:1053C000C90009188901380002F050FC069B360418
:1053D0001B031E432368002B21DB184BE2185342AA
:1053E0005A4180235B019C4652421A40144B62444E
:1053F0001A60144B1A60144B170099688F43FBD145
:10540000C023221D9B01134321222560A0601A6046
:105410002268002AFCDA0822E6601A60F8BD3F2301
:1054200022681340AB42D8D1A3681B051B0D8342F1
:10543000D3D1E368002ED0D1F0E7C0460040FDBFD5
:1054400000E0004000F0004000C0004080239B00CE
:105450001843014BD86270470080054010B5802486
:105460001B4BE4051C6000281AD00123194C18437B
:10547000194BDC61194C44401C62596298628021CE
:10548000134BC9051960164816490860E021C90484
:105490001960002A07D18022134B12061A6010BD32
:1054A0000D4BD861EBE753019B1A9B009A180F4BE9
:1054B00012019A4208D80E4B1A60074B5A6080229C
:1054C000094BD2051A60EAE7094A13601A00F4E7AB
:1054D00000B00540D3C007B0008005402D3FF84F15
:1054E000FCFF01000820014000A00540FFFFFF0075
:1054F000F03A0020AA23064A1B0113602F23054916
:10550000D360054B19605368002BFCDA7047C04626
:105510000040024000B0FA00006002409A4200D20F
:10552000885470477047C04610B5002803D04A68B9
:105530000B681100984710BD10B5002801D003F08A
:10554000E5FA10BDF0B557464546DE464E46E0B595
:1055500085B0984610AB1D78139B93469A4602235C
:10556000149A0F00134006000F9C12990193002B10
:105570002DD1013313409C465346002B66D18C42FB
:105580000DD21F2C00D912E10E9B30201B1902E016
:105590000133202C03D001341870A142F8D863469F
:1055A000002B14D0A24512D90E9B30201B191F2CA2
:1055B00021D8AC461500524602E00133202C17D00A
:1055C000013418709442F8D192462A006546D306F9
:1055D0002ED5530519D4002C11D1119B102B00D1BD
:1055E000D9E0022B1FD10E9960330B7001241AE011
:1055F00092462A006546D3063ED5530505D4A142FE
:1056000000D19FE0544500D19CE0119B102B65D048
:10561000022B06D11F2C65D862210E9B1B19197015
:1056200001341F2C5ED830210E9B1B1919700134D8
:105630001F2C57D8002D1BD1530700D570E013073E
:1056400050D520230E990B55013415E06346002BED
:105650006BD0002D00D070E00C2313426DD18C4232
:10566000A0D21F2C90D953462024202BC3D8AEE7BC
:105670002D230E990B550134930736D05B460393C7
:105680001A000E9B029499464B46013C551C185D2E
:1056900039004346B0472A00002CF5D1039A029BFB
:1056A000944663441D00019B002B0FD05B46EB1A10
:1056B00053450BD22A005D46541C43463900202036
:1056C000B0472200631B5345F6D32500280005B0E0
:1056D0003CBC90469946A246AB46F0BD930641D5E8
:1056E0001F2C52D95D46930712D1544538D25B46E0
:1056F00053441B1B0F941C000F9B5A469946551C84
:10570000434639002020B0472A00A542F7D14C4635
:10571000002CC8D00E9B039502942A009946B3E74B
:105720002B230E990B550134A6E78C4200D34EE78C
:105730001F2C00D828E7202449E701235B42994623
:10574000CA448CE7631E002B15D1119B102B19D076
:10575000022B00D147E730230E9901240B7069E733
:105760005D46D5E71F2C00D986E778210E9B1B19D3
:105770001970013455E71199023C1029AED01C0074
:105780000B0045E793060DD5002458210E9B1B19ED
:105790001970013445E7930604D558230E99012466
:1057A0000B7040E778230E9901240B703BE720240F
:1057B000F5E6C046F0B54546DE4657464E46E0B5EE
:1057C0009BB09846259B249C1D00089009910A9245
:1057D0000C9300220023200029000B9402F0FCFC13
:1057E000002800D0A7E10B9A0C9B92469B46802391
:1057F000289ADB001A400E9201D1062326938023BB
:10580000289A1B011A4056465B460D92334300D13D
:1058100061E15B465800CC4B400D9C46604402F071
:1058200009FDCA4ACA4B02F094FCCA4ACA4B02F0AC
:1058300069FC5B46C94A1B031B0B1A4304000D009D
:10584000C74B11005046002202F053FCC54AC64B1C
:1058500002F07FFC02000B002000290002F052FC45
:1058600002F000FD814602F0E5FCC04AC04B040096
:105870000D0002F06EFC0022BE4B02F043FC02F071
:10588000F1FCBD4A0600BD4B2000290002F061FC7E
:10589000040030000D000F9602F0CCFCB84AB94B62
:1058A00002F057FC02000B002000290002F021FC4E
:1058B00002000B0006000F0002F04BFC3200040057
:1058C0000D003B003000390002F01CFC002210905B
:1058D0001191AD4B2000290002F01DFC0022AB4BC2
:1058E00002F010FC02000B002000290002F013FC63
:1058F0000022A74B02F006FC02000B00200029004A
:1059000002F009FC0D008021040032003B00002061
:10591000C90502F0EEFB02000B002000290002F096
:10592000F1FB02000B001098119902F0F4FB002229
:105930008A4B02F0E7FB974A0F9B94466344002290
:105940001B0502F006FC05000C0002000B0050468F
:10595000594602F041FC00280BD001235B429C46D3
:10596000280021000022894BE14402F0D4FB05000D
:105970000C004B46C62663339E42B6410D9B7642D1
:105980000436002B00D0BCE0279B00279E4200D2AB
:105990009F1B0223289A1A400D9203D07342734131
:1059A0005B421F404B46002B07D0504659462A0009
:1059B000230002F0B0FB82468B46002200230B98A6
:1059C0000C9902F009FC002803D0802109065944F3
:1059D0008B4652465B465046594602F018FC00285A
:1059E00000D044E101226C4B52425046594602F02D
:1059F000F3FB002800D0D7E0289A684B03971340A8
:105A00000493269B524602935B46099900920193A8
:105A100008980A9A434600F0FFFC0200002E52D07C
:105A20002020289B089C034059424B415B42184070
:105A3000531C45309A4609994346A0474B46DA170E
:105A40009D18DB0F9946731E55409B46002412AEED
:105A500002E03C00202F0DD028000A2102F006F9B8
:105A6000671C30313419217028000A2102F0FEF839
:105A7000051EEED1052306935B4605930023049390
:105A80000A3303934B4601970096099F089E0293A1
:105A90005246434639003000FFF754FD0D9B02008B
:105AA000002B10D00A99431A279898420BD989469F
:105AB0000500434639002020541CB0474B462200C5
:105AC000E31A9D42F5D810001BB03CBC90469946A5
:105AD000A246AB46F0BD0D9B55465C46002B27D039
:105AE00000239946269B4B4500DDB1E00023269319
:105AF0008023289ADB001A43002328920026994627
:105B000042E723002B43EDD0254A264B5046594609
:105B100002F070FB002800D09FE0269B002B00D1F4
:105B200032E70E9B5A1E9341269AD31A26932BE7EF
:105B30000426994628E78022120694460C9BA2462A
:105B400063449B4653E6C04601FCFFFFFB799F5030
:105B50001344D33FB3C8608B288AC63F0000F03F90
:105B60000000F83F61436F63A787D23F71A37909B3
:105B70004F930A400000E03F1655B5BBB16B0240A1
:105B8000EF39FAFE422EE63F00002C400000244090
:105B900000001840FF030000FFFFEFFFFFF7FFFFCB
:105BA0002D431CEBE2361A3F0A9A289B14009B07F0
:105BB00015D1042F13D9B2464646151FED19BB4621
:105BC000099F0B95330039002020089D541CA847DD
:105BD0000B9B22009C42F5D1B0465F4656464D4B8A
:105BE00049469A464346B94622000425A346B04694
:105BF0001F000B915346013D541C585D09993B0011
:105C0000089EB0472200002DF4D13B005C460B9A61
:105C1000464698460D9B4F469146221D002B00D1CB
:105C2000FCE60A9BD31A9F4200D8F7E6B3464646E5
:105C3000BA46099F330039002020089D541CA8470C
:105C40000A9B2200E31A9A45F4D8B0465E46E5E680
:105C50004A469B1A013B26934AE700222E4B5046A8
:105C6000594602F0B9FA002800D03BE755E70A9BF5
:105C7000289A9A46920717D1032F15D9B2461A00CF
:105C80004646DC1EE419BB46099F0B9433003900DD
:105C90002020089C551CA0470B9B2A009D42F5D153
:105CA000B0465F465646AA461C4B49469B4643466D
:105CB000B94652460324B0461F000B915B46013C97
:105CC000551C185D09993B00089EB0472A00002C1E
:105CD000F4D13B000B9A4F469146524646469846B1
:105CE0000D9B0332002B00D198E60A9BD31A9F42EA
:105CF00000D893E6B3464646BA46099F33003900BA
:105D00002020089D541CA8470A9B2200E31A9A45AC
:105D1000F4D89AE734F3001080842E4130F3001059
:105D2000F0B5DE4657464E464546E0B597B005000D
:105D30000E0093461F00209A219B1000190002F0CC
:105D400066FA002800D0AEE2209821990122C54BC6
:105D5000524202F041FA002800D034E12098219903
:105D60000122C14B524202F04DFA002800D0C1E09E
:105D7000209821990022BD4B02F044FA002800D05F
:105D800008E1209821990022B94B02F025FA002859
:105D900000D0FFE0209821990022002302F01CFA95
:105DA000002800D074E200230D938023249ADB00A6
:105DB0001A40904600D0BAE10023AE4C06930794F7
:105DC0000EAB06249A462098219902F04BFA0990CE
:105DD00002F030FA02000B002098219902F089F9B4
:105DE000069A079B02F0B5F90A900B9102F05EFA51
:105DF00081460C9002F01AFA02000B000A980B99E7
:105E000002F077F900229C4B0A900B9102F0FAF90C
:105E1000002800D1E5E14B46013318000C9302F055
:105E200005FA069A079B02F0E5F9002800D0FBE18D
:105E3000002C00D09CE1099C200002F0FBF902003C
:105E40000B002098219902F054F900228A4B069009
:105E5000079102F0C1F9002800D1D5E14346202B7B
:105E600000D112E15C1C099B0A211800994601F03F
:105E7000D5FE424653463031995448460A2101F036
:105E8000CDFEA046814600281ED05346A846BA46FD
:105E90004D461F00B14600E03400202C00D162E2E4
:105EA00028000A2101F0BAFE661C30313C1921702D
:105EB00028000A2101F0B2FE051EEDD13B00454647
:105EC0005746B0469A464E460323249A1340012B68
:105ED00000D1B1E142462024202A00D1DCE00D9A15
:105EE000002A00D135E242465146541C40462D223C
:105EF0000A54D1E0249B5B0700D5ADE05F4B9A4686
:105F0000032398465B460693249B9B0718D1239B4B
:105F1000434500D84EE25B441C004346E41AB946B0
:105F20005A4637002E002500541C4B4639002020CD
:105F3000B0472200AC42F7D135003E004F460694F0
:105F4000B14644465646BA462F00069A013C551CB7
:105F5000305D53464946B8472A00002CF6D1069BCF
:105F60003D0043441A00249B9B0724D55B4623999C
:105F7000D31A99421FD92E00D0464F460D004346F2
:105F800039002020541CB0475B462200E31A9D4292
:105F9000F5D810E0249B5A460493239B31000393C9
:105FA000229B28000293209B219C009301943B009C
:105FB000FFF700FC0200100017B03CBC9046994669
:105FC000A246AB46F0BD249BD8469B0718D1239B25
:105FD000042B15D95B461C1F239BB8469C46644482
:105FE00037005A462E002500541C43463900202015
:105FF000B0472200AC42F7D135003E004746A046EC
:106000001F4BB9464246370004249A462E00534699
:10601000013C551C185D39004B46B0472A00002C46
:10602000F5D14246249B350004323E009B07C2D581
:106030005B462399D31A9942BDD93700C8462E0032
:106040000D00434639002020541CB0475B46220017
:10605000E31A9D42F5D8AEE70A4B9A4604239846C8
:1060600050E7C046FFFFEFFFFFFFEF7F65CDCD415B
:1060700065CDCDC180842E410000E03F44F3001087
:1060800034F300103CF30010A2460323249A13407B
:10609000012B00D1CEE02024D846002B17D1239B22
:1060A0009C4214D25B441B1BB8465A463700A1469B
:1060B0002E001D00541C434639002020B04722000A
:1060C000AC42F7D135003E004746A0464C46434619
:1060D0004246A146B84637002E0006935346013C7F
:1060E000551C185D39004346B0472A00002CF5D1F5
:1060F00006994B468C4663441A00249B35003E00AB
:106100009B0700D457E75B462399D31A994200D8DE
:1061100051E737002E000D00434639002020541C63
:10612000B0475B462200E31A9D42F5D843E7229B25
:10613000092B00D85BE10EAB9A4630235246137010
:1061400001229046229B2F325C1E4146203B504646
:1061500005E0013C425401319C4200D1EEE0092CA3
:10616000F7D10022A84B88468246069207932AE67A
:106170004346202B89D0631E069301230C9C434485
:1061800020000A21994601F071FD53464246303104
:10619000995420000A2101F069FD041E00D122E17A
:1061A000A84625004C46B9465746B24612E0069B23
:1061B0002800013B0A21069301F058FD661C30318E
:1061C0003C19217028000A2101F050FD051E00D164
:1061D000CFE03400202CEAD156464546BA464F4619
:1061E00053E700220A980B99884B01F0F5FF00282D
:1061F00000D01DE60C9B002B02D0DB0700D417E675
:106200000C9B01330C9313E60022069807997F4BF1
:1062100001F0F8FF002800D020E60123A446234027
:106220009C446346099319E6099B013309930023B3
:106230000C93FDE520239846239B002B00D1BFE063
:106240000D9B002B03D1249A0C33134202D0239BC5
:10625000013B2393239B434500D8B1E042463023C2
:10626000202A00D1B1E0424650462399541C835461
:106270008C4200D1A1E02200202CF7D120239946A6
:106280005B46B8468246370006935A462E0025E7FD
:10629000209A219B0020002101F02BFF0123209058
:1062A00021910D9381E5249BD8469B0718D1239B10
:1062B000032B15D95B46DC1E239BB8469C466444E1
:1062C00037005A462E002500541C43463900202032
:1062D000B0472200AC42F7D135003E004746A04609
:1062E0004B4BB9464246370003249A462E0053468C
:1062F000013C551C185D39004B46B0472A00002C64
:10630000F5D14246249B350003323E009B0700D462
:1063100051E65B462399D31A994200D84BE63700E1
:10632000C8462E000D00434639002020541CB047BB
:106330005B462200E31A9D42F5D83CE6354BE2006D
:106340009B181A685B68069207932023824698463A
:1063500039E5249A52073BD542465146541C4046E3
:106360002B220A5498E63B00454657464E469A462D
:106370008BE64546B0465646BA464F464346202B26
:1063800000D182E6069B40461A0042441100544662
:106390003022002B29D0431C2254202B00D173E63D
:1063A00018008B42F7D1A2465A1C904651462E2225
:1063B000CA5453E55B460693C2E5239B8246984642
:1063C00042460123202A00D089E52024D8467EE6D3
:1063D000249A4446120700D45EE6202251464046E5
:1063E00001340A5458E6C846C8E74346DCE7DA00F9
:1063F000084B9B185C681B6806930794002398461B
:106400000EAB229C9A46DEE465CDCD410000E03F14
:1064100030F3001048F30010F0B557464E4645469D
:10642000DE46E0B597B00792012206000F002098E3
:10643000219998465242CF4B01F0E4FE00284DD0FE
:10644000249B5B0700D541E1CB4B9A4603239B4637
:10645000079A249B14009B0711D1239B9B450ED2C6
:10646000190013008C4663441D005B46ED1A541C52
:10647000434639002020B0472200AC42F7D1B9464C
:10648000220037005D465646A246013D541C705D11
:1064900043464946B8472200002DF6D15246249B78
:1064A0003E005A444F469B0710D507992398531A2C
:1064B00098420BD989460500434639002020541CD8
:1064C000B0474B462200E31A9D42F5D8100017B0A2
:1064D0003CBC90469946A246AB46F0BD00222098AF
:1064E0002199A64B01F08EFE002800D0F3E0209801
:1064F00021990022A24B01F06FFE002800D0EAE0B3
:10650000209821990022002301F066FE002800D087
:1065100092E100230D938025249BED001D4000D0C7
:1065200017E10023974C089309940EAB06249B4671
:106530002098219901F096FE81460C9001F07AFE98
:1065400002000B002098219901F0D3FD089A099BC5
:1065500001F0FFFD0A900B9101F0A8FE824601F0C8
:1065600065FE02000B000A980B9901F0C2FD0022A3
:10657000854B0A900B9101F045FE002800D148E1BF
:1065800001239C46E244504601F050FE089A099BC4
:1065900001F030FE002800D09CE1002C00D006E184
:1065A0000C9C200001F046FE02000B00209821996F
:1065B00001F09FFD0022744B0890099101F00CFE40
:1065C000002800D176E1202D00D1BAE00C9B0A21F1
:1065D0001800994601F022FB5B4630315955484678
:1065E0000A2101F01BFB6C1C8146250000281AD0F3
:1065F0004D46BA46B1465F4600E03400202C00D13B
:1066000003E128000A2101F009FB661C30313C1926
:10661000217028000A2101F001FB051EEDD1350093
:10662000BB464E4657460323249A1340012B00D104
:106630000EE12024202D0BD00D9A002A00D034E149
:10664000249A520700D46FE12B2259466C1C4A55FC
:10665000079A1500002B12D1239B9C420FD21900E0
:1066600013008C4663441B1BA1461C00551C43466B
:1066700039002020B0472A00A542F7D14C46A24657
:10668000A9462A005B46013C551C185D390043466B
:10669000B0472A00002CF5D14B4653441A00249BE6
:1066A0009B0700D412E707992398531A834200D31B
:1066B0000CE789460500434639002020541CB047AA
:1066C0004B462200E31A9D42F5D8FFE62F4B9A462F
:1066D00004239B46BCE6209A219B1000190001F080
:1066E00096FD00281AD1209821990122284B524268
:1066F00001F072FD002811D1249B079A0493239B7B
:1067000039000393229B30000293209B219C00932D
:1067100001944346FFF74EF80200D7E6249B079A00
:106720000493239B39000393229B30000293209B08
:10673000219C009301944346FFF7F2FA0200C5E65C
:1067400083460323249A1340012B00D17FE02024A9
:106750007EE7229B092B00D8F2E00EAB9B4630234C
:106760005A461370229B01255C1E3022203B59465D
:1067700015E0C046FFFFEF7F44F3001065CDCD412B
:1067800065CDCDC180842E410000E03F3CF3001078
:10679000FFFFEFFF013C4A5501359C427BD0092C9D
:1067A000F8D100226C4B8B4608920993C0E6202D4D
:1067B000C7D06B1C50460A21994601F057FA5B4638
:1067C0003031595550460A2101F050FA013C8246B9
:1067D000002800D1B2E04B465546B146BA465F4666
:1067E00011E09B4628000A215E1CBB4401F03EFAE2
:1067F0005B463031197028000A2101F037FA013C5C
:10680000051E76D03300202BEBD1BB464E465746B3
:1068100097E700220A980B99504B01F0DDFC002805
:1068200000D0BAE65346002B02D0DB0700D4B4E612
:1068300001239C46E244B0E6209A219B00200021DF
:1068400001F057FC0123209021910D9363E6202550
:10685000239B002B46D00D9B002B03D1249A0C3395
:10686000134202D0239B013B2393239BAB4239D994
:106870003023202D3AD05946239A6C1C4B55944214
:106880002ED02500202CF8D12023079D8B469A4638
:10689000A9462A00F6E6324BE2009B181A685B68AC
:1068A0008B4608920993202542E62D2259466C1CFE
:1068B0004A55CDE6002208980999284B01F0A2FC20
:1068C000002800D07FE60123A44623409C44634671
:1068D0000C9378E64B4601330C9300239A465CE612
:1068E0008B46239D0123202D00D0A5E62024079D63
:1068F000C5E63500BB464E465746202D00D120E761
:10690000611930222B00002C09D058466B1C4255CF
:10691000202B00D114E71D008B42F7D183462E2295
:1069200059465D1CCA544EE6249A2C00120700D426
:106930008EE62022594601344A5589E64D46DCE769
:10694000DA00074B00259B185C681B6808930994C4
:106950000EAB229C9B46EBE565CDCD410000E03FB0
:1069600048F30010F0B5DE4657464E464546E0B5C2
:10697000A9B01E00329B90460A93BF4ABF4B834684
:106980008A461A60002968D0D1460025DA46307858
:1069900000280BD0013625281BD02A004346494643
:1069A000D04730786C1C25000028F3D1D3462A004C
:1069B000CA46454501D343465A1E43465146002028
:1069C000D847280029B03CBC90469946A246AB4621
:1069D000F0BD102330789B460E3B9C460300203BC5
:1069E000721CDBB20027A64C1100102B0DD89B00A7
:1069F000E3589F46012316001F433078721C0300A2
:106A0000203BDBB21100102BF1D90300303B092BE6
:106A100000D8AEE100239B462A2800D1CFE1002414
:106A20002E2800D1BDE10300683BDBB2122B00D958
:106A3000D3E3944A9B00D3589F46042316001F4378
:106A4000DBE7634616001F43D7E75B4616001F438C
:106A5000D3E7082316001F43CFE78B4B9B4693E7F2
:106A600080235B0070781F434E1C0300253BDBB284
:106A7000532B92D8854A9B00D3589F4670786C2838
:106A800001D100F0C0FC80235B001F434E1CECE7EB
:106A900080239B0070781F434E1CE6E770786828BF
:106AA00001D100F019FD80234E1C1F43DDE746286D
:106AB00001D100F058FC07220A9B04970733934347
:106AC000013294469C4462460A925A4602940392CA
:106AD0005C681B682A00009301944946434650466F
:106AE000FFF71EF9050052E72A006C1C4346494691
:106AF0002520D04725004AE70A9B1A1D1B680C92E7
:106B00000A931878002C00D0ABE3002801D100F0E4
:106B1000A2FF02211A00494201239C4643460890E5
:106B20000B9307E00A98634680469B1A43445B1820
:106B3000002B03D001321378002BF3D10B9B089864
:106B400098460A9BD31A08938023DB003B400B93A3
:106B500003D0089BA34200D9089402231F4001D10F
:106B600000F0DBFC002801D100F0BCFC0B9B002BEB
:106B700001D000F062FE0A9B2A005C1B23005446F1
:106B8000B2464E46B946474698463B003100551C32
:106B9000A0474346585D2A000028F6D1B8464F4624
:106BA000B1465646A246002F01D000F09BFC0C9B3C
:106BB0000A93ECE60A9B1A1D1B689346002B00D132
:106BC00042E3212217430A970F2020A90B940022A9
:106BD000089184460C0002E020290CD00A0061468E
:106BE0001940CFB238003730092900D80738511C76
:106BF000A0541B09F0D10B9C0A9B0191069308231A
:106C000005930833039300230293089B2A00009303
:106C10000494434649465046FEF794FC5B46050003
:106C20000A93B4E60A9B6C1C04330B940893BB07CD
:106C300000D478E30A9B2A00187849464346D04797
:106C40005B465D44012B01D800F07EFE2B005746C9
:106C50004D46B146464698460B9A541C33002900CF
:106C60002020B84722004445F7D1B046BA464E46E8
:106C7000A946250073E3C04665690010EC3A002080
:106C800050F1001094F1001025550010E0F10010B3
:106C9000782800D1ECE2582801D100F067FC6F2879
:106CA00001D100F051FD622801D100F04FFE102308
:106CB0003A009A430B92692801D000F039FF7B0516
:106CC00001D500F02BFD80239B001F40F73BFF3BCD
:106CD0000C93002F01D000F0C3FC80230B9A5B00C3
:106CE0001A40130094460A9A04320D92002B01D0E8
:106CF00000F0CAFD0B9B5B0601D400F0BCFD0A9BB3
:106D00001B78DA1798185040DA0F0A92002B08D136
:106D10000B9A1033110099430B91520501D500F0E5
:106D2000A2FE0B9B61279B0600D541275A4620AB4C
:106D3000FFB20E950F94B34608930A3F6446109233
:106D40000C9D1E000CE03033DBB2621C3355002872
:106D500001D100F017FC202A01D100F013FC14002F
:106D6000290000F083FFCBB20929ECD9DB19DBB293
:106D7000EBE70023010001E0160001329800C01883
:106D8000400040181178030008003038303B0928D3
:106D9000F2D908009B46B11C002416002E2800D012
:106DA00041E680237078DB001F430300303B092B52
:106DB00015D92A2800D1DAE20E00013133E60A990A
:106DC0000B1D09688B46002904DA02210F4359463E
:106DD00049428B467078B11C0A9316001FE60300E7
:106DE00000E03100A00000194000C0184B78303896
:106DF0001A00303A4E1C0400092AF2D91800023158
:106E000011E6202302009A43472A02D180231B0166
:106E10001F4302239843452801D11E331F430722F5
:106E20000A9B07339343013294469C446246196897
:106E30005868089109900A9203000A000B910C907F
:106E40000898099901F0E3F9002800D09BE201229B
:106E5000E34B52420B980C9901F0D4F90122E14B1B
:106E60005242002800D0D5E20B980C9901F0B4F9F9
:106E7000002800D0A2E3002200230B980C9901F017
:106E8000ABF9002801D000F055FD0B9A0C9B08923D
:106E90000D938023DB003B40179300D10624802311
:106EA0000D9A1B013B400E93130008990F910B4361
:106EB00001D100F0B6FCCC4B50009C46400D604424
:106EC00001F0B8F9C94ACA4B01F043F9C94ACA4BA3
:106ED00001F018F90D9A109011911303C74A0F99F8
:106EE0001B0B1A431B921A9100221A981B99C44B30
:106EF00001F0FFF8C34AC44B01F02BF902000B006C
:106F00001098119901F0FEF801F0ACF90F9001F022
:106F100091F9BE4ABE4B1090119101F01AF900226E
:106F2000BC4B01F0EFF801F09DF9BB4ABB4B16904A
:106F30001098119901F00DF910901191169801F027
:106F400079F9B74AB74B01F004F902000B00109829
:106F5000119901F0CEF802000B001090119101F090
:106F6000F8F8149015911098119902000B0001F097
:106F7000C9F800221E901F9114981599AA4B01F090
:106F8000CAF80022A94B01F0BDF802000B001498CA
:106F9000159901F0C0F80022A54B01F0B3F80200EA
:106FA0000B001498159901F0B6F8109A119B1490E3
:106FB000159180210020C90501F09BF802000B000B
:106FC0001498159901F09EF802000B001E981F9965
:106FD00001F0A1F80022894B01F094F8169B1A00E9
:106FE000944B9C46624413051D9300231C931C9AEA
:106FF0001D9B01F0AEF81490020016910B0008984A
:107000000D9901F0E9F800280AD00F9B1498013B74
:107010000F9316990022854B01F07DF8149016917C
:10702000C6230F9A633293429B415B420433109311
:107030000E9B002B1DD0169B149A134301D100F018
:10704000C1FC7D4A7D4B08980D9901F0D3F80028CA
:1070500009D000227A4B08980D9901F0BDF800285C
:1070600001D000F0AFFC002C03D0179B5A1E9341B7
:10707000E41A00230E93109B9B4502D95A46D31A5B
:107080000E9302233B40179306D0109B5A42534164
:107090000E9A5B421A400E920F9B002B07D0089865
:1070A0000D99149A169B01F036F808900D91002264
:1070B00000230B980C9901F08FF8002805D0802050
:1070C000000684460D9961440D910D99089A0B00B4
:1070D000089801F09CF8002801D000F0E2FC0122A1
:1070E000404B524208980D9901F076F8002801D0E3
:1070F00000F075FC534B089A3B4004930E9B02949E
:1071000003930D9B49460092019350462A00434643
:10711000FFF782F90200109B002B00D170E12020C4
:1071200007403B0059424B4100275B42511C18402D
:107130000B91434649464530D0470F9A109BD117D3
:10714000013B54180D93D20F20AB0E954C403D00DF
:107150000C9208930F961F0002E03500202E0DD0F0
:1071600020000A2100F082FD6E1C30317D1929704B
:1071700020000A2100F07AFD041EEED105230693BB
:107180000D9B32000593002304930A3303930C9B59
:1071900001920293089B0B9A00934946434650463E
:1071A0000E9D0F9EFEF7CEF9179B0200002B00D11B
:1071B00026E1431B9B4500D822E15C465746531C01
:1071C0009A46494643462020B8475246531B9C42A4
:1071D000F5D8BA461500FFF7DAFB0E0045E4C046C5
:1071E000FFFFEF7FFFFFEFFF01FCFFFFFB799F50E9
:1071F0001344D33FB3C8608B288AC63F0000F03FDA
:107200000000F83F61436F63A787D23F71A37909FC
:107210004F930A400000E03F1655B5BBB16B0240EA
:10722000EF39FAFE422EE63F00002C4000002440D9
:1072300000001840FF0300002D431CEBE2361A3F0C
:1072400080842E41FFF7FFFF102239009143113255
:1072500011430A917A0500D4B6E420AB00210893CB
:10726000CAE4002801D100F0F6FB611E1A0053E4C5
:1072700080231022DB003B400C920C2297430B979B
:107280003A00002B02D001239A430B9280270B9BDC
:10729000BF001F40692800D11BE5642800D118E514
:1072A000002F00D07CE280230B9A5B001A40130071
:1072B00094460A9A04320D92002B00D050E30B9BA7
:1072C0005B0600D445E30A9B1878002807D10B9A87
:1072D0001023110099430B91520500D5BFE30B9B7E
:1072E00061279B0600D5412720ABFFB20A950E947B
:1072F0000F9608930A3F65460C9C1E000AE0303347
:10730000DBB26A1C7355002800D111E2202A00D19B
:107310000EE21500210000F0A9FCCBB20929EED93C
:10732000DB19DBB2EDE75B46012B00D8A7E36B1E50
:107330009B4433005E469B4601E0250001344346F2
:107340002A00494620202700D047B442F5D15E46A6
:1073500002350A9B3A00187849464346D047089BB5
:107360000A93FFF714FB20231F43FFF7A4FB0A9A9D
:10737000B0781468F11CE343DB171C40131D0A931B
:107380000236FFF750FB2C00BB0710D15B46032BE6
:107390000DD9EC1E23002A005B440893434649465E
:1073A0002020541CD047089B22009C42F6D1032386
:1073B0000893DC4B22000B932B003D001F00089B21
:1073C0000B98511C013B0C910893C05C4946434605
:1073D000D047089B0C9A002BF2D13B002F00E21CF7
:1073E0001D00BB070CD5531B9B4509D95F46541C98
:1073F000434649462020D0472200631B9F42F6D8CF
:107400001500FFF7C4FAC0239B00B0781F43033672
:10741000FFF72BFB0B980C9900F0DEFE002800D044
:10742000CCE07B0700D46BE2BF4B089304230C93A2
:107430000B95BB071CD10C9B9B4500D82DE35A46EE
:107440005419E41A33002A004E46A94655469A4676
:107450000D97571C434631002020A8473A00BC42F4
:10746000F7D15346AA464D46B1461E000B970D9FD5
:10747000330056469A460B9A0C9C0D95089B013C8E
:10748000551C185D49464346B0472A00002CF5D1EB
:1074900053460B99B2468C461E000C9B0D9D6344CF
:1074A0001A00BB07ACD5531B9B45A9D933005C46DA
:1074B0004E4657469946531C9A4631004346202073
:1074C000B8475246531B9C42F5D84B46BA46B14684
:1074D00015001E00FFF75BFAC023B0781F43033688
:1074E000FFF7C3FA089B9B4501D8FFF760FB5A469C
:1074F0005419E41A33002A004E465746994601357E
:10750000434631002020B8472A00A542F7D14B4618
:10751000BA46B1461E00FFF74AFB089A531C934532
:1075200000D8A8E25B465B199B1A08971F0033003E
:107530002A004E46A14654469A460135434631003C
:107540002020A0472A00BD42F7D15346A2464C4610
:10755000B1461E005B460133089F08930A9B1878CA
:10756000002801D0FFF702FBFFF721FB0C233A00B4
:107570009A4314331A430B927B0500D4C7E01023BF
:107580000C9380E6109B5E469B460E9D0F9C0B9BCA
:10759000049406935B4605930C9B03930A9B02930A
:1075A000089B019200932A00434649465046FDF746
:1075B000C9FF0D9B05000A93FFF7E9F90B95BB077F
:1075C0001BD15B46042B00D8B0E233002C1F2A00ED
:1075D0004E46A94655469A465C440897571C434672
:1075E00031002020A8473A00A742F7D15346AA46C7
:1075F0004D46B1461E000B97089F4C4B0424089340
:1076000033004E46B94657469A460B9A0C95089B4E
:10761000013C551C185D31004346B8472A00002C38
:10762000F5D15346BA464F460B9AB1460C9D1E0003
:107630000432BB0700D4E3E6531B9B4500D8DFE6CA
:1076400033005C464E4657469946531C9A463100D5
:1076500043462020B8475246531B9C42F5D834E796
:1076600007220A9B07339343013294469C446246A7
:107670005F680A921A68FB1718931993189819995A
:107680000300534012930B007B4013939446129ACD
:10769000139B121A8B41129213936246FB0F1493A1
:1076A0003A4307D10B9A1023110099430B915205CD
:1076B00000D5E7E10B9A6123920600D54123DBB2A6
:1076C00020AA0A3B0E950F9410960027129C139D3A
:1076D00008920D930C9E0CE03032D2B2089C7B1CB9
:1076E000E255020004000D000A433FD0202B3DD09C
:1076F0001F00320000232000290000F0F9FAD2B266
:10770000092AE9D90D9B9C466244D2B2E6E7802360
:107710009B001F40F13BFF3B0C93C1E50A230C93F8
:10772000B1E5C04630F300103CF3001034F3001014
:107730000A9D0E9C0F9E0B9B049406935B4605933B
:107740000C9B039300232AE708230C938023DB0080
:107750003B40642800D090E53A000B97002B00D006
:1077600091E58027BF001740FFF7B3FA12941395F5
:10777000109E0F9C0E9D0B9A049406925A460592F9
:107780000C9A01930392149A0292089B2A00009388
:10779000494643465046FDF7D5FE0500FFF7F7F88A
:1077A00007220A9B07339343013294469C44624666
:1077B00003CB03000A920B4307D10B9A1033170037
:1077C0009F430B97520500D563E10B9A6123920604
:1077D00000D54123DBB220AA0A3B0E950F94002767
:1077E00008920D930C9C109615000CE03032D1B22B
:1077F000E95518007A1C3100334300D185E0202A76
:1078000000D182E017002200002300F071FAD2B20A
:1078100003000E00092AE9D90D998C466244D1B2C1
:10782000E6E70E9B002B00D0C7E00D9B149116934A
:107830000423109300230F931BE40A9B64195B1B22
:107840000A9333002A004E46B94657469A4608E046
:1078500043463100551CB8470A9B585D002862D04A
:107860002A00A242F4D153461500BA464F46B1460B
:107870001E00FFF798F90B9B1B0600D4F7E00A9B4C
:1078800000229B5EFFF73DFA0A9B1B68DA179818E7
:107890005040DA0F0E92002B06D10B9A10331100D4
:1078A00099430B9152051FD40B9A6123920600D580
:1078B0004123DBB220AA0A3B08920A9309E0303345
:1078C000DBB208997A1CCB55002810D0202A0ED0A4
:1078D00017000C9900F0CAF9CBB20929EFD90A9A1E
:1078E00094466344DBB2ECE7002220AB08930B9B89
:1078F000049406935B4605930C9B03930E9B4EE604
:107900008D4B089303230C9392E50E9D0F9C109EC4
:107910000B9B049406935B4605930C9B0192039387
:107920000023029331E75346BA464F46B1461E0044
:10793000FFF739F98022120694460B9B08930C9BA3
:1079400063440D93FFF7A5FA250008E502230C9385
:10795000FCE60B9B1B0600D498E00A9B1888B4E455
:107960000A9B1868002806D10B9A1023110099432E
:107970000B91520573D40B9A6123920600D54123D3
:10798000DBB220AA0A3B08920A930BE03033DBB249
:1079900008997A1CCB55002800D1CCE6202A00D1CA
:1079A000C9E617000C9900F061F9CBB20929EDD9AD
:1079B0000A9A94466344DBB2EAE70D9B149116934E
:1079C00000230F930F9B9C4257DDE41A013C802358
:1079D000DB001F43002310930F93FFF74AFB0B9527
:1079E000BB070FD10E9B042B59D99C462A002C1F94
:1079F0006444531C0B93494643462020D0470B9ABE
:107A00009442F6D104244D4B0B9A08930C97089B93
:107A1000013C571C185D49464346D0473A00002CAC
:107A2000F5D10B9A179B0C9F0432002B01D1FFF765
:107A300072FB0E99531B8B4201D3FFF76CFB43463D
:107A400049462020541CD0470E992200631B8B42CC
:107A5000F5D3FFF760FB00230893FFF775F820AB21
:107A60000022089367E620AB002208938FE50A9B6B
:107A70001B68FFF746F9089372E50024A7E72F007B
:107A8000250066E420AA0023089274E60A9B186881
:107A90001BE420AB002208933AE70B95E8E40B9532
:107AA000B0E72C00BB0710D10E9B032B0DD99C46D1
:107AB0002A00EC1E64440894434649462020541C86
:107AC000D047089B2200A342F6D1032308931C4B06
:107AD00022000B932B003D001F00089B0B98511CAC
:107AE000013B0C910893C05C49464346D047089B34
:107AF0000C9A002BF2D13B002F001D00179BE21CBB
:107B0000002B01D1FFF707FB0E99531B8B4201D3CA
:107B1000FFF701FB434649462020541CD0470E99ED
:107B20002200631B8B42F5D3FFF7F5FA0B9564E552
:107B3000063B17000C9309E644F3001034F30010E1
:107B400030F3001000B583B0009313000A00010069
:107B50000248FEF707FF03B000BDC0461D550010E8
:107B600000B585B0039101210290009303481300F2
:107B70004A4202A9FEF7F6FE05B000BD29550010E5
:107B800010B5094A84B01468002C09D00122009174
:107B90000300524203A90548A047012004B010BDCC
:107BA00001F004F80020F9E7EC3A00203955001004
:107BB00001480421014B184740150020E17B0010CB
:107BC000142310B50100188804331B88984710BD92
:107BD000162310B50100188802331B88984710BD82
:107BE000F0B5C64600B5002916D0142304000125BF
:107BF00098461827890046184346216818883B880C
:107C0000984701C4431E984140420540A642F3D123
:107C1000280004BC9046F0BD0125F9E7124A936F95
:107C20009B0815D29066D166002905D0FFE7FFE7D3
:107C3000FFE7516F106F704704B580210906C21726
:107C40005140002800D0C84306F016FE002104BDB4
:107C5000F0B5146E556E576F166FFFF7E3FF14669D
:107C6000556657671667F0BD000000D0114A936F44
:107C70009B0813D210665166002905D0FFE7FFE785
:107C8000FFE7516F106F704704B5002801D0002046
:107C9000C04306F0F1FD002104BDC046F0B5146EEE
:107CA000556E576F166FFFF7E5FF146655665767F9
:107CB0001667F0BD000000D094464E4A926F9208BD
:107CC000624601D230E0C046F0B54A4EB56F6D084D
:107CD000FCD3346E756E776F366F00F025F89446DE
:107CE000444A14665566576716676246F0BDC0463B
:107CF0009446404A926F9208624601D258E0C046CC
:107D0000F0B53C4EB56F6D08FCD3346E756E776F71
:107D1000366F00F04DF89446364A1466556657673C
:107D200016676246F0BDC046002B24DB11D0002947
:107D30003EDA00B5C943404200D1013100F038F8C5
:107D4000C943404200D10131DB43524200D10133EB
:107D500000BD002AEBD1002801D1002905D0002068
:107D6000C90FC90701D1C043410800B506F074FD31
:107D70000022002300BD00B500290ADBDB4352428C
:107D800000D1013300F014F8C943404200D1013161
:107D900000BDC943404200D10131DB43524200D112
:107DA000013300F005F8DB43524200D1013300BD3E
:107DB000002923D1002B18D1002A0CD0BC460D4F2E
:107DC00038667A6600210023FFE7FFE7FFE77A6F56
:107DD000386F67467047002801D00748010000B59A
:107DE00006F03AFD0022002300BD02000B00002037
:107DF00000217047000000D0FFFFFFFF002B00D0E4
:107E0000BFE0130C28D1002AE7D080B4114F3966A7
:107E10007A66FFE7FFE730B4040C7B6F396F1B0411
:107E200023433B667A66FFE7FFE7FFE7C04684B27D
:107E30007B6F3D6F1B0423433B667A66FFE7FFE7DA
:107E4000C04600232C042D0C7A6F386F001969414D
:107E5000B0BC7047000000D0F0B594460025140E69
:107E600001D112020835140F01D112010435940F0B
:107E700001D192000235D40F01D152000135D40B4B
:107E80000134254F7C66254C3C660E0C93B2FFE70F
:107E9000FFE7FFE73C6F6643360C7703BE4673434C
:107EA000DF0B5B04C01AB941130C7343DB18C91A0A
:107EB000CE086643360CB64493B273431F0F1B01C2
:107EC000C01AB941130C73431F0B1B05C01AB941EB
:107ED000860D8F023E436643360C092D24DB520A81
:107EE0007243801A7703460A6643360C16235B1BDF
:107EF000DE40DF40BF1964466643821B704604358E
:107F000006330100D940A840C01900D30131A24274
:107F100006D20023F0BD0000000000D0FFFFFFFFED
:107F2000121B0130F3D3F1E709277F1BFE406446A3
:107F3000A2B27243801A00D20139220C7243130C90
:107F40001204821A99410B00704604351337010060
:107F5000F940A840801900D30131002B02D1A24280
:107F60000AD2F0BD013000D30131121BFAD2013B1D
:107F7000F8D1A24200D2F0BD013000D30131121B72
:107F8000F7E7F0B51C0C00D080E00CB400251C0A0B
:107F900004D11B02160E3343120208351C0B04D108
:107FA0001B01160F3343120104359C0B04D19B00B7
:107FB000960F334392000235DC0B02D192185B41DD
:107FC00001351C00971864410134464F7C66464CCD
:107FD0003C660E0CFFE7FFE7FFE7C0463C6F6643D9
:107FE000360C7703BE4697B27743C01B00D20139E7
:107FF000C01B00D201399FB27743C91BC91B170CA4
:1080000077437E04FF0B801BB941CE086643360CD4
:108010000C2D33DBB644120B1F053A431B0B97B2F2
:108020007743C01B00D201399FB27743C91B170C9D
:1080300077433E043F0C801BB941860D8F023E43BF
:10804000664329277F1BFE400C3D7746AF40BF1992
:1080500030BCA2B2ABB272437343801A9941220C76
:108060007243130C1204801A994102000B0001376D
:10807000001BA941F9D2781E0021F0BD0C277F1BFF
:10808000FE4077467F0BAF40FF19E0E700245D1C00
:1080900007D0144F7D663966FFE7FFE7FFE7FFE78C
:1080A0003C6F95B29EB265436643401BB141150CCF
:1080B0001E0C6543664336042F0C3E432D04401BC3
:1080C000B141994204D202000B0020000021F0BD12
:1080D00001D19042F7D3801A994101349942F2D3E9
:1080E000F6E70000000000D0FFFFFFFF48404140DE
:1080F000484018B41B4B5B68FC46019308BD04DF85
:108100005783001018B4174B1B68FC46019308BD39
:1081100000DF618300109446134A926F920809D2DF
:10812000624618B40F4BDB68FC46019308BD0CDFB8
:10813000198600100C4AF0B5146E556E576F166F05
:108140006246FFF7EEFF084A1466556657671667E2
:10815000F0BD18B4034B9B68FC46019308BD08DFD3
:10816000BD8400104C3D0020000000D0FFB5504001
:108170004240504059404B40594000E0FFB5154F38
:108180004C00640D03D0BC4204D10C0314D8002071
:10819000090D09055C00640D03D0BC4204D11C0329
:1081A0000AD800221B0D1B0501264B4009D44B4069
:1081B00003D58B4200D18242FFBD9942FCD190424F
:1081C000FFBD0B43DB1803431343F5D0C9434918E4
:1081D000FFBD0000FF07000000B5FFF7CFFF8041A3
:1081E00000BDC04600B5FFF7C9FF01D9002000BDA2
:1081F000012000BD00B5FFF7B9FF01D9002000BD87
:10820000012000BD00B5FFF7B1FF804100BD012096
:1082100040054A00121804D85A00121801D800204C
:10822000704701207047002070470000002100289F
:1082300005D17047C1174840401AFAD0C90713B595
:10824000064B1B6898470CBC441CA2401005120B3F
:108250000349091B09051943114310BD103C0020B7
:108260001F04000010B54C00620D8023D218DB0003
:10827000D21A5B057E2A10DD9E3A13DACC17090369
:10828000490819435242D140640001341532202A72
:1082900005DAD0400843604310BD002010BD0846F9
:1082A000604310BDC80FC018013810BD18B4044B8E
:1082B0005B6AFC46019308BD24DFC98700100000FB
:1082C0004C3D0020132370B51C78012C11D01ADD11
:1082D0000F48FFF77DFC0F4D01008022280000F0C1
:1082E00043FB022C10D00C48FFF76AFC0B4B1860C4
:1082F00070BD084D0A4A29002B00803104C38B420F
:10830000FCD1AA64EFE7034D054AAA64EBE7C04637
:10831000534400004C3D00204C330000103C002032
:108320002583001007B5604601880A0A0230DF2A5B
:10833000FAD1C9B2820804D30288408800041043ED
:1083400000E00068014A5050039007BD4C3D0020FA
:108350000FB403BC0CBCF0B50124E407634000E09B
:10836000F0B50C0DCF0F661E3605891B640503D3CF
:10837000C943404200D30131640D03D0661CF60AA4
:1083800007D0E41B00207F00791C89078912803CFC
:1083900024031D0DDF0F6E1E36059B1B6D0503D3D9
:1083A000DB43524200D301336D0D03D06E1CF60A3D
:1083B00007D0ED1B00227F007B1C9B079B12803D9A
:1083C0002D032F1B661B58D4A446202E46DA2037D7
:1083D0001400BC401D00BD40F24033412A438018C8
:1083E0005941CB0F05D0C943C043002264425041DC
:1083F000514162464D0D28D10D0D07D100281FD0E7
:10840000241940414941013A0D0DF9D0640006D3C9
:10841000013000D30131002C01D140084000013A65
:108420000BD4941CE40A04D112051144DB0719444F
:10843000F0BDD907204B194300E0D9070020F0BD5B
:108440000029DDD1002CDBD1F0BD0132C607400888
:10845000CD0728434908002EE1D0D9E73C2E29DA80
:10846000203E40371400BC4000D00124F2401443A9
:108470001A00BB401C43D317ACE7AC46202F08DAE8
:1084800020360400B4400D00B540F840394128437F
:10849000A5E73C2F0CDA203F40360400B44000D062
:1084A0000124F84004430800B1400C43C117EAE737
:1084B00010001900002494E70000F07FF0B50C0DC7
:1084C000661E3605891BE60A6405640D02D0651C2C
:1084D000ED0A04D0002001210905803C2403A446B4
:1084E0001C0D671E3F05DB1BE70A6405640D02D007
:1084F000651CED0A04D0002201231B05803C2403E7
:108500007740644497B484B296B27443070C7E43B8
:10851000150C6F4380B26843361802D30120000463
:108520003F183004350C00197D41844688B29AB258
:1085300050430C0C62431F0C7C438EB27E43921955
:1085400002D301263604A4191604170C3618674105
:1085500001BC81B29AB25143040C62431B0C5C43D0
:1085600080B25843121802D30120000424181004CA
:10857000130C401863412D185E410020474106BC92
:1085800088B293B258430C0C6343120C544389B223
:1085900051435B1802D301210904641819041A0C11
:1085A000091862416D1856410020474118BCF90274
:1085B000720D1143F0026A0D1043ED020A0D03D152
:1085C0006D1940414941013B124E9B1B7600B3425D
:1085D0000ED26D0007D30130002671416646354347
:1085E00001D1400840001B05C918E4072144F0BD33
:1085F0000BDA013306D1013004D101314F0D01D026
:108600004908F2E7E1070020F0BD013631050020FE
:10861000EBE70000FF030000F0B51C0D671E3F05EF
:10862000DB1BE70A6405640D02D0661CF60A04D061
:10863000002201231B05803C2403D0252D060026A3
:10864000F6432E661E096E66CE0FF619B446490033
:108650004F0D02D07E1CF60A03D000200021403FBF
:108660003F033E1BB600B444013F7F05C91B4908C8
:108670002E6F013676089C02950D25437543ED1348
:108680007543AD1301356D10F603761B0CB4CC02A7
:10869000450D2C43A2B2B3B25A43270C7B43350C91
:1086A0006F43A4B26C431B1902D3012424043F1965
:1086B0001C041D0CA4187D4124196D41009A91B22F
:1086C000ACB26143170C7C432B0C5F4392B25A430C
:1086D000A41802D301221204BF182204230C52183A
:1086E0007B41019C6C431B19520ED9010A43440182
:1086F000A01A81B2B2B2514303145A43360C7343E9
:1087000087B27743D617D21900277E4136049B19CA
:108710001704160C7F185E417316ED18F30100263E
:1087200080337541A90F06D16400690AE8055B0A28
:10873000184309D22FE00422944480337541A90ADA
:10874000A8059B0A184326D3404149412404009AB6
:10875000019B0D005543641B4343E41A95B286B256
:108760007543170C7E43030C5F4392B25A43B6180D
:1087700002D301221204BF183204330C52197B4178
:1087800052429C41002C02D4002201305141400849
:10879000CA071043490802B06246D7079210084B37
:1087A000D218084B9A4203D212058918C919F0BD94
:1087B0000020002A01DC3900F0BD01331905F5E77E
:1087C000FD030000FE070000002200B5203200F08B
:1087D00004F8080000BD000000220B150AD410B5F3
:1087E000944600F031F81414013400DA0021CB175C
:1087F000144C20470020002170476244343A0CD4C6
:108800000C2A07DA04009140904052422032D440B2
:10881000214310BDD843D94310BD203207D40C46A4
:108820009440524220321141D040204310BD0800F4
:10883000C917203203D452422032104110BD180013
:10884000190010BDFB8700100A0DCC0F531E1B052D
:10885000C91A520503D3C943404200D30131520D16
:1088600003D0531CDB0A07D0121B00206400611CDC
:1088700089078912803A1203014BD21A704700000F
:10888000FF03000051434343C9188C46110C83B2C7
:108890004B4310B4040C614392B280B25043624324
:1088A0001C041B0C001910BC59411304120CC018F5
:1088B0005141614470470000132310B51C781348E0
:1088C000FFF786F9012C0BD004DD0100802210484F
:1088D00000F04AF80F48FFF773F90F4B186010BD0E
:1088E0000B4C01005422200000F03EF80B4B636556
:1088F000A365E36523666366A366E3662367636730
:10890000A367E3672362E361E4E7C04653460000E0
:108910004C3E00204C330000103C00202189001008
:1089200007B5604601880A0A0230DF2AFAD1C9B2C7
:10893000820804D3028840880004104300E00068E5
:10894000014A5050039007BD4C3E002001480421CD
:10895000014B184750150020E17B0010014B1B68AC
:108960001847000050150020014B5B6818470000B5
:1089700050150020F0B5C64600B5437C06000C003B
:108980001500002B06D1036811002000984704BC95
:108990009046F0BD002AFADD0A78037C00200A2AFE
:1089A0002CD00121012D1BD0184B984602E0390034
:1089B000BD4215D04B1EE25C635C4F1C0A2BF6D106
:1089C0000D2AF4D03368884203DA091A2018984730
:1089D000336802214046984738003900BD42E9D14A
:1089E000854203DD291A3368201898476419013C31
:1089F00023780D3B5A4253413374C8E7002BD0D142
:108A000002480221336898470120CAE7F8F30010B2
:108A1000F0B54F46D6464646314BC0B51C680700F8
:108A2000002C1BD02F4B98462F4B9A4602E0E4684F
:108A3000002C13D02368002BF9D042461268002A7C
:108A400001D0A242F3D1627C3D1D3E68002A0CD1C8
:108A5000310028009847E468002CEBD100233B60EC
:108A60001CBC90469946A246F0BD002EDFDD397948
:108A7000227C00200A292BD00121012E03D119E0EC
:108A800049464E4516D04B1EEA5C4B1C99466B5C22
:108A90000A2BF5D10D2AF3D02368814203DD091A90
:108AA0002818984723680221504698474846494667
:108AB0004E45E8D1864203DD311A236828189847CD
:108AC000AD19013D2B780D3B5A4253412374AEE75B
:108AD000002AD1D10448083998470120CCE7C04684
:108AE000E0360020E4360020F8F300100B6870B583
:108AF00005000C00802B04D05A1C2260E41825715C
:108B000070BD0800FFF784FF2368F5E7F0B5CE4697
:108B1000474680B583B06B46DD1CD02328701B060A
:108B20001C681F4B804601A91800994605F0ACFE51
:108B3000071E2DD1019B64B29C4224D0484605F00B
:108B4000CBFE184B01271C68002C25D0164E07E0E1
:108B5000012229002000FFF70DFFE468002C0AD055
:108B60002368002BF9D03368002BF1D0A342EFD05B
:108B7000E468002CF4D1002F0ED1404603B00CBCA9
:108B800090469946F0BD074B1C68002CDED1F4E7F7
:108B9000044B1C68002CD9D1484605F055FEECE783
:108BA000E01D0020E0360020E4360020F0B5DE466F
:108BB00057464E464546E0B583B0070005F0BCFC7D
:108BC000D02301AD1B06060029002F481C6805F0C4
:108BD0005BFE8246002849D1019B64B29C423FD093
:108BE000294805F079FE294B9B461C6801239A46CB
:108BF000002C40D0264B98460A2399460EE03200BE
:108C000039002000FFF7B6FE4B4601222900200064
:108C10002B70FFF7AFFEE468002C0BD02368002B0D
:108C2000F9D043461B68002BE9D0A342E7D0E468A3
:108C3000002CF3D15346002B1DD15B461C68002C41
:108C400006D06368002B1AD09847E468002CF8D14E
:108C5000300003B03CBC90469946A246AB46F0BDFE
:108C60000A4B1C689B46002CC4D1F1E7074B1C68DB
:108C70009B46002CBED1044805F0E6FDDDE7E46824
:108C8000002CDED1E4E7C046E01D0020E0360020E5
:108C9000E43600200D4B1A68002A12D0824203D11C
:108CA00009E0984207D01A00D368002BF9D10029B7
:108CB00000D0D06070470029FCD1C368D360C16088
:108CC000F8E70029F6D01860F4E7C046E036002047
:108CD000F0B5C646D02300B51F4EA2B01B06070054
:108CE0008846300001A91C6805F0CEFD051E07D19D
:108CF000019B64B29C4203D0300005F0EDFD0135CC
:108D00008422002101A8FFF729FE43463A0001A969
:108D10001248FEF725FF019B0700002B18D1104BCE
:108D20001C68002C06D06368002B0DD09847E468BF
:108D3000002CF8D1002D02D0300005F085FD380060
:108D400022B004BC9046F0BDE468002CEBD1F1E702
:108D500001A8FFF75DFEE2E7E01D0020ED8A0010AC
:108D6000E03600200FB400B583B004A901C9019119
:108D7000FFF7AEFF03B008BC04B0184710B500F011
:108D80008FF910BDF0B5CE464746040080B583B0DC
:108D9000FBF730FB2600002736184F41B94230D888
:108DA0002DD0B9461D4B1E4D984643461C68002CDD
:108DB00003D116E0E468002C13D02B68002B01D0FF
:108DC000A342F7D1A368002BF4D0012101A8984752
:108DD0000028EFDD6B46187903B00CBC904699462D
:108DE000F0BD01200021FBF711FB0E4B5A6A9145A3
:108DF000DBD89B6AB3420BD301204042ECE7B04280
:108E0000CFD901235B42994601267642F717C9E77D
:108E10009145CAD001204042DEE7C046E03600203E
:108E2000E436002000400540002903D0437C002B9D
:108E300000D10374417470477047C0460022014B53
:108E40001A707047473D0020012070474B79002081
:108E5000FF2B00D070478B79002BFBD1CB79012BF6
:108E6000F8D1082AF6D98A78014B09301A70F1E74F
:108E7000473D002070B5002915D115495379107967
:108E800009781B0203430020994200D070BD53783B
:108E9000012B0AD0022BF9D1002064220021FCF71B
:108EA000DDFA0120F2E70120F0E7D478917824027E
:108EB0000C430500E20502D5620A93401D000548F7
:108EC000FEF77EFE7F210300214028009847C04620
:108ED000473D0020554200000123037000487047C1
:108EE000FCF300104A780B7812021A438B7810B505
:108EF0001B041A43CB781B0613439622D2009342DD
:108F000000D010BD0348FEF75BFE002103000800FF
:108F10009847C0465542000070B5184C82B0050015
:108F20000E00200001A905F0AFFC002808D1D023D5
:108F30001B061B68019A9A421CD0200005F0CCFC4D
:108F4000002001F049FE002807D103256D422000D2
:108F500005F07AFC280002B070BD002001F054FE3C
:108F60000028F2D029003200002001F05BFE051E2F
:108F7000EBD0ECE703256D42ECE7C046183C00203F
:108F800010B51F20FCF78AF8FA200021800010BDE0
:108F900010B5064C0021200005F076FC002804D016
:108FA00000F074FE200005F04FFC10BD183C0020BE
:108FB000F0B546464F46D646C0B5364F82B08046DD
:108FC0000E00380001A905F05FFC00280ED1D02367
:108FD0001B061B68019A9A4205D102B01CBC904640
:108FE0009946A246F0BD380005F076FC002001F05D
:108FF000F3FD002832D00024002E34DD264B9946A4
:109000009A4612E0002843D100F040FE002001F013
:1090100089FE002001F0E0FD002824D0002001F0AE
:10902000BDFE002823D0A6421DDD0020351B01F027
:10903000B5FE8542E6DC43462A001919002001F0FE
:1090400029FE050000F022FE002001F06BFEFBF778
:10905000D1F94B46641918605960E4E700200021FB
:109060000D4B18605960380005F0EEFBB5E7FBF7D3
:10907000C1F953460D001A685B6800218446074811
:1090800012184B419D42EED8CDD19445CBD9EAE799
:109090000500D0E7183C0020081F002020A1070091
:1090A00010B51D4B84B01B7802F08AF81B491F20B5
:1090B000FCF704F801211F20FBF7DEFF1848FBF73F
:1090C000BFFAFAF76DFE0400FBF794F9FA220023C9
:1090D000920012184B41994218D901225242D317DB
:1090E00001210291002101910E4920000091FAF71F
:1090F0005BFE0400631E9C41E4B2002803D0012102
:109100000948FFF7C7FD200004B010BD9942E7D120
:109110009042E2D8E4E7C04680F90010918F001039
:10912000183C0020818F0010601500200048704717
:10913000B4F400100048704760F4001070B50400EB
:1091400016480378002B20D0002C06D1C1241448E7
:10915000144BA4004380048070BD052C1CD8124B16
:109160000F48A400E558811C002304E001330A8065
:109170000231132B0DD0EA5CDCB2002AF6D1C023F9
:10918000013464009B001C43E5E7112102F0A0FAC2
:10919000DAE7CA24A400DEE70020DDE7303D002046
:1091A000B836002009040000C8F40010F0B5574696
:1091B000DE464E46454698238024E0B56B4A64025D
:1091C000D75883B0274228D001222321684B0020A2
:1091D0005A54DA70674901F0B3FA8022664B920262
:1091E0001A65664B9A46FB061CD480235B011F421E
:1091F0004AD18023DB011F4200D08DE080231B0277
:109200001F4200D096E0BC4200D0AAE003B03CBCB4
:1092100090469946A246AB46F0BD102300249A46DC
:10922000FB06E2D5514B9B6D9846002B27D0524B45
:1092300000249B460123994643460126B8461F0059
:1092400004E001347600E4B2202C17D03E42F8D07E
:109250005B469E654B466508A3436D00ED18444B85
:109260006D019C466544280000F08CFB00286CD101
:109270000134B743E4B27600002FE5D1474680239E
:109280005B0154461F42B4D01C430023374A0021DF
:109290001360384A3A489360D3603A4A9360D36087
:1092A000394A9360D360394A9360D360384A9360F7
:1092B000D360384A9360D360374A9360D360374AAB
:1092C0009360D360364A9360D360364A9360D3602C
:1092D000354A9360D360354A9360D360344A9360D3
:1092E000D360344A9360D360334A9360D360F022F2
:1092F0009200FFF733FB314B314A00211A60002006
:10930000012201F0F1F980221B4B12031A65802320
:10931000DB011F4200D171E70122042100201C4320
:1093200001F050F91022144B1A6580231B021F42D2
:1093300000D168E70122052100201C4301F042F919
:1093400080220D4B12011A655DE74B46AA8AA97867
:1093500000200093002301F01BFA280000F03AFAE5
:1093600086E7210017487940FBF7FEFC000011500A
:10937000EC360020000010500030115010000100A9
:109380002C3700200800105010001050180010500A
:10939000200010502800105030001050380010509D
:1093A000400010504800105050001050580010500D
:1093B000600010506800105070001050F43A002007
:1093C00080011050E0F4001010B501210520FBF7DA
:1093D00053FE10BD10B500220021024800F02CFA07
:1093E00010BDC0460C3700208022024B5202DA64C6
:1093F0007047C04600201150F0B5C64600B50700C2
:1094000000F0C2F90C23354D3549AB670520FBF759
:1094100055FE40239846334C402200212000FFF7A0
:109420009DFA43460126A383212100232E4A66701C
:10943000A260136063545F3161844146A1870239A1
:1094400063542A4A2A496360E260A1620B60E262C7
:10945000284A63629360D360274A20009360D360F8
:10946000264A00219360D360254A40309360D36040
:10947000244A9360D360244A9360D360234A936064
:10948000D360234A9360D360224A9360D360224A18
:109490009360D360214A9360D360214A9360D36084
:1094A000204A9360D360204A9360D3601F4A936040
:1094B000D360F0229200FFF751FA1D4B1D4A38008D
:1094C0001A6080239B052E64EB6490231A4AEA50AD
:1094D000FFF78AFF04BC9046F0BDC0460000115063
:1094E000AD910010EC3600208400105000011050A7
:1094F0008000105000001050080010501000105054
:10950000180010502000105028001050300010504B
:1095100038001050400010504800105050001050BB
:10952000580010506000105068001050700010502B
:10953000F43A00208001105010D001000B785B0637
:1095400002D14B78052B00D070478A78014B1A6006
:10955000FAE7C04600001150F0B5CE46474680B548
:109560008B7848799C4607230340C8780A7980079E
:10957000800F1B021343C2B291467F2162466646AA
:109580001140D4094F00294D3A195201AA1896707A
:109590000126B44666466640567000269383D67010
:1095A0009077CA00012C27D0214880468801424488
:1095B000281882601660002927D01E4AC9009446E8
:1095C000614441603F223F3393434A46022A00D11F
:1095D0005B0019493F190A687F01D3180B60174BCC
:1095E000ED19EA605A4080231B0613434A4696064B
:1095F0001E436B681E600EE011488046880142449D
:1096000028188262166000290AD1002364012D19EE
:109610006B600C4BEB6001200CBC90469946F0BD92
:10962000064AC900944661444162CBE7EC3600200B
:109630008400105004001050F43A00200000105034
:10964000800010500001105000231C4A10B5936098
:10965000D3601B4A00219360D3601A4A1A48936072
:10966000D3601A4A9360D360194A9360D360194A51
:109670009360D360184A9360D360184A9360D360B4
:10968000174A9360D360174A9360D360164A936079
:10969000D360164A9360D360154A9360D360154A2D
:1096A0009360D360144A9360D360F0229200FFF776
:1096B00055F9124B124A1A6010BDC04600001050F6
:1096C00008001050100010502C37002018001050C7
:1096D000200010502800105030001050380010505A
:1096E00040001050480010505000105058001050CA
:1096F000600010506800105070001050F43A0020C4
:10970000800110507F2020B5150008404000C90995
:1097100040180449400140181A00290000F08CF854
:10972000012020BDEC3600207F2310B50B40C90975
:10973000002B03D102220748521A82668022580069
:109740004018054B4001C0181201002100F048F8F4
:1097500010BDC04600201150EC3600207F2310B50C
:109760000B400BD0C90958004018054B4001181890
:1097700000230022C370034900F032F810BDC04638
:10978000EC360020FFF7FFFF80220D4B520410B58E
:109790001A600C4B0C491A6010008B689843FBD17F
:1097A0000A4C9C2200212000FFF7D8F880220021DB
:1097B00052010748FFF7D2F80923636710BDC0467E
:1097C00000E0004000F0004000C0004000001150E8
:1097D000000010500023037443828382836170472A
:1097E00010B58368002901D01C682140002A11D0DF
:1097F0008024E400114322420CD01A6822420BD18B
:109800000A4A0A401A60FFE7FFE7FFE7FFE7FFE7C2
:10981000FFE78368196010BD7F2281780448CB0977
:109820001140044A9B009A58FBF79EFAFFFBFFFF8A
:10983000F4F4001074150020F0B5C646002300B5FE
:10984000838201330374436804001E68838B816143
:109850001F1C934200D9171C8025BFB2D21BE3788E
:1098600092B2ED0062823D43002B02D09025AD0103
:109870003D4301204340E3706378002B50D0002A21
:109880001DD1A023DB011D43384B1B6C384B3340EB
:109890008026B6051E436368A2681E6013685B05D8
:1098A00059D4344B2B401360FFE7FFE7FFE7FFE796
:1098B000FFE7FFE7A3681D6004BC9046F0BD80236E
:1098C0005B011D43294B1B6C9B0702D4A378DB096A
:1098D000DCD0A38B191C934200D9111C80278BB2BA
:1098E000FF00D21A98461F43E37892B26282002B9F
:1098F00003D090274146BF010F4301214B40E37045
:109900006378002B19D0002A02D18023DB011F438A
:10991000194B3F043340A026F6053D431E43BAE7EA
:109920003A00E068FFF720F8A369628A9C4680232A
:1099300067441B02A7611D43A1E7E068424640302F
:10994000A169FFF711F8A369628A4344A3618023E8
:109950001B021F43D7E77F22A1780848CB0911409B
:10996000074A9B009A58FBF7FFF9C04600001150C8
:10997000FFFFFFAFFFFBFFFFFFFFFFDFF4F400106F
:1099800074150020F0B5C64600B5067C0400002E14
:1099900000D1D8E083681A681D684378AD05AD0D25
:1099A000002B50D1838AEB189BB28382A18B626813
:1099B0008D4206D2002363821368300004BC9046B7
:1099C000F0BD1268520001D58D4269D0638A002B28
:1099D000F3D062681F1C16688B425FD88025BFB227
:1099E000DB1BE2789BB2ED0063823D43002A37D156
:1099F00001214A40E2706278002A3AD0002B47D019
:109A0000802252011543584A126C920757D4A2780B
:109A1000D20954D1554B33408026B6051E436368A6
:109A2000A2681E6013685B0500D593E0504B2B4085
:109A30001360FFE7FFE7FFE7FFE7FFE7FFE7A36844
:109A400000261D60B9E72A00C1688069FEF78CFF17
:109A5000A38AA269EB189BB25219A382A261A5E75F
:109A6000012190254A40E2706278AD013D43002A11
:109A7000C4D13A00A169E068FEF776FFA3699C466D
:109A800080231B021D43638A6744A761002BB7D163
:109A9000A023DB011D43344B1B6CBBE70F1C9DE770
:109AA000A26815686278AD01AD0D002A3DD1EB18B2
:109AB000A3828D4200D389E7002363827DE7A28BD6
:109AC000111C9A4221D880278AB2FF009B1A904627
:109AD0001743E2789BB26382002A03D09027414665
:109AE000BF010F4301214A40E2706278002A0ED084
:109AF000002B02D18023DB011F431E4B3F04334068
:109B0000A026F6053D431E4389E7191CDBE7E06804
:109B100042464030A169FEF727FFA3694344A36191
:109B200080231B021F43638AE2E7E1682A00403179
:109B3000A069FEF719FFA38AA18BEB18A382A36982
:109B40005B19A361B5E77F2381780B4A19400B4865
:109B5000FBF70AF97F22A1780948CB091140064A90
:109B60009B009A58FBF700F900001150FFFFFFAF70
:109B7000FFFBFFFFFFFFFFDF7415002014F500104F
:109B8000F4F40010024B5878431E9841C0B270475D
:109B9000E0340020024B18784007C00F7047C046E1
:109BA000E0340020014B18787047C046433D002048
:109BB000F8B54746CE462B4D80B52B780700002BD5
:109BC00004D001200CBC90469946F8BD53220021D8
:109BD0002548FEF7C3FE254C2000FAF731FD244B43
:109BE0001C60244C20001C30FAF746FD200001F0D8
:109BF00023FD214B1C60214B002B2AD0204E00243A
:109C00003000FFF769F91F4B1F4A984618609146CC
:109C100033780BE0424663001B191268DB009B5847
:109C2000984701343378E4B2A34209D39C42F1D37C
:109C300015D14B46984701343378E4B2A342F5D2AC
:109C40003800FFF7D9FB3800FFF7BEFB01232B706C
:109C5000B7E701F0B1F80A4B1B78002BF0D00023D6
:109C60001B68FFDE433D0020E034002098340020D4
:109C7000343500207C15002038350020D98E0010A6
:109C8000423D0020A8310020B9AD0010F0B5DE46FD
:109C900057464E464546E0B58BB001F097FA00288E
:109CA00000D18FE1CF4BD04E9B4607AC3568EA69B7
:109CB000EFF3108172B61368002BFCD0BFF35F8FF7
:109CC00029622800210001F03DFBEA692B6ABFF3FD
:109CD0005F8F0021116083F31088002800D171E1AB
:109CE0006378082BE2D85A469B00D3589F46636896
:109CF000002BDBD0A0689847D8E77F222179BB4BA7
:109D00000A405500C8095B191B181800012730309C
:109D1000C578BD43C570C5780337BD43C570002AFB
:109D200000D199E1B24ADB7C002A00D190E1B14A2E
:109D30001278934200D389E15A00D318AE4ADB006F
:109D40001268D318002B00D13CE11D69627920789C
:109D5000A368A847AAE70122A44F01213B78042069
:109D600013433B703323FA5C8A43FA54FA5C824310
:109D7000FA540133FA5C8A43FA54FA5C8243FA5487
:109D800023780020019300F095FE60232279134090
:109D9000602B00D151E1402B00D141E1D206D20E1F
:109DA000012A00D16AE1002A00D15BE1022A00D039
:109DB00043E17F22217A0A400F2A00D93DE1C809F8
:109DC00084465200B8188A4D6044C07C002D00D1F2
:109DD0008FE1884D2D78A84200D388E145002818EE
:109DE000854DC0002D682D18002B00D187E1002D76
:109DF00000D122E1E86800F05DFEEB6808AA0021CE
:109E00000198984716E1794B1B78DB0700D44DE7A2
:109E10007A4B002B00D149E700E000BF46E7734BC7
:109E20001A78D20700D441E7754A002A00D13DE7ED
:109E300018780007C00F00E000BF37E76D4D6C4A8F
:109E40002B78002A00D1B7E000276B491A0088461A
:109E50009F4214D2414609687B008C46DB19DB0027
:109E600063445B69002B0DD02078984701372A782E
:109E7000FFB2974200D919E713009F42EAD39F42ED
:109E800000D09CE00137FFB2974200D90EE71300E3
:109E9000F3E72378574D564A984600272B78002A37
:109EA00000D1B3E0574A9246534A91462A004546AC
:109EB00090460FE04A4612687B009446DB19DB00AF
:109EC00063445B6828009847434601371B78FFB21C
:109ED000BB420BD39F42EDD36BD15346280098472A
:109EE000434601371B78FFB2BB42F3D23F4D5322AA
:109EF00000212800FEF732FD1022FF21E81CFEF7AA
:109F00002DFD28002022FF211330FEF727FD00F051
:109F1000C7FD3D4B002B00D1C8E600E000BFC5E601
:109F20002378344D324A984600272B78002A50D0A7
:109F3000344A9246304A91462A00454690460FE000
:109F40004A4612687B009446DB19DB0063445B6879
:109F500028009847434601371B78FFB2BB420BD31A
:109F60009F42EDD325D153462800984743460137F9
:109F70001B78FFB2BB42F3D21C4D532200212800B4
:109F8000FEF7ECFC1022FF21E81CFEF7E7FC28009E
:109F90002022FF211330FEF7E1FC00F081FD237940
:109FA000AB7083E6019800F045FF2B78002B00D1C1
:109FB00092E200235B68FFDE002B00D176E60023EF
:109FC0005B69FFDE0BB03CBC90469946A246AB46AF
:109FD000F0BD404600F02EFF2B78002BCCD00023A4
:109FE0005B68FFDE48F5001038350020E0340020C3
:109FF000D98E0010423D0020A83100200000000052
:10A000000000000035AE001000000000404600F0E7
:10A0100011FF2B78002B00D168E700235B68FFDE7F
:10A02000C948002809D000F045FD08AA0021019880
:10A0300000E000BF002800D038E620780021FFF7BC
:10A0400073FB20788021FFF76FFB2FE69B1ADBB2B2
:10A05000002BB7D1BD4D79E662792078A36800F076
:10A060003DFD23E6202B00D128E1002BE5D16379CB
:10A07000092BE2D8B64A9B00D3589F46237A0F2B70
:10A08000DBD8B44AFB18DB78002A2BD0B24A12780E
:10A09000934225D2B14A5D00EB181568DB00ED183C
:10A0A000002DCAD0E86800F005FDEB6808AA002181
:10A0B00001989847002800D0F8E5602523791D40D5
:10A0C000BBD163790A3B012BB7D800F0F3FC63796D
:10A0D0000A2B00D150E108A9019800F06FFCE5E5DA
:10A0E0009B1ADBB2002BA8D19D489E4DDBE7401B9D
:10A0F000C0B2002800D1F8E00025002B9DD1637983
:10A100009946012B04D0002B00D1FAE0032B94D107
:10A11000E388002B1BD14B46BA18012B00D1FAE083
:10A12000130030229046634498444346DB789B07F3
:10A130000DD40198FFF7F8FA43460222DB78134367
:10A140004246D370D378012213434246D370002D88
:10A1500000D1ABE5E86800F0ADFCEB6808AA00218F
:10A1600001989847002000F0A5FC3423FB5CDB0736
:10A1700000D59BE5AFE7A37903931A007B789A4259
:10A1800007D07B78002B00D07EE1039B002B00D012
:10A19000FBE0039B08A901987B7000F00FFC85E5AC
:10A1A0007B7806AA0232137008A90123019800F0F7
:10A1B0001DFC7BE5E088030AC0B20F2B00D93CE709
:10A1C00069499A008A58974608A800F079FCA17955
:10A1D0000198FFF7FFF802223B7813433B7065E5D7
:10A1E000E388012B00D028E708223B7808A9934395
:10A1F00001983B7000F0E2FB58E50220397806AB8D
:10A200009A1C8B068908DB0F01400B43138008A9B9
:10A210000223019800F0EAFB48E5E388012B00D017
:10A220000BE708223B7808A9134301983B7000F024
:10A23000C5FB3BE54D4B002B00D1FEE600E000BF27
:10A24000C37881781B0202000B43019808A900F033
:10A25000CDFBEFE6464B002B00D1EEE600E000BF61
:10A26000021E00D1E9E6137808A9019800F0BEFBB0
:10A27000E0E62189FEF762FF021EF4D1DDE6022B43
:10A2800000D176E13B4B002B00D1D6E600E000BFC9
:10A29000002800D1D1E6C37882781B02134308A9B5
:10A2A0000200019800F0A2FBC4E6FEF73FFF122374
:10A2B000020008A9019800F099FBBBE6237A0F2B56
:10A2C00000D9BAE6234AFB18DB78002A13D0224AC9
:10A2D000127893420DD2214A5D00EB181568DB001D
:10A2E000ED18002D00D1A8E684E5002B06D11D4D08
:10A2F00005E79B1ADBB2002B00D09EE61848194DEB
:10A3000079E5BA18130063443033DB7806AA9B075B
:10A31000DB0F02327AE72F3398466244904443467B
:10A32000DB789B0700D412E70198FFF717FA434642
:10A330000222DB7893434246D370D3784A46934354
:10A340004246D37003E7C0460000000029B0001069
:10A350006CF50010D98E0010423D0020A83100207D
:10A3600045AF0010D4F5001094F500100000000077
:10A37000000000000000000006AB9A1C08A90123A1
:10A380000198157000F032FB90E4581EC0B2FEF741
:10A39000D1FE002800D150E64378022B00D04CE6D5
:10A3A0000125C3795A112A40120191463A789B112E
:10A3B00090461022414691430A0049460A43202113
:10A3C0002B408A435B0113433B7009239946C378B2
:10A3D00082781B021343C31881440493994500D328
:10A3E000C0E04D4601226B7802920B2B04D1EB7832
:10A3F00002932B78ED186B78042B00D01DE6002219
:10A40000049B90465B1B9BB29A46674A674B1B783E
:10A41000002A25D02A00454690469D421AD2644A19
:10A420006B0012685B199146DB0099444B469B68B0
:10A4300005925246414601989847082803D9534649
:10A44000834200D3A7E0594B01351B78EDB2AB42F4
:10A45000E3D2F2E59D4214D1564A574B9146E8E7C4
:10A4600052462900019800F0FBFCD046824608289D
:10A4700002D94346834242D24C4B1B78002B00D179
:10A48000DBE500239B68FFDE0198FFF7DDF8BB7872
:10A49000464D454A9A4600212B78002A00D181E595
:10A4A000434A90462A000D0091460FE0424612684A
:10A4B0006B0094465B19DB0063445B680198984726
:10A4C0004B4601351B78EDB2AB4205D39D42EDD32F
:10A4D00000D06EE5394BF1E7532200213800FEF73A
:10A4E0003DFA1022FF21F81CFEF738FA380020222E
:10A4F0001330FF21FEF732FA5346BB7045E62D4B71
:10A500009946294B9846029B012B35D0029B002B84
:10A5100017D0A9787A18D2780B00FF2A00D08CE5E2
:10A52000002206E08B18DBB2F818C078FF2800D0B4
:10A5300083E54046FB18D8700132029BD2B29A42A2
:10A54000F0D33800434629001330524600F07EFE17
:10A55000164B55441B78434500D26EE5049BAB4235
:10A5600000D93FE7164B002B00D112E600E000BFF8
:10A570000FE6FEF7DFFD8BE648468068A978844643
:10A580000D487B18DA7884450AD0FF2A00D054E5BC
:10A590004246DA70D5E743468246A8461D00B2E738
:10A5A00002230293B6E7C046D98E0010423D002038
:10A5B000A8310020D4F5001061AE001035AE0010B7
:10A5C0000000000070B586B06B4605000C00981CBA
:10A5D0000A220021FEF7C2F96B461D705C70032C45
:10A5E0004FD01BD9042C07D0052C40D13C4B1A78F6
:10A5F000D20766D406B070BD394B1A78D207F9D5A8
:10A6000004211A780A431A70364B1C68E269EFF38A
:10A61000108172B61368002B19D1FBE7022C26D1EA
:10A6200001212F4B1A788A431A701A780331A243FA
:10A630001A7000225A701A788A431A70294B1C68C3
:10A64000E269EFF3108172B61368002BFCD0BFF300
:10A650005F8F21626946200000F03AFFE269236AB9
:10A66000BFF35F8F0021116083F31088C2E71D4B99
:10A670001C68E269EFF3108172B61368002BE6D113
:10A68000FBE7174B1A785207B4D504210E201A782D
:10A6900068448A431A7000210A22FEF75FF90523F5
:10A6A00003AE73700F4B35701C68E269EFF31081D5
:10A6B00072B61368002BFCD0BFF35F8F21623100AC
:10A6C000C9E704211A788A431A70064B1C68E269AC
:10A6D000EFF3108172B61368002BB8D1FBE7C046C8
:10A6E000E03400203835002070B584B06B46060099
:10A6F0000D000A220021981DFEF730F9012301AC5C
:10A7000063700E4B25711D682670EA69EFF31083A4
:10A7100072B611680029FCD0BFF35F8F2B62210055
:10A72000280000F0D5FEEA692B6ABFF35F8F002195
:10A73000116083F3108804B070BDC0463835002026
:10A74000002330B585B001AD6B8028700633082238
:10A7500002A86B70FEF708F90C4B1C68E269EFF376
:10A76000108372B611680029FCD0BFF35F8F23629B
:10A770002900200000F0ACFEE269236ABFF35F8F7E
:10A780000021116083F3108805B030BD38350020FA
:10A79000F0B5C64600B584B01D006B4680460F007C
:10A7A000160000210622981DFEF7D8F8434601AC9A
:10A7B0002370072363700F4B65711D682771A660B6
:10A7C000EA69EFF3108372B611680029FCD0BFF379
:10A7D0005F8F2B622100280000F07AFEEA692B6A65
:10A7E000BFF35F8F0021116083F3108804B004BCB5
:10A7F0009046F0BD38350020F0B5DE464F4646465F
:10A800008346C0B50C00002A43D04978052916D1EB
:10A81000E678B607B60FB34211D17F23A1780B407B
:10A820000F2B0CD8531E98461B4B002599467F27AB
:10A830004B462000997800F0CDFC002805D100207F
:10A840001CBC90469946A346F0BD21005846FEF731
:10A8500083FE0028F3D0A378DA09012A13D0089ADE
:10A8600013702378E418454513D06378052BE6D19F
:10A87000E3789B079B0FB342E1D1A37801353B40BE
:10A880000F2BD5D9DBE7099A13702378E4184545D7
:10A89000EBD10120D4E7C046E03400207F2370B51F
:10A8A0008A7805000C0013400F2B01D9002070BDE1
:10A8B000054B2000997800F08DFC0028F6D021008F
:10A8C0002800FEF749FEF2E7E03400207F2370B550
:10A8D0000B40134C5B00C909E41864183034E57868
:10A8E000ED07ED0F04D1E3785B0703D5280070BDB9
:10A8F0000025FBE701210B4E4942306803F0D4FFED
:10A90000E378DB0707D4E3785B0704D4042201254E
:10A91000E3781343E370306803F096FFE6E7C04640
:10A92000E03400203435002070B50D0001210F4CBB
:10A930004942206803F0B8FF7F2129404B000C49B1
:10A94000ED09C91849193031CB780025DB0707D448
:10A95000CB785B0704D50422CB7801359343CB70C9
:10A96000206803F071FF280070BDC0463435002018
:10A97000E034002070B57F240C4065000E4C0600CA
:10A980006419C80924183034E5780020ED0700D593
:10A9900070BD0125E0782843E0703000FEF7B2FE7C
:10A9A0000028F5D10122E3789343E370E378033282
:10A9B0009343E370ECE7C046E034002070B50A4CE6
:10A9C0000600082220000D00FDF7CEFF0023002125
:10A9D000A360E36069563000C943C90FC901002272
:10A9E000FFF7C8FF70BDC04684340020F0B5C646EE
:10A9F0009046294C082200B5060020000D001F00DB
:10AA0000FDF7B2FF4346A3600023E381EB79AA7907
:10AA10001B0213431A1CBB4200D93A1C97B2A281F5
:10AA2000002B12D0002F1DD04346002B2ED03B1CF4
:10AA3000402F1DD89FB223787F2B1ED80021174AA4
:10AA40003B003000FFF796FF09E000216956002324
:10AA5000C943C90FC90100223000FFF78BFF04BCB6
:10AA60009046F0BD23787F2B12D800210022E7E723
:10AA700040239FB223787F2BE0D9084C3A0041460F
:10AA80002000FDF771FF80212200D9E70020E6E7D2
:10AA900080210022D4E7C04684340020A034002066
:10AAA00010B5142200210248FDF758FF10BDC04622
:10AAB00084340020014B18617047C0468434002064
:10AAC00010B5054C010008222000FDF74DFF0023C2
:10AAD000A360E36010BDC04684340020F8B53B4C51
:10AAE0001D0023780600DA09C9098A4212D0002025
:10AAF000002D0ED1364B002B03D021003000FEF785
:10AB00001DFD2369002B5AD02200022130009847F6
:10AB10000120F8BDA7687F2B08D80020002FF8D0AF
:10AB200038002A002B49FDF71FFFA768E289E38858
:10AB3000521992B27F19E281A760934201D03F2D52
:10AB400013D82369002B05D022000121300098473B
:10AB500000281DD0002161560023C943C90FC90137
:10AB600000223000FFF706FFD3E7A089811A0D1CF1
:10AB700089B2402916D82378ADB27F2B14D8002192
:10AB800082421ED0134A2B003000FFF7F3FEC0E7CD
:10AB900000213000FEF7C8FD30008021FEF7C4FD23
:10ABA0000120B6E74025E6E782420CD0094C2A0096
:10ABB00039002000FDF7D8FE80212200E3E70120C4
:10ABC000A7E70022DFE780210022DCE784340020B1
:10ABD0003D950010A034002010B50400FEF7D2FF10
:10ABE000002801D1002010BDFEF7D4FF0028F9D1C4
:10ABF000B62080004443034800190379012018401F
:10AC0000F1E7C046AC3100200300B6208000584375
:10AC100010B5034B1030C01800F06AFB10BDC046E1
:10AC2000AC310020F0B5B625AD0045432C00C6463A
:10AC3000174E1034A41900B592B2200000F0D0FBDA
:10AC40000700200000F06EFB3F2803D8380004BC4A
:10AC50009046F0BD7319D97800209846FFF736FE6C
:10AC60000028F3D0200000F05DFB3F2805D84346C4
:10AC70000020D978FFF758FEE8E796239B00EA18F2
:10AC800043469219D97800204023FFF773FEDDE791
:10AC9000AC310020F0B5B625AD0045432C00C646CA
:10ACA0001F4E2C34A41900B592B2200000F050FCC5
:10ACB0000700200000F01CFB3F2803D8380004BC2C
:10ACC0009046F0BDFEF75EFF0028F7D0FEF762FF6A
:10ACD0000028F3D1200000F00BFB0028EED0731900
:10ACE000997800209846FFF7F1FD0028E6D0A623CA
:10ACF0009B009C466544AE1931004022200000F0C4
:10AD00006FFB43469978002805D0030032000020ED
:10AD1000FFF730FED2E70020FFF706FECEE7C04681
:10AD2000AC310020F8B50500FEF72CFF002801D15A
:10AD30000020F8BDFEF72EFF0028F9D1B624A400AC
:10AD400065432E00144F2C36F619300000F0D0FA6F
:10AD50000028EDD07C19A1780020FFF7B7FD00286E
:10AD6000E6D0A6239B009C466544ED1929003000DF
:10AD7000402200F035FBA178061E08D003002A000F
:10AD80000020FFF7F7FD0028D2D03000D1E70020E7
:10AD9000FFF7CAFDCCE7C046AC3100200300B62067
:10ADA0008000584310B5034B2C30C01800F0BAFA9D
:10ADB00010BDC046AC310020B622F0B51B4C83B0AC
:10ADC000920000212000FDF7C9FDFF236371184B9D
:10ADD00080260025E380012708232100200076003B
:10ADE00023732781320048310095073B103000F073
:10ADF00043FA2100200049313200FF31009701233E
:10AE00002C3000F039FA92239B00E6183000F9F755
:10AE100017FC94239B00A662E61865623000F9F7E0
:10AE20000FFC2664656403B0F0BDC046AC31002061
:10AE300000C2FFFF10B5094C052200212000FDF7DC
:10AE40008DFD20002C34103000F0F6FB200000F0C7
:10AE5000F3FB0121200000F015FC10BDAC310020F7
:10AE6000F0B54B7983B00600022B03D000252800F3
:10AE700003B0F0BD8B79022BF8D12F4FBB78002B9C
:10AE8000F4D18B7809253B700C780C196378242B4E
:10AE90000BD1082A02D81FE0AA421DD32378E41858
:10AEA000ED186378ADB2242BF6D0052B2CD0042BF3
:10AEB00012D163790A2B0FD1204B277801930133EC
:10AEC0000093E119022302223000FFF795FC0028CD
:10AED000CCD00E35ED19ADB2194C200000F022FA9D
:10AEE0003F28C4D92600103EF1780020FFF7EEFC81
:10AEF0000028BCD0200000F015FA3F2812D8F178C5
:10AF00000020FFF711FDB2E721003000FFF7C6FC7B
:10AF10000028ABD0A3787B702378ED18E418ADB28D
:10AF20006378C4E792239B00E218F1784023002065
:10AF3000FFF720FD9BE7C046AC310020AE3100207A
:10AF4000BC310020F8B560231400127813400022B1
:10AF5000202B01D01000F8BD2E4D637927792E7873
:10AF60001B023B439E42F5D16378212B43D009D984
:10AF7000222B24D0232B14D1002945D0022912D012
:10AF80000122E7E7202B0CD1002936D00229F7D186
:10AF9000214B002BF4D0A91D0020FDF7A3FF0122B7
:10AFA000D8E70022D6E71D4B002BE9D0E178A37843
:10AFB00009021943002000E000BF0122CAE700296E
:10AFC00022D00229DCD10126A178E47828002402CD
:10AFD0000C4331002C71A1432C3000F053FB104B7B
:10AFE000002BCDD03100620832402140002000E02B
:10AFF00000BF0122AEE70029C2D10A4A072321007F
:10B00000FFF7F4FC0122A5E72100FFF7D7FC01229E
:10B01000A0E7C046AC310020E58E00100000000023
:10B0200000000000B2310020F8B54746CE4680B59A
:10B030005D4C1E00E37880460D008B4263D1962361
:10B0400027009B001037E118B2B2380000F080FAF8
:10B05000564B002B1CD06379FF2B19D0002E17D034
:10B060000022914605E001239C46E1444E450FD065
:10B070006379962292004A44A25C9A42F3D1380046
:10B0800000F048F90028EED1617900E000BFEAE75E
:10B09000474B484C002B04D0200000F03BF900281F
:10B0A0005BD0200000F03EF93F2859D8103CA3782F
:10B0B000AB4205D0012420000CBC90469946F8BD57
:10B0C0003D4B002B02D0002000E000BFFEF75AFDF0
:10B0D00000281DD1394C200000F00AF90028E9D1E0
:10B0E000002EE7D0B306E5D12C3CA1784046FFF70F
:10B0F000EDFB2500041EDDD0A97800230022404688
:10B10000FFF738FCD7E7A3788B42D9D00024D2E7E9
:10B11000FEF740FD294C0028DDD1200000F0E8F8C2
:10B120000028D8D025002C3DA9780020FFF7CEFBC1
:10B130000028D0D09B239B00E71839004022200034
:10B1400000F04EF9A978002829D003003A00002029
:10B15000FFF710FC0028ADD1BDE700E000BFA0E77D
:10B160002700103FF9780020FFF7B0FB002801D13D
:10B17000BB789DE7200000F0D5F83F2805D8F97886
:10B180000020FFF7D1FBBB7892E792239B00E218E7
:10B19000F97840230020FFF7EDFBBB7888E700201B
:10B1A000FFF7C2FB97E7C046AC310020000000006B
:10B1B00000000000BC31002000000000D831002059
:10B1C00010B50020FEF7F4FC10BDC04610B5FEF728
:10B1D000E9FC10BD072310B54479027923401B0216
:10B1E0001A43C3789B079B0F022B1BD00DD800205E
:10B1F000012B09D102394B425941124B00209C4688
:10B20000614491424041C0B210BD02394B425941A4
:10B21000F023002049429B001940403191424041B7
:10B22000C0B2F1E7022905D00020402393424041FB
:10B23000C0B2E9E7044B9C46624450425041C0B260
:10B24000E2E7C046FF03000000FEFFFFF0B5002468
:10B250007F27002A0FD04D78052D06D13D008E782E
:10B2600035406D00F6094519AB550D786419A4B247
:10B270004919A242EFD8F0BDF8B54746CE4680B591
:10B28000984608AB1F7880230400894615001B02EE
:10B2900000269A4227D84069002803D0012149425C
:10B2A00003F002FBA069002803D00121494203F00A
:10B2B000FBFA4B4623604346A5806D00ADB2E380A8
:10B2C0006B1EA381002360696D42E3812772658153
:10B2D0002382002801D003F0B7FAA06901260028D4
:10B2E00001D003F0B1FA30000CBC90469946F8BD8D
:10B2F000C189028A89B292B28B1A9BB2914202D260
:10B3000042899B1A9BB28288101C9A4200D9181C51
:10B3100080B27047C389008A181A43425841C0B2AC
:10B320007047C04610B5C489018AA4B289B2631AB5
:10B3300082889BB28C4202D240891B1A9BB2D01ADF
:10B3400080B210BD70B5040080690D00002803D0E4
:10B350000121494203F0A8FAE089218A80B289B22A
:10B36000421A92B2884202D26389D21A92B2A38858
:10B37000934208D2C21A92B298422DD26089121A10
:10B3800092B222821A00002A02D11EE0C91A89B2A2
:10B390008B42FBD92368E2889C46514328006144D4
:10B3A000FDF7E2FA228A012592B2531C9BB29A421F
:10B3B0000ED9002362899B189BB2A06923820028C2
:10B3C00001D003F041FA280070BD0025238A9BB20A
:10B3D000A2899A42F1D2EDE7A0899042D1D2CDE77D
:10B3E000F8B54746CE460400806980B50E001700C8
:10B3F000002803D00121494203F056FAE289218A4C
:10B4000092B289B2551AADB28A4202D26389ED1A5C
:10B41000ADB2A388AB420AD2D11A89B29A424CD2B9
:10B420006289891A89B21D002182218A89B2002D80
:10B4300047D03A1CAF423BD895B28B4203D8C91AC9
:10B4400089B28B42FBD95B1A9FB2E3885943984675
:10B4500023689C466144BD4224D94046784383B268
:10B460001A0030009946FDF77FFA43463000EA1B88
:10B470005A43484492B22168FDF776FA228A92B282
:10B4800053199BB29A421ED962899B189BB2A0693C
:10B490002382002801D003F0D7F928000CBC904685
:10B4A0009946F8BD424630006A43FDF75DFAE5E78C
:10B4B0002A1C95B28B42C2D9C5E7A2898A42B2D270
:10B4C000AEE7238A9BB2A2899A42E0D2DCE7C0466B
:10B4D000F8B5040040690E00002803D0012149425C
:10B4E00003F0E2F9E589238AADB29BB2EA1A92B27F
:10B4F000AB4202D96389D21A92B2A388934222D076
:10B5000028009D4203D3C01A80B28342FBD923682E
:10B51000E2889C46504331006044FDF725FA6B1CDD
:10B520009BB29D420BD962899B189BB26069E381F3
:10B530000127002801D003F087F93800F8BDA2895F
:10B540009A42F3D2EFE7277A002FD9D1F5E7C04628
:10B55000F0B54F46D64646460500C0B514000F006C
:10B56000002A05D120001CBC90469946A246F0BD99
:10B570004069002803D00121494203F095F9EA8887
:10B58000EE899046298A2A7AB6B289B2AB88002A17
:10B590000ED1721A92B28E4202D26989521A92B2B6
:10B5A0009A1A111C92B2A24200D9211C8CB207E057
:10B5B0009C4205D34246E41A54430E003F191C0036
:10B5C00030009E4203D3C01A80B29842FBD21B1AAD
:10B5D0009BB29946434658432B689C4660444C4571
:10B5E00015D8424639006243FDF7BEF9A3199BB254
:10B5F0009E4202D8AA899A4202D26A899B189BB2BB
:10B600006869EB810028ADD003F01EF9AAE74B462C
:10B61000414659438BB21A0039009A46FDF7A4F906
:10B620004B46E21A434639005A43514492B22868C5
:10B63000FDF79AF9DAE7C04610B504004069002822
:10B6400003D00121494203F02FF9A069002803D05B
:10B650000121494203F028F90023E3812382A388D2
:10B6600060695B009BB25A1E5B42A2816381002825
:10B6700001D003F0E9F8A069002801D003F0E4F854
:10B68000012010BD70B5040040690D00002803D0F2
:10B690000121494203F008F9A069002803D00121E3
:10B6A000494203F001F960692572002801D003F0D6
:10B6B000CBF8A069002801D003F0C6F8012070BDC6
:10B6C00010B5024800F0EAF810BDC046083B002063
:10B6D000013930B5002900D1B4E06F4B1A7812114E
:10B6E000D5B22C003034092A00DDAEE00470012907
:10B6F00000D1A6E00F221C78224014003034092A21
:10B7000000D9A4E04470022900D19AE05A781211BD
:10B71000D5B22C003034092A00DD9BE08470032967
:10B7200000D18EE00F225C78224014003034092AC8
:10B7300000D991E0C470042900D182E09A781211F6
:10B74000D5B22C003034092A00DD88E004710529C7
:10B7500077D00F229C78224014003034092A00D977
:10B760007FE0447106296CD0DA781211D4B225003A
:10B770003035092A00DD77E08571072961D00F2275
:10B78000DC78224014003034092A00D96FE0C471FB
:10B79000082956D01A791211D5B22C003034092A52
:10B7A00000DD0734047209294BD00F221C79224096
:10B7B00014003034092A01D93732140044720A299E
:10B7C0003FD05A791211D4B225003035092A01DD53
:10B7D0003734250085720B2933D00F225C79224043
:10B7E00014003034092A49D8C4720C2929D09A7916
:10B7F0001211D5B22C003034092A42DC04730D2911
:10B800001FD00F229C79224014003034092A3AD8E4
:10B8100044730E2915D0DA791211D5B22C003034C8
:10B82000092A33DC84730F290BD0DA790F231340F4
:10B830001A003732092B2BD9C273102901D01030CE
:10B8400000E040180023037030BD07344EE7373264
:10B85000140057E7073461E7373214006AE707340A
:10B8600074E7373214007CE73734250084E7373239
:10B870001400C471082900D08CE7E2E737321400C5
:10B88000B2E70734BAE737321400C1E70734C9E733
:10B8900030331A00D0E7C046083B002010B588B00E
:10B8A00004000D2200216846FDF758F80D22002102
:10B8B00004A8FDF753F84B236A4604A913706846A1
:10B8C0000D2202F0B9FF1521082269442000FDF77E
:10B8D0004BF808B010BDC046F0B546468046354B23
:10B8E000D64643445A1E93418022520294464F4604
:10B8F0005B421340304A6344C0B513602F4A0D00C9
:10B900002F49136018008A689043FBD10620F9F78D
:10B91000ADFB80268146E90D6802AB0DAA02022428
:10B92000760006E0914507D312184B413C00B74220
:10B9300002D0A71C002BF5D080272602361B7F00E3
:10B9400003E05746361B012F31D07B1E310048469D
:10B950009A46FCF78BF98542F3D23900534661438E
:10B960001B0242461461126840465340FF221202F5
:10B97000134080225201024313600368072058409D
:10B98000CF23034013604246802303209B012432CF
:10B990001A4310604246171D1F43022348463B606E
:10B9A000FCF764F91CBC90469946A246F0BD210004
:10B9B0000023D6E70040FCBF00E0004000F000405C
:10B9C00000C00040002070477047C046F0B5CE462A
:10B9D000474680B583B06B46591D13230B700D3B52
:10B9E0006B44994601244A46002313702300C26821
:10B9F000D02793403F06BB610C4B05000122180085
:10BA0000984602F059FF6B46DE1D3200012349467D
:10BA1000404602F059FFEB689C407C613078EB694E
:10BA2000C01A03B00CBC90469946F0BD00C003405C
:10BA3000F0B5CE46474680B585B06B46D9710368F0
:10BA4000364A5B680400934262D10921222369448B
:10BA50000B70183B6B449846012742460023137035
:10BA60003B00C268D02693400F253606B361012201
:10BA70006D442B4802F020FF01232A00414628484C
:10BA800002F022FF3B00E268934073612A789046FF
:10BA9000FF2A3AD00B2180206A466944087003A827
:10BAA0008146D2790270B36101221D4802F004FF81
:10BAB00001232A0049461A4802F006FF3B00E268CB
:10BAC00093400122736101260E2742446F443A706D
:10BAD0000D21D022A220694412060870904693617D
:10BAE0000F48012202F0E8FE01232A0039000C4829
:10BAF00002F0EAFE0123E2689340424653613000BF
:10BB000005B00CBC90469946F0BD00220026DBE74C
:10BB100069460122073198470600F0E7E1BB0010B3
:10BB200000C00340F0B5C64600B503682A4A1B6949
:10BB300082B00400934249D16B46D91C13230B7089
:10BB400001AB984601250023424613702B00C268C2
:10BB5000D02793403F06BB610122204802F0ACFE93
:10BB60006B46DE1D3200012341461C4802F0ACFE4C
:10BB7000E3689D407D613078E369C01A002827D0D2
:10BB8000E36906220133E3616B460125591D002359
:10BB90006A440B7013702B009046E268D0279340E4
:10BBA0003F06BB6101220D4802F086FE6B46DE1D9A
:10BBB000320001234146094802F086FEE3689D40B9
:10BBC0007D61307802B004BC9046F0BD9847D5E75F
:10BBD00001204042F6E7C046CDB9001000C0034046
:10BBE000F0B55746DE464E464546E0B587B004AB55
:10BBF0000C00591C22230B7004AB9F1C0125002351
:10BC00003B702B008146C068D026834036060292E6
:10BC10009046B3610122374802F04EFE04AA9446D2
:10BC2000072363449A46390001235246314802F003
:10BC30004BFE4B46DB6851469D40C4467561097812
:10BC40002A008C4460460390FF2805D9FF20401A43
:10BC500084466144029003910299002927D08C46C2
:10BC6000A4446246019204AAD71C802293467F3ADC
:10BC7000904605AE2278D0253270424659469A4009
:10BC80002D0639701B48AA613900012202F014FE0A
:10BC9000012352463100174802F016FE4B46424639
:10BCA000DB6801999A4001346A618C42E2D104ABAD
:10BCB000591DA223D0240B7004AB9D1D039B2406A9
:10BCC0002B700C48A261012202F0F6FD52460123BE
:10BCD0002900084802F0F8FD4B46DA68012393403A
:10BCE0000298636107B03CBC90469946A246AB46B9
:10BCF000F0BDC04600C00340F0B5D6464F464646AC
:10BD0000C0B50368454A1B6984B00400934200D063
:10BD10007FE06B46D91D13230B7002AB98460125BB
:10BD20000023424613702B00C268D02793400F2691
:10BD30003F06BB6101226E44394802F0BDFD01237C
:10BD400032004146364802F0BFFDE3689D407D6108
:10BD50003078E369C01A00285DD00D210D236944B5
:10BD60000B7001336B4499460023984601264B46DD
:10BD700042461A703300E268D02593400F272D0603
:10BD80006F44AB610122264802F096FD494601232B
:10BD90003A00234802F098FD3300E2680B219340FB
:10BDA0006B613A7869449246424640460A7003AA5B
:10BDB00091461070AB610122194802F07DFD4946A1
:10BDC00001233A00164802F07FFD3300E2680921A2
:10BDD00093406B613A78694490468D220A70833AA9
:10BDE0006A44504691461070AB6101220C4802F043
:10BDF00063FD01233A004946094802F065FDE36806
:10BE000040469E406E6104B01CBC90469946A246D6
:10BE1000F0BD98479FE701204042F4E7CDB90010FC
:10BE200000C00340F0B54546DE464E465746E0B5F5
:10BE30000126050089B0C0688846F7F70FFD33007A
:10BE4000EA68D02493402869240663626361431C36
:10BE50000FD0F7F703FD33002A690A20934063628D
:10BE6000A361F8F76DF92B690A209E406661F8F727
:10BE700067F9C849C848FFF72FFD01211020F7F7DF
:10BE8000D5FC01211220F7F7D1FC01211320F7F78F
:10BE9000CDFC0820F7F7E2FCD024802324065B00C9
:10BEA000636263616B46D91C422301260B70002339
:10BEB00001AF3B703300EA68B74893400122A361A9
:10BEC00002F0FAFC1F2201236A443900B24802F052
:10BED000FBFC3300EA68002793406A466361D27F27
:10BEE000122A07D0380009B03CBC90469946A246B9
:10BEF000AB46F0BD11216F3269440A7091466F3A2A
:10BF00006A449246802250460270A3617F3AA2485A
:10BF100002F0D2FC1F22514601236A449E4802F0DF
:10BF2000D3FC3300EA6893409A4663614346D917CD
:10BF3000AB61C9045B0B19434346984AD8040023FC
:10BF4000FBF7D6FE17218623694480460B7006ABAB
:10BF50009B4643465A461B0C137053460122A3616D
:10BF60008D4802F0A9FC1F2201236A4459468A48E1
:10BF700002F0AAFC3300EA68152193408722694445
:10BF800063610A70713A6A44924642465046120A08
:10BF90000270A3610122804802F08EFC1F225146EC
:10BFA00001236A447C4802F08FFC3300EA681321C5
:10BFB000934088224046694463610A7005AA107064
:10BFC0009246A3610122744802F076FC1F2251467A
:10BFD00001236A44704802F077FC3300EA680F21BD
:10BFE00093408E22694463610A7004AA17709046D8
:10BFF000A3610122684802F05FFC1F224146012331
:10C000006A44654802F060FC3300EA680D21934001
:10C010008F226944636190460A70813A6A441770BE
:10C020009246A36101225C4802F046FC1F22514661
:10C0300001236A44584802F047FC3300EA680B21A8
:10C0400093400C22694463610A7003AA17709246F8
:10C05000A3610122504802F02FFC1F2201236A44F1
:10C0600051464D4802F030FC3200EB6809219A40FD
:10C070008C206B466944626108700320DB7F0A37BD
:10C0800003436F443B704448A261012202F014FC58
:10C090001F22390001236A443F4802F015FC330097
:10C0A000EA6802AF93406A46D11DA62263610A7016
:10C0B000A23A3A703848A361033A02F0FDFB1F220E
:10C0C000390001236A44344802F0FEFB3300EA6879
:10C0D0001B219340CD226944636107AF0A70493A3E
:10C0E0003A702D48A361833A02F0E6FB1F22390023
:10C0F00001236A44284802F0E7FB3300EA6819216B
:10C1000093401A278B22694463616F440A70603A36
:10C110003A702148A3612A3A02F0CEFB1F2239006F
:10C1200001236A441C4802F0CFFB3300EA681D215A
:10C130009340892269441E2763610A7042466F4416
:10C140003A701548A3618E3A02F0B6FB1F223900FF
:10C1500001236A44104802F0B7FB3300EA680E4836
:10C1600093406A46511D4A4663610A706A46971DAC
:10C170004A463A70A361803A02F09EFB1F220123D7
:10C1800039006A44044802F09FFBEB6801279E4097
:10C190006661A7E6D430000000C003400048E80113
:10C1A000F0B5CE46474680B587B06B460125894637
:10C1B000D91C002301AF3B7098462B00C268D026E3
:10C1C000934036060D700400B3610122794802F0F5
:10C1D00073FB172201236A443900764802F074FB8E
:10C1E0002A00E36800209A406B467261DB7DDB43E6
:10C1F0009B0700D19FE06B46591D12230B706B46C5
:10C200009F1D43466B483B70B261012202F054FB14
:10C21000172201236A443900664802F055FB2B00BF
:10C22000E26893406A467361D17D08220A4200D0D9
:10C2300086E009210A25D026812269446D4436060C
:10C240000A702A705B48B361803A02F035FB17220E
:10C250002900012501236A44564802F035FB2B00D2
:10C26000E26893404A467361002A00D07FE01121C2
:10C2700022621D22694412270A704A466F443A70AE
:10C280004C48B361012202F017FB17223900012349
:10C290006A44484802F018FB2A00E3680F219A40DC
:10C2A0006B469D207261DB7D6944087004AFAB432F
:10C2B0003B704048B261012202F0FEFA17223900B9
:10C2C00001236A443B4802F0FFFAE36815219D40D0
:10C2D0008D23756169441627D0260B70002336061E
:10C2E0006F443B700122B5613248984602F0E4FA8F
:10C2F00017220125390001236A442E4802F0E4FA8E
:10C300002B00E26813219340A222694473610A70F2
:10C31000424605AF3A702748B361013202F0CCFAC9
:10C32000172201236A443900224802F0CDFAE3685B
:10C3300001209D40756107B00CBC90469946F0BD48
:10C3400069469220073102AF08703A701948B3610C
:10C35000073A02F0B1FA172201236A44390015485E
:10C3600002F0B2FA2B00E2689340736161E70D219D
:10C370001D2269440E270A7000226F443A7025621C
:10C380000132B3610B4802F097FA172239000123FA
:10C390006A44084802F098FA2A00E3680B219A40A0
:10C3A0009D206B466944726108700120DB7D03AFFC
:10C3B00003437DE700C00340F0B50124D6464F4655
:10C3C00046462300C0B5C26884B0050093400029EA
:10C3D0003DD00F226A449046826A002A17D06A46EE
:10C3E000D026D11DC02202AF0A703606803A3A70BC
:10C3F0004448B3613F3A02F05FFA012342463900F4
:10C40000404802F061FA2300EA6893407361092111
:10C4100081220A26D02469440A706E44023224061E
:10C4200032703848A361823A02F046FA012342464C
:10C430003100344802F048FA0123EA68934063610E
:10C44000012004B01CBC90469946A246F0BD0921CB
:10C4500081220A27D02669440A706F4436060232C8
:10C460003A702848B361823A02F026FA0F236B44EF
:10C470009846390001234246224802F025FAEB682B
:10C4800012229C400B279246113A74616F4403AE0E
:10C49000914603E00020F7F753FEEB6852463A70EE
:10C4A000002232704A46D0249A402406A261390004
:10C4B0000122144802F000FA0123424631001148DB
:10C4C00002F002FA4B46EA689340424663611178F3
:10C4D00008220A42DED00D210E26922069446E44C5
:10C4E000087032700748A361012202F0E5F90123C8
:10C4F00042463100034802F0E7F94A46EB689A40A9
:10C5000062619DE700C00340F0B5DE4657464E46E7
:10C510004546E0B58BB06B468A46D91D12230B7099
:10C5200002AB984600239946012643464A461A70B4
:10C530003300C268D027934027243F060500BB6123
:10C5400001226C44B74802F0B7F9012322004146AA
:10C55000B44802F0B9F93300EA6893407B6122786D
:10C5600090465246002A00DC37E10D211D22694425
:10C570000A700F3A6A444846934610702E620122B0
:10C58000BB61A84802F098F9012322005946A5484A
:10C5900002F09AF93200EB680B219A409D20694421
:10C5A0007A61087003A88146012023780343484636
:10C5B0000370BA619B48012202F07EF949460123CB
:10C5C0002200984802F080F93300EA68092193407C
:10C5D000A22269447B610A70983A6A4450469146A7
:10C5E0001070BB6101228F4802F066F949460123B1
:10C5F00022008C4802F068F9EB6815219E409223D6
:10C600007E61D027424669440B7099467C3B6B445F
:10C610003F069A461A70BE6101260122814802F047
:10C620004BF90123220051467E4802F04DF93300B8
:10C63000EA68132193404A4669447B6140460A7088
:10C6400005AA91461070BB610122764802F034F9C8
:10C65000012322004946734802F036F93200EB68A4
:10C6600041469A4060237A610B40402B00D073E032
:10C6700000202B6AE861002B66D119211320694440
:10C6800008700730684480460370BA61654801222B
:10C6900002F012F9414601232200624802F014F927
:10C6A0003300EA681F2193407B61227869449046F9
:10C6B0001022D0270A7000223F0608AE3270594877
:10C6C000BB61013202F0F8F831000126012322009B
:10C6D000544802F0F9F83300EA681D2193408D2098
:10C6E00069447B6108706F38684481462278027023
:10C6F000BB6101224B4802F0DFF8494601232200CA
:10C70000484802F0E1F83300EA681B21934007A88B
:10C710008122814669447B610A700270BB61803A64
:10C72000404802F0C9F80123220049463D4802F082
:10C73000CBF8EB689E407E6140460BB03CBC904617
:10C740009946A246AB46F0BD1721222369440B70DF
:10C7500006AB9846187098E722236B44984621212F
:10C7600000234046694403700E702E48BA610122CE
:10C7700002F0A2F84146012322002A4802F0A4F860
:10C780003300EA68002193407B6122788846862A3C
:10C79000D2D08D22253169440A70673A6A444046F6
:10C7A00091461070BB6101221E4802F085F849468F
:10C7B000012322001B4802F087F83300EA68232196
:10C7C0009340812269447B610A7009AA91468622BE
:10C7D00048460270BB61853AA2E74A4611212A62A7
:10C7E0001D2269440A700B3A6A444846924610700A
:10C7F000BB6101220B4802F05FF801232200514681
:10C80000084802F061F83200EB680F219A409D2041
:10C810007A61237869440870B34304A803708146A1
:10C82000BA61DFE600C00340F0B5C64600B582B08D
:10C830006B46591D1A230B70143B6B449846012418
:10C840004246002313702300C268D02793403F065E
:10C850000500BB610122114802F02EF86B46DE1D77
:10C860003200414601230D4802F02EF8EB689C404F
:10C870007C61A869FBF7DEFC8022094BD205FBF73F
:10C88000ABFC431E984143420720347818409D304A
:10C89000201A02B004BC9046F0BDC04600C0034060
:10C8A000DD4ABF41F0B5CE46474680B585B06B4600
:10C8B0008946591CC023012400270B70BE3B6B44E2
:10C8C0001F7098462300C268D02593402D060600AD
:10C8D000AB6101224E4801F0EFFF0F2201236A44B1
:10C8E00041464B4801F0F0FF2300F26893404A466E
:10C8F0006B61002A67DD6A46D11D1D220A7002AAFB
:10C90000177034629046AB610122414801F0D4FFB8
:10C910000F2201236A4441463D4801F0D5FF220021
:10C92000F36869469A409D2005316A61087068463F
:10C930006B46871D0120DB7B03433B703448AA61B3
:10C94000012201F0B9FF0F22390001236A44304867
:10C9500001F0BAFF2300F26801AF93406A46D11C90
:10C96000A2226B610A704A463A70AB6101222848E4
:10C9700001F0A2FF0F2239006A440123244801F08C
:10C98000A3FFF3680D219C400E276C618123D02505
:10C9900069440B706F4404332D063B700122AC6177
:10C9A0001B4801F089FF0F2201236A44390018480F
:10C9B00001F08AFF0123F26893406B6105B00CBC63
:10C9C00090469946F0BD0B211D2269440A7003AAC6
:10C9D000177037629046AB6101220D4801F06CFF81
:10C9E0000F2201236A444146094801F06DFF2200ED
:10C9F000F36809219A406B460A279D206A61DB7B18
:10CA000069446F44A34308703B70AA61AEE7C04617
:10CA100000C00340F0B5CE4647460500012080B572
:10CA2000EB6885B09840002A25D10B000E2900DD67
:10CA3000A5E06A46D11C89220A70DA43D217134056
:10CA4000D026702201AC1343360623700122B06158
:10CA50004E4801F031FF0F2201236A4421004B4868
:10CA600001F032FF0123EA689340736105B00CBC0A
:10CA700090469946F0BD112929DD142900DD80E09A
:10CA80006B46CC1ED91DCD2302AE0B70463B3370D6
:10CA9000D0230F271B06986101223C48984601F0DD
:10CAA0000BFF310001266F4401233A00374801F0A3
:10CAB0000BFF3300EA689340424653616A46511DBA
:10CAC0008B220A70853A6A449146312227E00C0095
:10CAD000022958DB0B21CD2369440B7003AE493B7F
:10CAE0003370D0230F271B069861012227489846F0
:10CAF00001F0E2FE310001266F4401233A00234891
:10CB000001F0E2FE3300EA68092193404246536196
:10CB10008B2269440A70813A6A4491462B22484626
:10CB20000270424619489361012201F0C5FE0123BB
:10CB30003A004946154801F0C7FE3300EA680D2166
:10CB400093404246536189220E2669440A700A3A8C
:10CB5000FF3A023C14436E443470D0242406A3618F
:10CB600081320A4801F0A8FE01233A00310007484B
:10CB700001F0AAFE0123EA689340636176E70E2381
:10CB800057E714217CE70224A4E7C04600C0034015
:10CB9000F0B54546DE4657464E46E0B5050087B03F
:10CBA000052900DC0AE10C2900DDFCE0062900D1A2
:10CBB00004E109014BB298460921B12369440B7085
:10CBC000A73B6B44994601264A46C32313703300A2
:10CBD000EA68D027934017243F06BB6101226C44CA
:10CBE000944801F069FE494601232200914801F072
:10CBF0006BFE3300EA6893406A46D11DB7227B6121
:10CC00000A7002AA91460A2248460270BB61093A9C
:10CC1000884801F051FE012322004946854801F071
:10CC200053FE3300EA6893407B610D211E22694464
:10CC30000E26D0270A7000223F066E4432709146BD
:10CC4000BB6101327B4801F037FE31000126012330
:10CC50002200784801F038FE3200EB680B219A4040
:10CC60009E2369447A610B7003AB9A460F232078A8
:10CC7000034040461843030050460370BA616D48B4
:10CC8000012201F019FE012322005146694801F0FA
:10CC90001BFE3300EA680F2193401D2269447B612B
:10CCA00048460A7004AA90461070BB610122614890
:10CCB00001F002FE0123220041465E4801F004FE1D
:10CCC0003200EB689A407A6123781B11092B6EDCE5
:10CCD00059499B005B58994613211E236944D0276C
:10CCE0000B7000233F0605AE33705248BA61012233
:10CCF0009B4601F0E1FD31000126012322004D4851
:10CD000001F0E2FD3300EA68112193407B61227853
:10CD10006944924626220A70143A6A44584690465C
:10CD20001070BB610122434801F0C6FD414601235A
:10CD30002200404801F0C8FD3300EA68310093400A
:10CD40007B61984653461B1199404846FAF766FFA7
:10CD50000100FA2080002778FAF760FF10282ADC0B
:10CD600008239F431521A62369440B70903B6B4415
:10CD7000D0261F70994643463606B36101222D48DE
:10CD800001F09AFD2200012349462A4801F09CFD4A
:10CD90000123EA689340736107B03CBC9046994612
:10CDA000A246AB46F0BD40235B42984604E7012310
:10CDB0005B42994690E708231F43D3E76B46591D12
:10CDC000B1230B70AB3B6B44984601264246C5230A
:10CDD00013703300EA68D027934017243F06BB61E5
:10CDE00001226C44134801F067FD414601232200F3
:10CDF000104801F069FD3300EA6893406A46D11C8F
:10CE0000B7227B610A7001AA90460C22404602704C
:10CE1000BB610B3A074801F04FFD01232200414658
:10CE2000044801F051FD3300EA68934060227B61C1
:10CE30009046FAE600C00340ECF50010F0B5DE467F
:10CE4000454657464E46E0B5050085B00800FBF75D
:10CE5000F1F9974B002206000F00FBF7C3F90023FE
:10CE60009846002855D1934B002230003900FBF73B
:10CE7000B9F91023984600284BD18F4B002230007F
:10CE80003900FBF7AFF920239846002841D18B4B9E
:10CE9000002230003900FBF7A5F93023984600281E
:10CEA00037D1874B002230003900FBF79BF9402334
:10CEB000984600282DD1834B002230003900FBF723
:10CEC00091F950239846002823D17F4B002230004F
:10CED0003900FBF787F960239846002819D17B4B6E
:10CEE000002230003900FBF77DF9702398460028B6
:10CEF0000FD1774B002230003900FBF773F9431E46
:10CF000098410F227023404290435B4280469C46EA
:10CF1000E0446B46591D1D230B709A46173B6B442A
:10CF20009B460023994601265B464A461A70330009
:10CF3000EA68D02793400F243F066C44BB6101226E
:10CF4000644801F0B9FC594601232200614801F010
:10CF5000BBFC3200EB689A406B46D91C9D237A617A
:10CF60000B7001AB9B460F232078034040461843CB
:10CF7000030058460370BA615648012201F09CFC38
:10CF8000594601232200534801F09EFC3300EA6811
:10CF9000484693406A46D11D52467B610A7002AAF8
:10CFA00090461070BB6101224A4801F085FC0123C4
:10CFB00022004146474801F087FC3200EB689A4066
:10CFC0007A6123781B11092B6ADC43499B005B586B
:10CFD00099460B211E236944D0270B7000233F067E
:10CFE00003AE33703B48BA6101229B4601F064FCFA
:10CFF0003100012601232200364801F065FC330090
:10D00000EA68092193407B6122786944924626228E
:10D010000A701C3A6A44584690461070BB6101225F
:10D020002C4801F049FC414601232200294801F027
:10D030004BFC3300EA68310093407B6198465346CD
:10D040001B1199404846FAF7E9FD0100FA208000DB
:10D050002778FAF7E3FD102826DC08239F430D21EB
:10D06000A62369440B70983B6B44D0261F709946E9
:10D0700043463606B3610122164801F01DFC22002A
:10D0800001234946134801F01FFC0123EA6893403D
:10D09000736105B03CBC90469946A246AB46F0BDD4
:10D0A00001235B42994694E708231F43D7E7C04614
:10D0B0000078BE400050C4400078CE400050D440BC
:10D0C0008084DE40805CE4408084EE408084FE40CA
:10D0D00080840E4100C00340ECF50010F0B5CE4650
:10D0E000474680B5050083B00C00082900DD082400
:10D0F0006B46591D1D230B70173B6B44994600234B
:10D100004A461370EA680133D027984693403F0699
:10D11000BB610122194801F0CFFB6B46DE1D3200D6
:10D1200001234946154801F0CFFB4346EA686946AA
:10D1300093409D207B6103313278087001AF052C4C
:10D1400000DA05240E20043C8243640014433C7042
:10D15000D0242406A3610122084801F0ADFB32006F
:10D1600001233900054801F0AFFB0123EA68934031
:10D17000636103B00CBC90469946F0BD00C003400B
:10D18000F0B5CE46474680B583B06B468946591DFB
:10D19000A0230B709A3B6B4498464B4642460124B1
:10D1A0001B1213702300C268D0259340174E2D0622
:10D1B0000700AB610122300001F07EFB6A46414668
:10D1C00001230732300001F07FFB2300FA68484654
:10D1D00093406A46D11CA1226B610A7001AA1070AB
:10D1E0009046AB610122300001F066FB6A460123E4
:10D1F00007324146300001F067FBFB689C406C61E0
:10D2000003B00CBC90469946F0BDC04600C0034038
:10D21000F0B5CE46474680B583B06B46591D1E23F8
:10D220000B70183B6B44994601244A460023137047
:10D230002300C268D0259340194E2D060700AB612C
:10D240000122300001F038FB07236B449846494621
:10D2500042460123300001F037FB2200FB6869469B
:10D260009A409E20033143466A61087001A88146B6
:10D2700004201B78034348460370AA613000012252
:10D2800001F01AFB012342464946300001F01CFB25
:10D29000FB689C406C6103B00CBC90469946F0BDA5
:10D2A00000C0034009490A4B0831196009490022AE
:10D2B00099600821D9600331196101395A605961B7
:10D2C0009A61DA611A625A629A62704714F6001023
:10D2D000582F002000C00340F0B545464E46DE46BC
:10D2E0005746C54BE0B59846CB5C85B00E0015009F
:10D2F0008844002B00D158E22A2B00D125E20022DD
:10D30000414602E02A2F00D11EE20132D2B28F5CE8
:10D31000002FF7D188460020B84C424606E0052889
:10D320002ED85B0023540130C0B2135C002BF6D022
:10D330002D2BF6D1431CDBB2994692469046CA4447
:10D34000052807D80522121AD2B20132201840212E
:10D35000FBF704FB53464846197800230A00303A8D
:10D36000D2B200290CD0092A00D9FEE799005B1837
:10D370005B009B1842460130C0B2DBB2115CEDE7A6
:10D380005B00DBB2012F00D1E1E160221343A37106
:10D39000002319002A1D944259410A00211D8D4283
:10D3A0005B41134300D1ECE1AB0700D0E9E1236816
:10D3B0002B6023792B7163796B71A379AB7133780F
:10D3C000002B00D1EFE12A2B00D1BBE1002202E0CB
:10D3D0002A2F00D1B6E10132D2B2B75C002FF7D1CB
:10D3E000002006E005282CD85B0023540130C0B291
:10D3F000335C002BF6D02D2BF6D1431CDBB29846C4
:10D40000B146C144052807D80522121AD2B201320A
:10D4100020184021FBF7A2FA4B464046197800231A
:10D420000A00303AD2B200290BD0092A00D9FEE70F
:10D4300099005B185B0001309B18C0B2DBB2315C15
:10D44000EEE75B00DBB2012F00D183E160221343E2
:10D45000002128000F000B3084424F41EA1D3800A4
:10D46000271DBA424941A371014300D17BE19107D5
:10D4700000D078E1236813602379EB7263792B7312
:10D48000A3796B735E4AB35A002B00D08BE0012264
:10D490006B7B0F2013436B730E220E230321A954C1
:10D4A000F0222A540A22FF32B25C02339BB2002AD5
:10D4B00009D00B36FF360136EA54721E127801335A
:10D4C0009BB2002AF7D18024A4002B53C020FBF785
:10D4D0001DFB0020FBF71AFBC0224A4BEA522A5BD5
:10D4E000531E9BB2002A00D15BE16A1C9146FF3CAF
:10D4F000A8469944FF3C0CE03800FBF707FB414A83
:10D500002B789446444464442370340001354D45DF
:10D510001ED02F78661CF6B2C02F2CD0DB2FEBD19B
:10D52000DB20FBF7F3FADD20FBF7F0FA354A434640
:10D5300094461B1963441F70130002344644263B73
:10D540006644E4B2FF3B0135337026004D45E0D11F
:10D550004546C020FBF7DAFA2A4B00209C46AD195D
:10D56000433B6544FF3B2B7005B03CBC904699465D
:10D57000A246AB46F0BDDB20FBF7C8FADC20FBF788
:10D58000C5FA204A434694461B19283A6344FF3A99
:10D590001A70634602344644273B6644E4B2FF3BBC
:10D5A00033702600B2E7013BB35201239C463F3360
:10D5B000984663460E20B4461900039201938946AB
:10D5C0000D4A8B004B4491465B004B4463441E0064
:10D5D0001B78002B00D1C4E02A2B00D1A1E000224F
:10D5E00002E02A2F00D19BE00132D2B2B75C002FBB
:10D5F000F7D1019100220EE0070300002C1F00204C
:10D600006E04000002020000052A56D85B00A354F5
:10D610000132D2B2B35C002BF6D02D2BF6D1531CC5
:10D62000DBB201919946052A00D9C0E04346A354D4
:10D630004B46062B00D190E0931CDBB20293494687
:10D640004346B3466354029BCB44062B18D01900C3
:10D65000D31CDBB29A46434663545346062B0FD085
:10D66000131DDBB20293514643466354029B062BC3
:10D6700006D0190043466354012A00D18AE0637141
:10D680005B461B78019A9A460023494691465246CA
:10D690008246180013001A00303AD2B2002B00D193
:10D6A00089E0092A00D9FEE78300C3185B00013135
:10D6B0009A18C9B2D0B2735CEDE701915B00DBB29E
:10D6C000012F30D060221343A371237801992B548A
:10D6D0006278431C9BB2EA54A278831C9BB2EA5442
:10D6E000E278C31C9BB2EA542279031D9BB2EA5430
:10D6F0006279431D9BB2EA54A279831D9BB201312A
:10D70000EA54CAB2019262466146039EC31D925B0F
:10D710009BB2571E8F53002A0AD0180001994EE77A
:10D720000191012766E7202252421343DBB2CBE787
:10D7300001275C1E295D0830394366461A0080B215
:10D740002955ABE601274BE688460127E3E5E022B1
:10D7500013431CE6E02213437AE6B3790A009A46A3
:10D7600092E7002746E722786B73EA7162782A72A3
:10D77000A2786A72E278AA722279EA7262792A73CE
:10D7800080E623782B7063786B70A378AB70E378B6
:10D79000EB700EE65B461B78019A9A460223994687
:10D7A00072E70226D5E600271AE60027B3E5F35C08
:10D7B0000A009A4668E74B460193030050467DE70E
:10D7C000F0B55746DE464E4645468E23E0B5170077
:10D7D0000022DB00FA540B7883B08A460120C02B6C
:10D7E00006D003B03CBC90469946A246AB46F0BD7D
:10D7F0004B78002B00D1BFE1FF2B00D13AE2602231
:10D800000025DB4BFA5453465A78D94B6C1C9C4686
:10D81000A0B23918521061440A70202A01D00500C4
:10D82000441C53469A78D24BA0B29C4639185210E9
:10D8300061440A70202A01D00500441C5346DA785E
:10D84000CB4BA0B29C463918521061440A70202A72
:10D8500001D00500441C53461A79C54BA0B29C4622
:10D860003918521061440A70202A01D00500441C66
:10D8700053465A79BE4BA0B29C46391852106144A7
:10D880000A70202A01D00500441C53469979A4B29D
:10D89000C8062200000F14D0B54B3C199C46DE3B55
:10D8A0006444FF3B2370A91CEC1C89B2A4B2220083
:10D8B0007918092800D9BCE153466144303008701A
:10D8C000997949B2002908DAA94A3B199446E13A04
:10D8D000FF3A634401341A70A2B2A54BBA189C46B1
:10D8E0000023624413705346DB795B103B70203B8E
:10D8F0005A42534152465B42127A9BB25C1CA1B21F
:10D9000052107A54202A01D00B004C1C5246527AF5
:10D91000A1B252107A54202A01D00B004C1C52465E
:10D92000927AA1B252107A54202A01D00B004C1CDA
:10D930005246D27AA1B252107A54202A01D00B005A
:10D940004C1C5246127BA1B252107A54202A01D0AC
:10D950000B004C1C5246527BA4B2D0062500000F8F
:10D960000DD02D223A55DC1C9A1CA4B292B225008F
:10D97000092800D971E153463030B8545A7B52B26D
:10D98000002A03DA2A233B550134A5B2002352466C
:10D990007B55527BD20700D56EE10E335344994636
:10D9A000852301229B009C469046BC440D3246468E
:10D9B0009346B8464F46E146B3B201934B463A7898
:10D9C0006B4D52101A70203A53425A410123AC4613
:10D9D00092B2991AB30000939B195B00787889B2D0
:10D9E00043445B18401063441870202801D1524210
:10D9F00091B25F4C009AA44692194D1C5200ADB2F0
:10DA0000B87842445219401062442B00107020280C
:10DA100003D002318BB229001D00554C009AA44658
:10DA200092195200F8784244D218401062441070A3
:10DA3000202803D06B1C9BB229001D004C4C009A7F
:10DA4000A4469219520038794244D21840106244D8
:10DA50001070202803D06B1C9BB229001D00444C81
:10DA6000009AA4469219520078794244D218401084
:10DA700062441070202803D06B1C9BB229001D004B
:10DA80000F24BA79501020401AD0394C009AA4467D
:10DA9000921952004244D318DE3C6344FF3C1C7090
:10DAA0008B1C9BB29C46CB1C9BB21D00092800D945
:10DAB0009CE02F4962448C46303062441070BA7941
:10DAC00052B2002A0CDA009A0135921952004244EF
:10DAD000D318274A9446E13A6344FF3A1A70ABB22E
:10DAE000009A9419224A6400944600224444E318A0
:10DAF00063441A705B46012207339BB29B46BB7995
:10DB00001A4270D10A239C465B4601360737E1442E
:10DB10004D2B00D050E7443B47461A000193154B6C
:10DB2000FA523A23BB725B46524602339BB2D25C36
:10DB3000002A74D0FE245B46FF34D91CE41A89B253
:10DB4000A4B251440334022303E001330131A34260
:10DB500005D0F81842720A781800002AF5D100237F
:10DB6000381883728E230122DB00FA54002038E635
:10DB70000A0200006E0200000B008978C02925D03F
:10DB8000002302320224C0255646BC4607E00200AC
:10DB90003970B15C01339BB21400C02913D0501C02
:10DBA000F71880B2DB29F2D134196478DC2C32D03A
:10DBB000DD2CECD1023292B23970B15C01339BB2F0
:10DBC0001400C029EBD1B2466746534400221A70B4
:10DBD00053461B782E4A5B10BB54203B5A4253419C
:10DBE0005B429DB20FE64746019A98E764461519D5
:10DBF000274CD318A446DA3C6544FF3C2C701C002B
:10DC00000D1D0A216444FAF731F83031ADB22170AC
:10DC1000BA792B0054E702323D7092B2B9E7012085
:10DC20000023381883728E230122DB00FA5400206F
:10DC3000D7E5174BBA189C46DA3B6144FF3B0B70A3
:10DC400063460A212C1DD518FAF710F853463031D7
:10DC5000A4B229709979220033E631210433B954F2
:10DC600027399CB2FAF702F85346303179555A7B7E
:10DC7000250084E60220B4E5064ABB523A23BB7273
:10DC800053461A7C002ACAD00E239B4652E7C04650
:10DC90000A0200006E020000F0B5C64600B50B781F
:10DCA0000E00002B4AD02A2B43D0002201E02A2D5F
:10DCB0003FD00132D2B2B55C002DF8D10020204C0B
:10DCC00006E0052821D85B0023540130C0B2335C44
:10DCD000002BF6D02D2BF6D1471CFFB2F319984636
:10DCE000052808D80522121AD2B201322018402184
:10DCF000FAF734FE4346197800230A00303AD2B2CC
:10DD0000002902D0092A0BD9FEE75B00DBB2012D06
:10DD100011D0602213432000A37104BC9046F0BDD3
:10DD200099005B185B0001379B18FFB2DBB2F15D15
:10DD3000E3E70125C2E7E0221343ECE70025BDE756
:10DD40002C1F002010B5062000F06AFB0120F6F71A
:10DD5000EDFFC046F0B557464546DE464E46E0B5B7
:10DD60000D000B3583B00700162D28D8102900D9D7
:10DD7000C1E000F0A7FA102518230220CE4EF318B8
:10DD80001A005C68083A944200D160E1032362689B
:10DD90009A431300E268A168CA6091600122E31807
:10DDA000596838000A435A6000F08EFA20000830A3
:10DDB00003B03CBC90469946A246AB46F0BD072353
:10DDC0009D4300D597E0A94200D994E000F07AFA8B
:10DDD000F823FF339D4200D85EE1680A00D18EE04F
:10DDE000042800D939E138239846A80980443930FD
:10DDF000C100B14E71180839CC68A14218D0032374
:10DE000062689A431300521B0F2A00DD1DE1002AAD
:10DE1000C0DA03239C4608E06246636893435A1BBA
:10DE20000F2A00DD11E1002AB4DAE468A142F3D13F
:10DE3000320034690832944267D003236168994301
:10DE40008A460B00491B0F2900DD12E17261326125
:10DE50000029A3DA994A924500D948E1DB08FF3A44
:10DE60009910FF3A8A40DB0071689B190A43996850
:10DE70007260E360A1609C60CC60012183109940D6
:10DE8000914248D80A4205D10323984349000430FF
:10DE90000A42FBD003239846C3009946B144CC46BE
:10DEA00082466346DC68A44507D1F9E0002A00DB1E
:10DEB0000EE1E468A44500D1F2E042466368934372
:10DEC0005A1B0F2AF2DD0120804661190543656067
:10DED000A068E5680836C560A8604046F160B1609A
:10DEE00010434860CE608E603800E25000F0ECF9DC
:10DEF000200008305CE70C2300203B6058E78021BD
:10DF00003F2389004020984673E7012172688310FF
:10DF100099409142B6D90323B46862689A43904607
:10DF2000AA4203D3531B0F2B00DD80E0644B654AEC
:10DF30009A4693461B681268EB18013200D138E10B
:10DF4000614A944663441B0B1B03009300993800FD
:10DF500000F0BCF903008146013300D1F6E04346EE
:10DF6000E218824200D9EFE051464968009B8C4696
:10DF7000514663444B60824200D14BE159460968E7
:10DF8000013100D15DE149468A1AD31852465360E7
:10DF900007234A461A40019200D120E108214B464E
:10DFA00089469B1A99440099484B49449B1A5B1A2D
:10DFB0001B051B0D0091380019009B4600F086F9E7
:10DFC000431C00D15AE1534652465B6849465B44C4
:10DFD00053604A46B260801A012258441043486098
:10DFE000B44211D041460F2900D827E107200C394F
:10DFF00081436068024005200A43626062185060F5
:10E0000090600F2900D941E15246D26A934201D96A
:10E010005246D3620322B468616891430A005146B4
:10E02000096B8B4200D895E051460B6392E00122C8
:10E03000290013431143651961603800B5606B60B6
:10E0400000F042F920000830B2E64046F0E6DC6815
:10E050000230A34200D1EBE698E614286ED954288A
:10E0600000D9A9E06E239846280B80446F30C10088
:10E07000BFE6012360191D43656070613061C260B5
:10E0800082601A0053460A4342603800E15000F0B3
:10E090001BF9200008308BE62B00E80808336DE6FA
:10E0A00008239B46073BDC449B46DA4443465246E2
:10E0B000134200D0F5E667E0D8190020FF01000008
:10E0C000341F0020D01900200F100000081000009D
:10E0D0000122E318596838000A435A60E368A268CD
:10E0E000D3609A6000F0F0F82000083060E65A0A29
:10E0F000042A3AD9142A00D983E05B239846904435
:10E100005C32D20008235B429C46B21894446346BA
:10E110009968032399468C4559D04B464A689A43DF
:10E12000524502D989688C45F7D1CB6872689C4604
:10E130006346A160E3609C60CC609EE65B239846EA
:10E1400080445C30C10054E6B4427ED00323B468FE
:10E1500062689A43531B954202D80F2B00DD66E795
:10E16000380000F0B1F8002022E69A0938239846DA
:10E1700090443932D200C5E74B461A68083B013853
:10E1800091469A4200D098E043460342F4D1736826
:10E190008B4373604900994200D9BCE6002904D141
:10E1A000B9E6042294464900E2440B42F9D05046B5
:10E1B00072E610330093C9E6AA235B00984233D875
:10E1C000DD3B9846E80B80447830C10011E64346B9
:10E1D00001229B109A4073681A437260A8E7009B63
:10E1E00038004B4400931B055B421B0D19009B46F6
:10E1F00000F06CF8431C00D0E5E6002300989B4635
:10E20000E1E6542A29D81A0B6E23984690446F32BF
:10E21000D20077E7110500D0B0E60120009AB1687E
:10E22000424402434A60EFE6254B984220D87C23C3
:10E230009846A80C80447D30C100DAE54B465A6010
:10E240008EE75B464A461A60A2E651464968009B43
:10E250008C46514663444B6090E6AA2149008A42AD
:10E260001CD8DA0B7723984690447832D20049E7DD
:10E27000FE217E2389007F209846BAE5009B019805
:10E280009C460023083860449B469CE621003800E9
:10E29000083100F0D3F953465B68B5E608498A4275
:10E2A00006D89A0C7C23984690447D32D20029E708
:10E2B000FE227E239200984624E773686AE7C046F0
:10E2C000540500007047C0467047C046002370B533
:10E2D000064C050008002360F6F72AFD431C00D019
:10E2E00070BD2368002BFBD02B60F9E70C400020A9
:10E2F00010B580210400FFF72DFDB7239B00E050EF
:10E30000002807D002000023803208C09042FCD1D0
:10E31000002010BD01204042FBE7C046B7239B0010
:10E32000C25810B50023002A01D0180010BDFFF715
:10E33000DFFF0300F9E7C046F8B505000C00160042
:10E340001F2909D8B727BF00C359002B09D0A40043
:10E350001C1920682660F8BD162303600120404286
:10E36000F9E7FFF7C5FF002801D1EB59EFE70120DE
:10E370004042F0E770B505000C001F2922D8B723F2
:10E380009B00C358002B0ED08A009B181A68002AE5
:10E3900009D0012A10D0511C10D000212000196092
:10E3A0009047002070BD280000F07EF82200010098
:10E3B000280000F065F8F5E70020F3E71623036076
:10E3C0000120EFE71623036001204042EAE7C04640
:10E3D00070B505000C001F291DD8B726B60083595B
:10E3E000002B10D0A2009B181A68002A09D0511CDB
:10E3F0000FD0012A12D00021200019609047002080
:10E4000070BD0120FCE7FFF773FF002803D1AB5973
:10E41000E8E70220F4E701204042F1E70320EFE7BC
:10E4200010B5034B01001868FFF7A4FF10BDC046EC
:10E43000A015002010B5044B0A001B68010018004D
:10E44000FFF77AFF10BDC046A0150020B722064B8B
:10E4500092001B6810B59A580020002A00D010BD09
:10E460001800FFF745FFFAE7A015002010B5034B91
:10E4700001001868FFF7ACFF10BDC046A0150020D2
:10E48000002370B5074C050008001100236000F060
:10E49000C7F9431C00D070BD2368002BFBD02B6054
:10E4A000F9E7C0460C40002010B500F0B1F910BDEE
:10E4B000024670B50A4392072AD11E4DEE0104C8E8
:10E4C00008C9541B9443344017D0D0B2D9B2401A73
:10E4D0002106014310D190B299B2401A21040143A0
:10E4E0000AD110021902000A090A401A2102014346
:10E4F00002D1100E190E401A70BD9A42DFD010BA28
:10E5000019BA884201D9012070BD0020C04370BDF6
:10E5100002780B7801300131002A09D09A4207D1E4
:10E5200002780B7801300131002A01D09A42EFD0F5
:10E53000D01A70BD0101010110B5040083070AD093
:10E540000378002B23D0032202E00378002B1CD099
:10E5500001301042F9D102680E4B0F49D318934392
:10E560000B420FD1043002680A4BD31893430B427D
:10E5700008D104300268074BD31893430B42F1D003
:10E5800000E001300378002BFBD1001B10BD002000
:10E59000FCE7C046FFFEFEFE80808080F8B50C00E0
:10E5A0000600FFF78FFE204FBB685D6803239D4385
:10E5B0001E4B2C1B9C466444240B1D4B013C240326
:10E5C0009C4207DD00213000FFF780FEBB685B192D
:10E5D000984204D03000FFF777FE0020F8BD61427A
:10E5E0003000FFF773FE431C0DD00122BB682D1BCA
:10E5F00015435D600F4B30001A68141B1C60FFF759
:10E6000063FE0120EAE700213000FFF75FFEBA68F1
:10E61000831A0F2BDEDD08490968401A0549086096
:10E6200001210B435360D5E7D8190020EF0F0000FC
:10E63000FF0F0000381F0020D0190020F8B5CE468B
:10E640004746050080B50C1E55D0FFF73BFE210064
:10E6500008394F68012438000323A0430A1856687C
:10E660009E43B146644EB368934229D04B465360F3
:10E67000D3189C463C4242D10F68C91B8B68C01915
:10E68000984663465F6808239C46B4442740E045AB
:10E690006AD04346CC68DC60A360002F32D10124ED
:10E6A00048440443A0469368544C0F18A34200D139
:10E6B0007FE0D268DA60936043464B60386025E0C3
:10E6C00003004B443C4206D10A68891A88689B18AB
:10E6D000CA68C260906001221A434A60484AB16029
:10E6E00012689A4204D8474B28001968FFF756FF72
:10E6F0002800FFF7E9FD0CBC90469946F8BD5F681D
:10E700002740CCD0012303434B6008503E4B984236
:10E710001AD9430A042B33D8820914003932383409
:10E72000D200B218083A936803279A4239D05C683D
:10E73000BC43844233D99B689A42F8D1D368CB60FA
:10E740008A609960D160D3E7C008FF3B8210FF3B2D
:10E7500093407268C000134373608619B368CE603B
:10E760008B60B160D960C3E7002F41D1030090688E
:10E770004B44D2681C43C26090604C60CB50B7E7FA
:10E78000142B07D9542B1CD8020B14006F326E3493
:10E79000D200C6E71C005C335B34DA00C1E71A0024
:10E7A000CCE70123A410A3407068034373601300F7
:10E7B000C5E7D9609960CB608B6043464B60386099
:10E7C00096E7AA225200934205D8C20B1400783271
:10E7D0007734D200A5E70D4A934205D8820C140085
:10E7E0007D327C34D2009CE7FE227E24920098E7A2
:10E7F00004434C6010607BE7D8190020E01900202A
:10E80000D4190020341F0020FF010000540500002F
:10E8100058220120014B40421A6070470C400020F2
:10E8200058220120014B40421A6070470C400020E2
:10E83000F8B5C0460000000001B40248844601BC9F
:10E84000604700BF8903002001B40248844601BC30
:10E85000604700BFE901002001B40248844601BCC2
:10E86000604700BFD904002001B40248844601BCBF
:10E87000604700BF0903002001B40248844601BC80
:10E88000604700BFD904002001B40248844601BC9F
:10E89000604700BF0901002001B40248844601BC62
:10E8A000604700BF8D02002001B40248844601BCCD
:10E8B000604700BF5101002001B40248844601BCFA
:10E8C000604700BF8D04002001B40248844601BCAB
:10E8D000604700BF3504002001B40248844601BCF3
:10E8E000604700BFC100002001B40248844601BC5B
:08E8F000604700BFC5130020C2
:10E8F800281B001046200010281B0010281B0010A1
:10E90800281B0010281B001038240010341C00108D
:10E91800281B0010281B0010281B0010281B0010A3
:10E92800281B0010281B0010281B0010281B001093
:10E93800281B0010281B0010281B0010281B001083
:10E94800281B0010281B0010281B0010281B001073
:10E95800281B0010281B0010281B0010281B001063
:10E96800281B0010281B0010382000109A280010BF
:10E978008A2800107A2800106A280010C42800107D
:10E98800AA280010502800105045315258462D35FD
:10E99800000000005045315258462D330000000059
:10E9A80041505A4D444D00000000000000494445C4
:10E9B800312D31000000000000494445322D32005D
:10E9C8000000000056312C436F6E74726F6C6C65DA
:10E9D800722030310000000030303030300000004C
:10E9E8004E432C436E74722C35562C3132562C32D1
:10E9F80034560000556E6B6E6F776E20636F6D6DC9
:10EA0800616E642E0A0A00006B6973730A000000C5
:10EA1800202020456E746572204B495353206D6F3A
:10EA280064652E0A00000000736176650A00000024
:10EA3800202020536176652073657474696E67734E
:10EA480020746F20666C6173682E0A0072656164B9
:10EA5800203C666C6173682F72616D3E0A0000008D
:10EA6800202020526561642073657474696E677331
:10EA78002066726F6D20464C415348206F722052B9
:10EA8800414D2E0A000000006D7963616C6C2F7394
:10EA9800657276657263616C6C2F64657374696EF8
:10EAA8006174696F6E2F70617468312F706174685A
:10EAB800320A00002020204150525320736574749C
:10EAC800696E67732E0A0000667265712F73707223
:10EAD8006561642F7072652F726174652F706F772E
:10EAE80065722F70612F62616E642E0A000000004B
:10EAF8002020204C6F52612073657474696E6773AF
:10EB08002E0A00004C6F526120415052532072650A
:10EB18006D6F7465207377697463686572207769AF
:10EB28007468206275696C6420696E204B49535380
:10EB380020544E432E0A0000204669726D77617298
:10EB4800652076657273696F6E203A2025730A0016
:10EB58002053697A65206F66207374727563742018
:10EB680020203A2025752E0A0A00000041505253F1
:10EB78002073657474696E67730A000020204D79EC
:10EB88002063616C6C2020202020202020203A2047
:10EB980025730A0020205365727665722063616CC4
:10EBA8006C20202020203A2025730A00202044656C
:10EBB8007374696E6174696F6E20202020203A207A
:10EBC80025730A00202050617468203120202020FD
:10EBD8002020202020203A2025730A002020506180
:10EBE80074682032202020202020202020203A2055
:10EBF80025730A0A000000004C6F52612073657487
:10EC080074696E67730A0000202046726571756525
:10EC18006E6379202020202020203A2025750A00C4
:10EC28002020537072656164696E67466163746F12
:10EC380072203A2025690A002020507265616D62B1
:10EC48006C6520202020202020203A2025690A00F9
:10EC58002020436F64696E6752617465202020200C
:10EC680020203A2025690A0020205478506F7765C3
:10EC7800722020202020202020203A2025690A0008
:10EC88002020506153656C6563742020202020206B
:10EC980020203A2025690A00202042616E647769A5
:10ECA800647468202020202020203A2025750A003E
:10ECB80025630000536F7572636520616464726533
:10ECC80073733A2025730A446967697065617465CE
:10ECD800727320282575293A20257320257320254D
:10ECE800732025730A446174613A2025730A000071
:10ECF8004D6573736167652066726F6D2073657209
:10ED08007665723A2025732028636F6D6D616E6495
:10ED1800202575290A00000041636B6E6F776C65CA
:10ED280064676520726571756573743A2025730A86
:10ED3800000000004572726F72206465636F646939
:10ED48006E672041505253206672616D652E000037
:10ED58007265616400000000666C61736800000001
:10ED680072616D0073617665000000006B697373F2
:10ED780000000000456E746572696E67204B495348
:10ED880053206D6F64652E0A00000000596F7520CE
:10ED980063616E2065786974204B495353206D6F09
:10EDA800646520766961204B49535320636F6D6D0C
:10EDB800616E64203C3078433020307846462030FD
:10EDC8007843303E0A0000006D7963616C6C000086
:10EDD8004D7943616C6C2073657420746F202573C2
:10EDE8002E0A000073657276657263616C6C0000B0
:10EDF80053657276657243616C6C20736574207418
:10EE08006F2025732E0A00007061746831000000BD
:10EE1800506174683120636C65617265642E0A0004
:10EE280050617468312073657420746F2025732EC7
:10EE38000A00000070617468320000005061746854
:10EE48003220636C65617265642E0A0050617468D3
:10EE5800322073657420746F2025732E0A00000019
:10EE6800646573740000000044657374696E6174AE
:10EE7800696F6E2073657420746F2025732E0A00E5
:10EE880066726571000000004552524F523A207474
:10EE9800686174206973206E6F7420612076616CDC
:10EEA80069642076616C75652E0A00004C6F5261AA
:10EEB800206672657175656E637920736574207458
:10EEC8006F2025752E0A000073707265616400005A
:10EED8004C6F526120737072656164696E67206659
:10EEE8006163746F722073657420746F2025752EAA
:10EEF8000A000000707265004C6F526120707265E4
:10EF0800616D626C652073657420746F2025752EA1
:10EF18000A00000072617465000000004C6F5261C5
:10EF280020636F64696E672072617465207365740D
:10EF380020746F2025752E0A00000000706F776519
:10EF4800720000004C6F526120747820706F7765F2
:10EF5800722073657420746F2025752E0A000000D6
:10EF680062616E64000000004C6F52612062616E45
:10EF78006477696474682073657420746F202575DC
:10EF88002E0A0000706100004C6F52612050412031
:10EF980073657420746F2025752E0A00726573746A
:10EFA800617274006C6F72610000000052652D0080
:10EFB80045726173696E6720464C415348207265FB
:10EFC80067696F6E2E2E2E00646F6E650A00000052
:10EFD80057726974696E672073657474696E6773B4
:10EFE80020746F20464C4153482E2E2E00000000FE
:10EFF8004E6F2076616C6964206461746120666F6D
:10F00800756E6420696E20464C415348206D656DCD
:10F018006F72792E205573696E6720646566617515
:10F028006C742076616C7565732E0A00466F756E78
:10F03800642076616C69642073657474696E6773A3
:10F0480020696E20464C415348206D656D6F72797A
:10F058002E0A0000436F6D706F7365204150525344
:10F068002066726F6D204B495353206672616D653F
:10F07800000000005374617274696E67204C6F520F
:10F088006120726164696F0020205B204641494C11
:10F098004544205D0A00000020205B20444F4E4577
:10F0A800205D0A0025730000526563656976656412
:10F0B800207061636B6574202852535349203D20AA
:10F0C800256964426D290A004552524F523A204E32
:10F0D8006F206F7220636F7272757074656420415F
:10F0E800505253206672616D652E0A004E6F207370
:10F0F80070696E6C6F636B732061726520617661F5
:10F10800696C61626C650000486172647761726560
:10F1180020616C61726D20256420616C7265616488
:10F128007920636C61696D656400000048617264F0
:10F1380020617373657274000A2A2A2A2050414E8E
:10F148004943202A2A2A0A00526A00100A6A001033
:10F158000A6A00104A6A00100A6A00100A6A001057
:10F168000A6A00100A6A00100A6A00100A6A001087
:10F178000A6A00103A6A00100A6A0010426A00100F
:10F188000A6A00100A6A0010F46900109C6A0010EC
:10F19800DA710010906A0010DA7100107C6A0010B1
:10F1A800DA710010DA710010DA710010DA710010EB
:10F1B800DA710010DA710010DA710010606A00105C
:10F1C800DA710010DA710010DA710010DA710010CB
:10F1D800DA710010606A0010E86A00109A6900107D
:10F1E8009A6900109A6900109A6900109A690010CB
:10F1F8009A6900109A6900109A6900109A690010BB
:10F208009A6900109A6900109A6900109A690010AA
:10F218009A6900109A6900109A6900109A6900109A
:10F228009A6900109A6900109A6900109A6900108A
:10F238009A6900109A6900109A6900109A6900107A
:10F248009A6900109A6900109A6900109A6900106A
:10F258009A6900109A690010026E0010AE6A0010D8
:10F26800026E00109A6900109A6900109A690010DD
:10F278009A6900109A6900109A6900109A6900103A
:10F288009A6900109A6900109A6900109A6900102A
:10F298009A6900109A6900109A6900109A6900101A
:10F2A8009A690010906C00109A6900109A69001011
:10F2B8009A6900109A6900109A6900109A690010FA
:10F2C8009A6900109A6900109A690010906C0010F1
:10F2D800246C0010906C0010026E0010AE6A0010D2
:10F2E800026E00109A690010906C00109A69001064
:10F2F8009A6900109A6900109A6900109A690010BA
:10F30800906C0010B46B00109A6900109A69001094
:10F31800F86A00109A690010906C00109A69001041
:10F328009A690010906C00106E616E00666E692D0F
:10F3380000000000666E692B00000000666E690020
:10F34800000000000000F03F000000000000244022
:10F3580000000000000059400000000000408F40FD
:10F36800000000000088C34000000000006AF84068
:10F378000000000080842E4100000000D01263418C
:10F388000000000084D797410000000065CDCD4102
:10F3980006005250BBFF3CB6DCF30010060052508A
:10F3A800E182887FC4F3001006005250D3F0754202
:10F3B800BCF3001052656C6561736500626F6F7411
:10F3C800325F77323571303830000000312E332EFD
:10F3D800300000007069636F000000006D61696EA5
:10F3E8000000000041707220323920323032320081
:10F3F8000D0A0000398E00103D8E00104D8E001051
:10F40800758E0010498E0010000000000600525052
:10F4180053B4F4A120F40010555342207374646966
:10F428006E202F207374646F7574000052617370BE
:10F438006265727279205069000000005069636F3C
:10F4480000000000426F61726420434443000000E2
:10F4580052657365740000000902540003010080BE
:10F468007D080B00020202000009040000010202EC
:10F4780000040524002001052401000104240202DF
:10F48800052406000107058103080010090401008E
:10F49800020A000000070502024000000705820278
:10F4A8004000000904020000FF00010512010002EB
:10F4B800EF0201408A2E0A00000101020301000048
:10F4C8000000000034F4001044F40010303D002027
:10F4D8004CF4001058F40010556E68616E646C6549
:10F4E800642049525120307825780A00657020251B
:10F4F800642025732077617320616C72656164797B
:10F5080020617661696C61626C65000043616E27F9
:10F518007420636F6E74696E7565207866657220F5
:10F528006F6E20696E616374697665206570202549
:10F5380064202573000000006F757400696E000078
:10F54800AC9C0010209F0010929E00103C9E001062
:10F558001E9E0010069E0010569D0010FA9C00107A
:10F56800EE9C0010FAA10010E0A100103AA00010D3
:10F578001AA200103AA00010C8A10010B4A10010EF
:10F588003AA00010A0A1001076A100103AA0001027
:10F59800AAA200107EA2001072A200103AA00010C9
:10F5A8003AA0001054A200107EA200103AA0001049
:10F5B8003AA000103AA000103AA000103AA000109B
:10F5C8003AA000103AA0001034A20010B9AD001003
:10F5D80035AE001061AE001045AF001029B0001024
:10F5E80000000000781E0000A0280000F03C000089
:10F5F80040510000127A0000E4A2000024F4000048
:10F6080048E8010090D0030020A107000000000096
:10F618000000000031BA0010E1BB0010C5B90010AD
:10F62800C9B90010CDB9001025BB0010F9BC0010F5
:10F63800080052500A38A504090052500001000081
:0CF648004CF600105350492043530000C2
:10F654003F020181B00300840000000080040181A6
:10F66400B0B0ABF000000000F0800181B0AB08B195
:10F674000000000080160181B0B0ABF00000000073
:10F6840080020181B0B0AB30000000008004018131
:10F69400B0B0AB300000000080010181B0B0AB100D
:10F6A4000000000080060181B0B0ABF00000000053
:10F6B40080030181B0B0AB700000000080080181BC
:10F6C400B0B0ABF00000000080060181B0B0AB30F8
:10F6D4000000000080030181B0B0AB7000000000A6
:10F6E400800A0181B0B0ABF000000000800101810C
:10F6F400B0B0AB100000000080040181B0B0AB30AA
:10F704000000000080040181B0B0AB3000000000B4
:10F7140080060181B0B0ABF00000000080040181DC
:10F72400B0B0ABF00000000080020181B0B0AB309B
:10F734000000000080020181B0B0AB300000000086
:10F7440080020181B0B0AB30000000008004018170
:10F75400B0B0ABF00000000074B20181B0AB3080F7
:10F7640000000000800A0181B0B0ABF0000000008E
:10F774003F020181B0AB30800000000080060181AF
:08F78400B0B0ABF00000000082
:10F78C00D00BFF7F01000000500CFF7FBCFEFF7F01
:10F79C00800CFF7FB0B0A880600DFF7FAB10808025
:10F7AC00EC0EFF7FB0B0A880580FFF7FB0B0AA80DE
:10F7BC00C80FFF7FB0AB3280D415FF7FAB108080B9
:10F7CC00A019FF7F90FEFF7F781EFF7F94FEFF7FC6
:10F7DC002C21FF7FAB1080809C22FF7F010000005A
:10F7EC000C23FF7F88FEFF7F3840FF7F0100000065
:10F7FC00D0C1FF7F84FEFF7F2CC2FF7F88FEFF7F7E
:10F80C0018C3FF7F8CFEFF7FCCC3FF7F90FEFF7F72
:10F81C00DCC4FF7F94FEFF7F00C6FF7F98FEFF7F56
:10F82C0074C9FF7F9CFEFF7F84CBFF7FA0FEFF7F10
:10F83C00CCCCFF7FA4FEFF7FE4CFFF7FA8FEFF7F31
:10F84C0058D0FF7FACFEFF7FC0D1FF7FB0FEFF7FA3
:10F85C0034D3FF7FB4FEFF7FD8D5FF7FB8FEFF7F88
:10F86C0070D8FF7FBCFEFF7F0CD9FF7FC0FEFF7FEF
:10F87C0094D9FF7FC4FEFF7F20DAFF7F01000000D8
:10F88C004CDAFF7FC0FEFF7F2CDFFF7F0100000002
:10F89C00F40CFF0FB0A90280880DFF0FB0B0A88048
:10F8AC00D40DFF0F01000000E00DFF0FB0B0AA80D7
:10F8BC00140EFF0F9CFEFF7FD40EFF0F0100000003
:10F8CC00D00EFF0FAA3F39801C0FFF0FB0B0A880DD
:10F8DC00280FFF0FB0B0AA80680FFF0FB0B0A88040
:10F8EC007C0FFF0F01000000780FFF0FB0B0A88055
:10F8FC00800FFF0F010000000810FF0FAA0FB2804D
:10F90C007010FF0F58FEFF7F4813FF0FB0B0A88098
:10F91C006413FF0F54FEFF7FC015FF0F01000000A2
:10F92C003017FF0F008404804017FF0FB0B0A88081
:10F93C004017FF0F40FEFF7F281AFF0F0084048042
:10F94C00481AFF0FB0B0A880601AFF0F010000002A
:10F95C00B4020010A80200109C02001098F30010D2
:10F96C0090020010A4F30010B0F3001038F6001051
:08F97C0040F6001014F4001025
:10F98400D02330B500251B065D57002406E003682C
:10F99400BFF35F8F1C6081F3108820BF0268EFF310
:10F9A400108172B61368002BFCD0BFF35F8F03790C
:10F9B4007F2BECD905710368BFF35F8F00221A60B7
:10F9C40081F3108830BDC046030010B50068EFF322
:10F9D400108472B60268002AFCD0BFF35F8F042241
:10F9E4009A56002A0BDB00290FD000200A601B68FE
:10F9F400BFF35F8F00221A6084F3108810BDD022F9
:10FA04001206126801201A71F1E70020EFE7C046E0
:10FA1400F0B5C64600B50C00070001F081F9FA22E2
:10FA240005000E00920020000023002101F090F94F
:10FA34002C002A00350024184D41AE422FD9012450
:10FA44006442E517D0231B061B68002698460BE08A
:10FA54003B68BFF35F8F1E6081F31088200029008C
:10FA640001F086F9002818D13A68EFF3108172B6D4
:10FA74001368002BFCD0BFF35F8F3B797F2BE7D952
:10FA840043463B713B68BFF35F8F00221A6081F3EA
:10FA94001088012004BC9046F0BD0020FAE7AE4275
:10FAA400D0D1A242CBD8CDE70268EFF3108172B671
:10FAB4001368002BFCD0BFF35F8FFF23037103682F
:10FAC400BFF35F8F00221A6081F3108840BF704734
:10FAD40030B5094C2378002B0DD180230748084901
:10FAE4005B05F0221D6812069A18043385508B4278
:10FAF400F7D10123237030BD443D00204C35002054
:10FB04000001001010B5024B0133984710BDC046E8
:10FB14004C350020054B1A6880239B005340C022BB
:10FB240092001340024A13607047C0460C800140A3
:10FB34000C900140034B1A68C0239B009343024A74
:10FB4400136070470C8001400C900140F0B5802395
:10FB54004F464646D6464218C0B59B0306000F00E2
:10FB64009A4201D901F0E4F814251824288823883E
:10FB74001149984723888246104928889847238842
:10FB840081460F492888984723880E49804628884B
:10FB940098470400FFF79CFFD047C84780223900EC
:10FBA4003000D8235202C047A047FFF7ABFF1CBC6C
:10FBB40090469946A246F0BD4946000045580000CB
:10FBC4005245000046430000F8B54E465746DE460F
:10FBD40045468023E0B517008218060089469B033A
:10FBE4009A4201D901F0A4F81425182428882388FE
:10FBF40011499847238883461049288898472388C1
:10FC040082460F492888984723880E4980462888C9
:10FC140098470400FFF75CFFD847D0473A004946AD
:10FC24003000C047A047FFF76DFF3CBC90469946A3
:10FC3400A246AB46F8BDC046494600004558000000
:10FC44005250000046430000F0B5D6464F464646A3
:10FC54001423C0B51827984681460D0018882249F8
:10FC64003B881400984743468246204918883B88BD
:10FC7400984743461E49060018883B8898478046A3
:10FC8400FFF726FFD047B047FFF744FFC02022000C
:10FC940008264005163F230013431BD03100836A16
:10FCA40019401F420BD0002C09D0131B0D2B06D872
:10FCB4004B461B78013C036601239C46E144002922
:10FCC400E9D0002AE7D0036E013A2B7023000135F6
:10FCD4001343E3D1FFF72EFFC047FFF713FF1CBC0C
:10FCE40090469946A246F0BD49460000455800009A
:10FCF40046430000F0B5C6468C461D001C00022198
:10FD0400042700B526002E431BD0002D0DD0C66855
:10FD140031420AD02E000836A64206D96646367805
:10FD2400013D86600126B046C444002CEAD0C66872
:10FD34003742E7D08668013C1670260001322E4314
:10FD4400E3D1180004BC9046F0BDC04630B50300B2
:10FD5400002A09D002258818DC682542FCD00C78DA
:10FD640001319C608842F7D1D968490704D504243D
:10FD74009968D9680C42FBD11024D9680C42FCD193
:10FD8400D968490704D504249968D9680C42FBD181
:10FD940001211000196230BD7047C04603685A0043
:10FDA40003D45B005B08C01870478022120613431B
:10FDB400F9E7C046F0B557464E46DE464546E0B53F
:10FDC400814683B09246002925D04B1E9B460027CE
:10FDD40001935B46FB18DC0FE4184B466410E50006
:10FDE4005E193000FFF7DAFF019B8046A3420BD077
:10FDF400280008304844FFF7D1FFD04506D8013821
:10FE0400504509D2671CE4E7504505D9A74202D002
:10FE1400631E9B46DDE70026300003B03CBC9046E1
:10FE24009946A246AB46F0BD012809D0022805D068
:10FE3400002801D0002070470248FCE70248FAE796
:10FE44000248F8E75D0C0020750C0020690C0020C6
:10FE540030B5234B83B005008C1E002B26D001A99E
:10FE6400200000E000BF00281CD001992200FFF709
:10FE7400A1FF041E16D0FFF791FF6368A864012B4D
:10FE84002AD0201D002B23DBFFF788FF0023E86422
:10FE94002B650368002B0FDBFFF780FF2861002030
:10FEA40003B030BD002309202B61F9E70D480E494A
:10FEB400091AC9100191D9E71801000FFFF7B4FF1F
:10FEC4002861431E98410823404298430930E7E7DC
:10FED4000123E8642B65DCE7002305202B61DFE7C1
:10FEE400000000008CF700105CF90010036810B5E6
:10FEF4000400DA0705D448309B070ED500F06CFCEB
:10FF040023685A070ED51A0713D5DB0604D420003C
:10FF1400D130FF3000F06CFC10BD00F059FC2368B8
:10FF24005A07F0D42000D03000F05AFC23681A0796
:10FF3400EBD420005130FF3000F056FC2368E4E796
:10FF44000368002B00D01B18180070470920704765
:10FF54007047C04670B504000D0008E02B6C2A0001
:10FF640063612100012023699847082807D1296C7F
:10FF74002000FFF76DFF0028F0D000F0E1FE072815
:10FF8400FBD10020296CFFF7E3FF281D00F00AFCD9
:10FF9400F0B5CE46474680B5C3682E4C9846A54476
:10FFA4008369060014000431402205A8994600F034
:10FFB400D7FE002304AD049323E0F0222B6C5200FF
:10FFC400736129007CA800F0CBFE7CAA3100336960
:10FFD400200098478A9B07006B6403934B46009567
:10FFE40001933200330021000120C04700281FD1B3
:0CFFF400F0227CA95200280000F0B2FEB0
:020000041001E9
:100000000024082F1FD1296C3000FFF723FF611E49
:100010008C41070009340028D1D0AB6B10216B64F0
:100020004B46214301930095330032000120C04725
:10003000002800D009273800F5239B009D440CBC04
:1000400090469946F0BD072FF4D12000296CFFF7A8
:1000500081FF05A800F0A8FB2CFCFFFF406C704757
:1000600070B5CB6BFAB00B6404000E004022043173
:1000700003A800F077FE01235B42029306E002AA88
:10008000210023699847050008280AD1129B200007
:1000900019000193FFF7DEFE0028F0D009207AB0A6
:1000A00070BD02A8FFF724FF062DF7D13100200014
:1000B000FFF752FF10B58261DA6BC1601A64190054
:1000C0000022FFF767FF10BD436970B50B64C3687A
:1000D00004000D00002B15D10A0023690100022045
:1000E0009847072807D0082803D129002000FFF7E8
:1000F00033FF00F027FE0020296CFFF72BFF281D9F
:1001000000F052FB0122FFF745FF00F01BFEC04646
:10011000C36810B5002B05D0CB6B00220B64FFF732
:1001200039FF10BDFFF79CFFFBE7C0467047C04694
:10013000836810B5002B02D001000120984710BD44
:10014000012906D0002906D003390220012900D94F
:1001500070470120FCE7002B08D10F2A06D8920037
:1001600082185268009B00201A60F1E70220EFE736
:1001700000B585B003AB0A00009300210023FFF710
:10018000DFFF039805B000BD012906D0002906D085
:1001900003390220012900D970470120FCE7002B18
:1001A00008D10F2A06D8009B92001B688218536062
:1001B0000020F1E70220EFE700B585B003AB039222
:1001C00000930A0000230021FFF7DEFF05B000BD09
:1001D00070B51A4CD36BA544136406000D0019A822
:1001E000111D402200F0BEFD01235B42189314E074
:1001F0000C2118A802AAFFF7DFFF290018A8B047B2
:10020000002812D1069B18AA02A90830019398472A
:10021000040005280AD0092807D0289B02A8190045
:100220000193FFF717FE0028E2D0092418A8FFF772
:100230005FFE200090239B009D4470BDC0FDFFFF2A
:10024000F0B5DE4657464E464546E0B51600032259
:100250000D0011008BB01F000193EB6C01401C1DC1
:10026000009107A91B688B460894002F6BD01A0CCD
:100270001B045946079302230B72FD3313409B0066
:100280004A72E418009B022B00D1AC6B2B6DDB078C
:1002900047D4002305930833034002932768002FB7
:1002A00000D112E1019B022B49D063882788984630
:1002B0000434012340469A469843AB6C0F2199467B
:1002C00081443000FFF754FF0021814506D83900F2
:1002D00053469943494488428941494243465A001A
:1002E00002231340012217403B43012B3AD0002B3D
:1002F00030D0022B1BD12368009A5F007F08002AB0
:1003000067D1002906D0029A002A00D17CE0002F94
:1003100000D1A9E0002B00DA04340137BF00E41952
:10032000BCE75946300000F00BFB002810D0092034
:100330000BB03CBC90469946A246AB46F0BD636804
:1003400008349846B5E71B0207935B461A8199E784
:100350000820EDE7009B002B02D0002900D08DE0A3
:1003600004349BE7009B002B1AD1002916D0236888
:10037000DF0F63689A1CDAD02A00583206920133E4
:1003800000D1BDE0201DFFF7DDFD06AB01003A0006
:10039000280000E000BF002800D082E008347DE79C
:1003A0000D2130002F6AFFF7E3FE8742F6D1AB6ADA
:1003B0009C42F3D12000FFF7F3FC0F210200300034
:1003C000FFF7FAFE30002A000021FFF7F5FE0720B4
:1003D000AEE72B6A0D2130009846FFF7C9FE804535
:1003E00001D0236896E7AB6A9C42FAD10023EB6206
:1003F00004332B63231DAF626B632368002B00DA89
:1004000086E00123059388E7002F2DD058239C46D2
:10041000AC4463460393231D99460023984606ABDC
:10042000220004933B004C464746B24698462E00B5
:10043000914603E004342F00454542D0039B200041
:100440000693FFF77FFD049B0100002230007D1C16
:1004500000E000BF0028EDD04346B84635004C46CA
:1004600056461F009845BCD10D213000FFF780FE95
:10047000069B28626B62AC62062059E72000FFF7FA
:100480008FFC04340700AC63280000E000BF0028A4
:1004900000D14CE730003A000F21FFF78DFE072016
:1004A00046E707000D213000FFF762FE2862022FA9
:1004B0002BD1069BEB622B002C336B62AC620620C7
:1004C00036E735004C465646CEE75946300000F038
:1004D00037FA002800D02AE7059B002B00D137E728
:1004E0000F213000FFF744FE0E2102003000FFF71D
:1004F00063FE3000094A0F21FFF75EFE072017E771
:100500000D213000FFF734FE2862069B6B62D5E7B1
:1005100038000130800020184DE7C0460000000080
:1005200010B50023FFF78CFE10BDC04610B50123A7
:10053000FFF786FE10BDC04610B50223FFF780FE10
:1005400010BDC046F0B5CE46474680B50500C3B0E5
:1005500014001E00012955D000294BD0032922D0B8
:10056000042949D1002B47D1102A45D8102203680D
:100570001A4200D0F1E020AF380000F03DF900232E
:100580000120A96B02009A40144203D00E689A0021
:10059000BE5004310133042BF4D13800A96300F0BC
:1005A00029F9002029E0032B26D11404230C160C72
:1005B0009846F318102B1FD8082203681A4200D05F
:1005C00098E020AF380000F013F94246AB6BF6001C
:1005D0001C00002A08D0D400F21A1C19BA18196895
:1005E000D15004339C42FAD1AC63380000F0FEF8DD
:1005F000002002E0002B24D0022043B00CBC904627
:100600009946F0BD130C14049846240C012E2ED0EC
:10061000052EF1D11B19202BEED842460F2A70D996
:10062000A146002C7ED1AA6B4346AA630F2B00D8AB
:100630009AE04B46002BDBD0684600F0D3F8002050
:10064000DBE700231004A96B000C013632009A404E
:10065000104204D00F689A00AA1857600431013381
:10066000102BF3D10020A304C7D4A963C5E71B193D
:10067000102BC1D843460F2BBED82B681E4206D084
:100680000322280093432B60483000F0A5F820AFE8
:10069000380000F0A1F8AA6B002C24D04346DB0000
:1006A000FF180023994664000023A400D158F95094
:1006B00004339C42FAD14B4612196F46002B0FD0DF
:1006C0004046102800D210204B46D9000023103895
:1006D000C0003818D458C45004339942FAD1521883
:1006E000012EA1D120AF04323800AA6300F072F8C5
:1006F000002082E7934303605130FF3000F078F828
:100700005FE7102B3BD910225242914699442B6847
:10071000194208D0022228008B4313432B60483033
:1007200000F05EF82B6804221A4221D143460F2BB9
:1007300003D820AF380000F053F86F46380000F0BF
:1007400053F810244346AA6BE41A002CB8DD434644
:1007500020AFDB006400FF18A6E793430360D130AD
:10076000FF3000F049F806E720A800F037F860E70E
:10077000280093432B60D03000F036F8D6E72B6882
:100780000B4207D0022228008B4313432B604830D2
:1007900000F026F820AF380000F022F8A146AA6B3E
:1007A000002C00D07AE73FE7011C343138C9043B04
:1007B0009C461D60A646011C20313CC990469946C6
:1007C000A246AB46011C0831FCC941680068E546F9
:1007D00000BDC0467047C0467047C0467047C0461F
:1007E0007047C0467047C0467047C0467047C04615
:1007F0007047C0467047C0467047C04601B401A864
:1008000001B585B0FFB408A841464A4653465C4648
:1008100065463EC001A83EC80F98009000230CB466
:1008200001A9FFF71DFC109B12B0184701B401A8E5
:1008300001B585B0FFB408A841464A4653465C4618
:1008400065463EC001A83EC80F98009000230CB436
:1008500001A9FFF739FC109B12B0184701B401A899
:1008600001B585B0FFB408A841464A4653465C46E8
:1008700065463EC001A83EC80F98009000230CB406
:1008800001A9FFF745FC109B12B0184701B401A85D
:1008900001B585B0FFB408A841464A4653465C46B8
:1008A00065463EC001A83EC80F98009000230CB4D6
:1008B00001ABFFF7FFFB109B12B0184701B401A872
:1008C00001B585B0FFB408A841464A4653465C4688
:1008D00065463EC001A83EC80F98009000230CB4A6
:1008E00001AAFFF775FC109B12B01847027A0300AB
:1008F000002A0BD1427A002A0FD0013A4272426894
:10090000111D416003211268017202E0013A027276
:100910000268100E12021A607047B020FCE7C04651
:1009200000B585B003AB00930C2200230021FFF734
:1009300007FC039805B000BD10B5FFF7F1FF10BD2F
:10094000F0B557464E464546DE460023E0B587B033
:1009500003930F339846083B994680231B030600F8
:100960000F009A463800FFF7C1FF0400B02800D1FD
:10097000C3E003062AD5030042469343DBB2802B33
:1009800000D171E0902B3DD0A02B00D185E0B02BA1
:1009900050D0C02B00D196E003004A469343DBB20F
:1009A000D02B0AD15346024001321A4305230121BC
:1009B0003000FFF7C7FD0028D4D00924200007B07D
:1009C0003CBC90469946A246AB46F0BDFF23820050
:1009D00013401D1D05AB9B4600930D2200230021F3
:1009E0003000FFF7ADFB630620D4059B9C466544B1
:1009F00005955B460D220093002100233000FFF790
:100A0000C3FBAFE7833B03400D2BD6D005AD0240BF
:100A10000095002300213000FFF792FB0095002392
:100A20000D2200213000FFF7AFFB9BE7059B5D1B0C
:100A30000595DEE7B12874D0B22800D1CFE0B32805
:100A400000D184E0FC230340B42BB6D04A46534681
:100A5000024001321A43012101233000FFF772FDE9
:100A6000002800D17EE7A8E704023800FFF73EFF28
:100A7000802520432D02A8429FD004010005020CCE
:100A8000002300213000FFF75DFD002895D12C42A6
:100A900000D167E70123039364E7FF234A461B0164
:100AA0001900824311410A001A40030702D580232E
:100AB000DB011A43002300213000FFF743FD00282B
:100AC00000D14FE779E7C6284CD0C7285ED0030095
:100AD0004A469343DBB2C02B6DD0C82872D0C928D8
:100AE00000D06AE73800FFF701FFF02302031B0381
:100AF000134042460240013257E7039B0024002B7B
:100B000000D05BE705AD00950E2200213000FFF715
:100B100017FB009500230F2200213000FFF734FB64
:100B20004CE73800FFF7E2FE002800D145E703005C
:100B300042469343DBB2002B00D03EE70200002187
:100B40003000FFF7FFFC002800D10BE735E7380045
:100B5000FFF7CCFEF02302031B0313404246024082
:100B6000013277E73800FFF7C1FEF02302031B03D1
:100B700013404246024001321A430323032130004E
:100B8000FFF7E0FC002800D1ECE616E73800FFF79D
:100B9000ADFE021E00D110E7030041468B43DBB2DD
:100BA000002B00D009E704213000FFF7CBFC002820
:100BB00000D1D7E601E74346A0221C4001341203CE
:100BC0002243DAE73800FFF791FE434602009A43DA
:100BD000D2B210321840120301300243E6E605ABF0
:100BE00000939B460D22002300213000FFF7A8FA56
:100BF0003800FFF77BFE030618D57F25B03C059B28
:100C00002840A0409C466044059038000734FFF718
:100C10006DFE0306F3D481217F23890003408C46B7
:100C2000A340059A62449B180593E2E60224F2E78A
:100C3000030000B5DB6C85B05A680800120201920F
:100C40001A0001A908324A6003220A72DB794B724A
:100C5000FFF776FE05B000BD10B5FFF76DFE806CA6
:100C600010BDC04610B5FFF767FEC26CD3799B007C
:100C70000833D01810BDC04610B500F063F8C04668
:100C800010B5FFF7F9FFC046F0B588420AD98B18B6
:100C9000984207D2531E002A03D0CA5CC254013BBB
:100CA000FBD2F0BD0F2A09D80500002AF9D0002395
:100CB000CC5CEC5401339342FAD1F2E70D000543CA
:100CC0000C000300AD0729D11500103D2D092F019F
:100CD0003F18103726681E6066685E60A6689E60D2
:100CE000E6681034DE601033BB42F3D10F240135C7
:100CF0002D01491914404519032C11D90023CE5850
:100D0000EE500433E61A032EF9D80323043CA4085A
:100D10000134A4002D1909191A40C6E70500C6E7D9
:100D20002200C2E701B40248844601BC604700BF0C
:100D3000F543001001B40248844601BC604700BF7F
:100D4000994D001001B40248844601BC604700BFC1
:100D500045DD001001B40248844601BC604700BF75
:100D60008588001001B40248844601BC604700BF7A
:100D70006989001001B40248844601BC604700BF85
:100D8000794100100000081010000000E01400205D
:100D900000000000081E002078360020000000003F
:100DA0000000000088360020000000000000000065
:100DB0001000000000000000000001000000000022
:100DC0000000000000000200000000000000000021
:100DD0000000030000000000000000000000FF0011
:100DE0000000000000B5486801318E46004770469B
:100DF00009380149884700BDD152001000000000A9
:100E000000000000503300004C3300005433000059
:100E1000523300004D5300004D4300005334000096
:100E200043340000B18F001000000000198F001043
:100E3000000000000001000040F5001044F5001023
:100E40004C3F002010000C000000E0FF1F000000DD
:100E50000000000000000000000000000000000092
:100E600000000000A81500200000000000000000A5
:100E700094180020FC1800206419002000000000D5
:100E80000000000000000000000000000000000062
:100E90000000000000000000000000000000000052
:100EA0000000000000000000000000000000000042
:100EB0000000000000000000000000000000000032
:100EC0000000000000000000000000000000000022
:100ED0000000000000000000000000000000000012
:100EE0000000000000000000000000000000000002
:100EF00000000000000000000000000000000000F2
:100F000000000000000000000000000000000000E1
:100F10000000000001000000000000000E33CDAB17
:100F200034126DE6ECDE05000B000000000000004E
:100F300000000000000000000000000000000000B1
:100F400000000000000000000000000000000000A1
:100F50000000000000000000000000000000000091
:100F60000000000000000000000000000000000081
:1012900000000000FFFFFFFF000002000000000050
:1012A00000000000D8190020D8190020E019002003
:1012B000E0190020E8190020E8190020F0190020AA
:1012C000F0190020F8190020F8190020001A002059
:1012D000001A0020081A0020081A0020101A002006
:1012E000101A0020181A0020181A0020201A0020B6
:1012F000201A0020281A0020281A0020301A002066
:10130000301A0020381A0020381A0020401A002015
:10131000401A0020481A0020481A0020501A0020C5
:10132000501A0020581A0020581A0020601A002075
:10133000601A0020681A0020681A0020701A002025
:10134000701A0020781A0020781A0020801A0020D5
:10135000801A0020881A0020881A0020901A002085
:10136000901A0020981A0020981A0020A01A002035
:10137000A01A0020A81A0020A81A0020B01A0020E5
:10138000B01A0020B81A0020B81A0020C01A002095
:10139000C01A0020C81A0020C81A0020D01A002045
:1013A000D01A0020D81A0020D81A0020E01A0020F5
:1013B000E01A0020E81A0020E81A0020F01A0020A5
:1013C000F01A0020F81A0020F81A0020001B002054
:1013D000001B0020081B0020081B0020101B002001
:1013E000101B0020181B0020181B0020201B0020B1
:1013F000201B0020281B0020281B0020301B002061
:10140000301B0020381B0020381B0020401B002010
:10141000401B0020481B0020481B0020501B0020C0
:10142000501B0020581B0020581B0020601B002070
:10143000601B0020681B0020681B0020701B002020
:10144000701B0020781B0020781B0020801B0020D0
:10145000801B0020881B0020881B0020901B002080
:10146000901B0020981B0020981B0020A01B002030
:10147000A01B0020A81B0020A81B0020B01B0020E0
:10148000B01B0020B81B0020B81B0020C01B002090
:10149000C01B0020C81B0020C81B0020D01B002040
:1014A000D01B0020D81B0020D81B0020E01B0020F0
:1014B000E01B0020E81B0020E81B0020F01B0020A0
:1014C000F01B0020F81B0020F81B0020001C00204F
:1014D000001C0020081C0020081C0020101C0020FC
:1014E000101C0020181C0020181C0020201C0020AC
:1014F000201C0020281C0020281C0020301C00205C
:10150000301C0020381C0020381C0020401C00200B
:10151000401C0020481C0020481C0020501C0020BB
:10152000501C0020581C0020581C0020601C00206B
:10153000601C0020681C0020681C0020701C00201B
:10154000701C0020781C0020781C0020801C0020CB
:10155000801C0020881C0020881C0020901C00207B
:10156000901C0020981C0020981C0020A01C00202B
:10157000A01C0020A81C0020A81C0020B01C0020DB
:10158000B01C0020B81C0020B81C0020C01C00208B
:10159000C01C0020C81C0020C81C0020D01C00203B
:1015A000D01C0020D81C0020D81C0020E01C0020EB
:1015B000E01C0020E81C0020E81C0020F01C00209B
:1015C000F01C0020F81C0020F81C0020001D00204A
:1015D000001D0020081D0020081D0020101D0020F7
:1015E000101D0020181D0020181D0020201D0020A7
:1015F000201D0020281D0020281D0020301D002057
:10160000301D0020381D0020381D0020401D002006
:10161000401D0020481D0020481D0020501D0020B6
:10162000501D0020581D0020581D0020601D002066
:10163000601D0020681D0020681D0020701D002016
:10164000701D0020781D0020781D0020801D0020C6
:10165000801D0020881D0020881D0020901D002076
:10166000901D0020981D0020981D0020A01D002026
:10167000A01D0020A81D0020A81D0020B01D0020D6
:10168000B01D0020B81D0020B81D0020C01D002086
:10169000C01D0020C81D0020C81D0020D01D002036
:1016A000D01D002000000000000000004D89001047
:1016B000B17B0010C5820010B988001039030010FA
:0C16C000811A0010C1B60010A5D2001065
:04000005100001E9FD
:00000001FF
